:1000000002FF29CFC39FFF50011E22021FDE00FC0A
:10001000F8F0E1C2000096004B00258012C0096094
:1000200068A8E802FDE9A3E004F0700612FF0DE005
:1000300004F02202FE0410AF028003D38001C392B9
:100040000D900DDAE0FEA3E0FFAC23AD24EE420CF0
:10005000EF420D900DDAECF0A3EDF0A20D92AF227D
:1000600010AF028003D38001C3920D900DDAE0FE41
:10007000A3E0FFE523F4FCE524F4FDEE520CEF527F
:100080000D900DDAECF0A3EDF0A20D92AF22900DE1
:10009000DAE0FEA3E0FFAC23AD24EE520CEF520DEC
:1000A000ED4C6002D322C322900DDAE0FEA3E0FF04
:1000B000AC23AD24EE520CEF520DAA23AB24EDB5C8
:1000C0000B06ECB50A02D322C322852381752300D7
:1000D0002210AF028003D38001C3920D900925E066
:1000E000B4010A900925E4F0852399802C900DAB8A
:1000F000E0FEA3E0FF0FBF00010E7C037DFFEE5288
:100100000CEF520D900DABECF0A3EDF08C0E8D0FBB
:100110009009A912FF02E523F0A20D92AF228524D7
:1001200083852582E06013852483852582E0F5237D
:100130001200D1782412FF4280E422852483852591
:1001400082E4936014852483852582E493F5231249
:1001500000D1782412FF4280E222901295E4F0E56B
:1001600027452670030201E8E5287038AE26AF2740
:1001700074108E0C8F0DFF12FEEB8C0E8D0F90E025
:10018000FA12FF02FEE493FFEE901295E0901284C3
:1001900012FF17EFF0AE26AF27740412FEC38E26AF
:1001A0008F27803BAE26AF27740A8E0C8F0DFF126F
:1001B000FEEB8C0E8D0F90E0FA12FF02FEE493FF2F
:1001C000EE901295E090128412FF17EFF0AE26AF7A
:1001D00027740A8E0C8F0DFF12FE768C268D2790C9
:1001E0001295E004F002015F901295E090128412E3
:1001F000FF177430F0E528700B901295E00454FE60
:10020000901295F0901295E0C39529502790129482
:100210007401F0901294E0FE901295E0F404252908
:10022000C39E40107430F5231200D1901294E02444
:1002300001F050DF901295E06018901295E014F0F4
:10024000901295E090128412FF17E0F5231200D16E
:1002500080E2AE2AAF2B8E248F2512013B22AE2CDA
:10026000AF2D8E548F557556127557A612F94A75D3
:10027000541075553BAE2CAF2D8E568F5712F90783
:10028000B40110742DF5231200D17554127555A6C2
:1002900012FA38E52E9018FDF82828739012A6E07F
:1002A000F5277526007528007402F529752AE17571
:1002B0002B1512015A9012A7E0F527752600752814
:1002C000007402F529752AE1752B1512015A901256
:1002D000A8E0F5277526007528007402F529752A0F
:1002E000E1752B1512015A802875541275559675B3
:1002F00056127557A612F98D75241275259612019E
:100300001E800E800C800A80088006800480028097
:1003100000AE2FAF308E248F2512013B2275541270
:100320007555A975560E75570B12F98D9012B1E4DB
:10033000F09012B1E0D3940750249012B1E09012E3
:10034000A912FF17E0C39430FE9012B1E090127A28
:1003500012FF17EEF09012B1E02401F050D32210FA
:10036000AE028003D38001C3920DAE24AF2574800A
:10037000520F7E00EF4E605D900EDAE014541F9035
:100380000EDAF0900EDAE07F07900EDC12FE86E5C2
:1003900023F0900EDAE07F07900EDD12FE86E52452
:1003A000F0A3E525F0900EDAE07F07900EDF12FE55
:1003B00086E527F0AE28AF298E548F55900EDAE0EF
:1003C0007F07900EE012FE86AE83AF828E568F5767
:1003D00012F94A805B900EDBE07F07900EDC12FE84
:1003E00086E523F0900EDBE07F07900EDD12FE869F
:1003F000E524F0A3E525F0900EDBE07F07900EDF0B
:1004000012FE86E527F0AE28AF298E548F55900E48
:10041000DBE07F07900EE012FE86AE83AF828E5641
:100420008F5712F94A900EDBE004541F900EDBF058
:10043000A20D92AE22C28C901073E526F0A3E527A0
:10044000F0A20E9205900DC8E0B4031B7524A075B0
:1004500025D712013B75252675240012011E75242F
:10046000E175250A12013BE581149012B2F0901259
:10047000B2E0F8900DC6E6F0A308E6F0E581C3947B
:1004800002F58122900DB2E0FEA3E0FFAC23AD2483
:10049000EF2DFDEE3CFC900DB2ECF0A3EDF0E5810C
:1004A000149012B3F09012B3E0F8900DC6E6F0A3EA
:1004B00008E6F0E581C39402F58122900DC6E0FEC6
:1004C000A3E0FFEF4E601CE581149012B4F090128F
:1004D000B4E0F8900DC6E0F608A3E0F6900DC6E48F
:1004E000F0A3F022222222900DCF74A0F0A374E199
:1004F000F0900DCDE4F07E027F008E238F24120059
:1005000036900DCCE4F0900DD9E4F022C20F229089
:100510001027E0700C901026E07006901028E06024
:10052000028003C20F22901022E0FEA3E0FFEF4EF4
:10053000701774F8900DCAF0901027E4F09010280E
:10054000E4F0901026E4F0800690102212FEB5D25E
:100550000F22308C1130040690106FE0600280038F
:10056000C20F22D20F22901071E0FEA3E0FFEF4EE7
:10057000600A901071E4F0A3F0D20F22901073E0A3
:10058000FEA3E0FFEF4E600CD28D901073E4F0A359
:10059000F0D20F22C20F22900DC8E0D39401402167
:1005A0007524C37525B012013BE52CF5277526008F
:1005B0007401F5287401F529752AE1752B0A1201D9
:1005C0005AE52C90191BF82828737526B27527D088
:1005D000C3920E120435807C7526B37527C0C39272
:1005E0000E120435806E7526B47527B0C3920E12B4
:1005F000043580607526B57527A0C3920E120435A8
:1006000080527526B6752790C3920E120435804429
:100610007526B7752780C3920E120435803675266D
:10062000B8752770C3920E12043580287526B975E7
:100630002760C3920E120435801A7526BA752750AA
:10064000C3920E120435800C7526BB752740C392E9
:100650000E1204352274649012CDF8E4F0E8A3F091
:100660001204BB900DD9E0901939F8282873020ABA
:10067000CE900DCCE0B4101D900DCF74C3F0A374D8
:10068000BCF0900DCE7401F0900E31E4F0900E2984
:100690007401F08023900DCCE0B4111C900DCF7448
:1006A000C3F0A374EAF0900DCE7401F0900E317493
:1006B00001F07405900E29F0740290000CF0901077
:1006C00070F07428900E1DF0900DCE7401F0900D16
:1006D000CDE4F0900DD9E4F0020ACE7526A275277C
:1006E000E0C3920E120435900DD9E4F0020ACE90C8
:1006F0000DC8E0603D900DCCE0B410097524C475C0
:10070000251712013B900DCCE0B411097524C47576
:10071000253A12013B900DE0E0FEA3E0FF8E268F0C
:10072000277401F5287402F529752AE1752B0A1240
:10073000015A900DE0E0FEA3E0FF74016F4E6006E9
:1007400074066F4E700C7526A1752700C3920E12A9
:100750000435900DE0E0FEA3E0FF740C6F4E700CCA
:100760007526C27527C0C3920E120435900DE0E0C5
:10077000FEA3E0FF74166F4E700C7526A9752770E6
:10078000C3920E120435900DE0E0FEA3E0FF741753
:100790006F4E700C7526AA752760C3920E12043531
:1007A000900DE0E0FEA3E0FF74256F4E700C7526FF
:1007B000AB752750C3920E120435900DE0E0FEA3F6
:1007C000E0FF741C6F4E700C7526AC752740C39209
:1007D0000E120435900DE0E0FEA3E0FF74186F4E9A
:1007E000700C7526AD752730C3920E120435900D2E
:1007F000E0E0FEA3E0FF74196F4E700C7526AE7535
:100800002720C3920E120435900DE0E0FEA3E0FF16
:10081000741A6F4E700C7526B0752700C3920E12B5
:100820000435900DE0E0FEA3E0FF741B6F4E700CEA
:100830007526AF752710C3920E120435900DE0E0B7
:10084000FEA3E0FF74246F4E700C7526B07527F080
:10085000C3920E120435900DE0E0FEA3E0FF742376
:100860006F4E600674346F4E700C7526B17527E0BC
:10087000C3920E120435900DE0E0FEA3E0FF743742
:100880006F4E60030209297554127555C475560ED2
:1008900075573512F98D9012B7E4F09012B7E0D386
:1008A000940750249012B7E09012C412FF17E0C3CF
:1008B0009430FE9012B7E090127A12FF17EEF0908B
:1008C00012B7E02401F050D3901280E0603B75260F
:1008D000C17527D0C3920E1204359012CDE0FEA34D
:1008E000E0FF8E238F24120484901280E09012CFB8
:1008F000F09012CFE0F52C1205979012CDE0FEA3F8
:10090000E0FF8E238F24120484901281E09012CF96
:10091000F09012CFE0F52C1205979012CDE0FEA3D7
:10092000E0FF8E238F24120484900DD9E4F0020A94
:10093000CE900DC8E060257524C475256212013B78
:10094000900DE0E0FEA3E0FF8E268F27752801744E
:1009500002F529752AE1752B0A12015A900DE0E083
:10096000FEA3E0FF74806F4E600674FF6F4E70321E
:10097000900DDEE0FCA3E0FD7A017B00EC520AED75
:10098000520BEB4A600E7526A17527F0C3920E122A
:100990000435800C7526A57527B0C3920E12043558
:1009A0008064900DDEE0FEA3E0FF7401520F7E0034
:1009B000EF4E7046900DE0E0FEA3E0FF74156F4E21
:1009C000700E7526A37527D0C3920E1204358028A9
:1009D000900DE0E0FEA3E0FF740A6F4E700E7526E6
:1009E000A27527E0C3920E120435800C7526A875F7
:1009F0002780C3920E120435800C7526A47527C07B
:100A0000C3920E120435900DD9E4F0020ACE900D77
:100A1000D9E4F0020ACE900DD9E4F0020ACE900D8E
:100A2000D9E4F0020ACE900DD9E4F0020ACE900D7E
:100A3000C8E060267524C475257D12013B900DE049
:100A4000E0FEA3E0FF8E268F277401F5287402F5DF
:100A500029752AE1752B0A12015A7400900E34F0A0
:100A6000900E32F8E4F0E8A3F0900DE1E09019B1B7
:100A7000F828287380537526BD752720C3920E125F
:100A8000043580457526BE752710C3920E120435B5
:100A90008037900DC8E060097524C475259D12014A
:100AA0003B7526BF752700C3920E120435801A7558
:100AB00026BF7527F0C3920E120435800C7526C030
:100AC0007527E0C3920E120435900DD9E4F0229000
:100AD0000DC8E060217524DE7525BB12013BE52CB5
:100AE000F5277526007401F5287401F529752AE1AA
:100AF000752B0A12015AE52C901957F8282873759E
:100B000026D175275FC3920E120435807C7526D2DC
:100B1000752713C3920E120435806E7526D2752781
:100B2000C7C3920E12043580607526D375277BC328
:100B3000920E12043580527526D475272FC3920E5B
:100B400012043580447526D47527E3C3920E12042F
:100B50003580367526D5752797C3920E12043580D9
:100B6000287526D675274BC3920E120435801A7548
:100B700026D67527FFC3920E120435800C7526D732
:100B80007527B3C3920E120435221204BB7464900D
:100B900012D9F8E4F0E8A3F0900DD9E0901975F8B7
:100BA00028287302107B900DCCE0B40F1B900DCF62
:100BB00074DEF0A374D3F0900DCE7401F0900E317A
:100BC000E4F0900E297401F0900DCCE0B4121C906A
:100BD0000DCF74DEF0A374F9F0900DCE7401F09097
:100BE0000E317401F0742C900E29F0740390000CF7
:100BF000F0901070F0900DCDE4F0900DD9E4F0027B
:100C0000107B900DCCE0B4121B900DC8E06009750C
:100C100024DF75252012013B7526D975271BC39249
:100C20000E120435900DCCE0B40F0C7526C5752757
:100C30006BC3920E120435900DD9E4F002107B9034
:100C40000DC8E060267524DF75253312013B900D39
:100C5000E0E0FEA3E0FF8E268F277401F5287402E2
:100C6000F529752AE1752B0A12015A900DE0E0FE74
:100C7000A3E0FF74166F4E700C7526CA752757C314
:100C8000920E120435900DE0E0FEA3E0FF74176FA2
:100C90004E700C7526CB75270BC3920E120435903F
:100CA0000DE0E0FEA3E0FF74256F4E700C7526CBBF
:100CB0007527BFC3920E120435900DE0E0FEA3E04D
:100CC000FF741C6F4E700C7526CC752773C3920E83
:100CD000120435900DE0E0FEA3E0FF74186F4E7033
:100CE0000C7526CD752727C3920E120435900DE0A2
:100CF000E0FEA3E0FF74196F4E700C7526CD7527CA
:100D0000DBC3920E120435900DE0E0FEA3E0FF7409
:100D10001A6F4E700C7526CF752743C3920E1204BE
:100D200035900DE0E0FEA3E0FF741B6F4E700C7574
:100D300026CE75278FC3920E120435900DE0E0FE8B
:100D4000A3E0FF74246F4E700C7526CF7527F7C390
:100D5000920E120435900DE0E0FEA3E0FF74236FC5
:100D60004E700C7526D07527ABC3920E12043590C9
:100D70000DE0E0FEA3E0FF743D6F4E700C7526D8C9
:100D8000752767C3920E120435900DE0E0FEA3E0D4
:100D9000FF74016F4E600674066F4E700C7526D995
:100DA0007527CFC3920E120435900DE0E0FEA3E04C
:100DB000FF740C6F4E700C7526DA752783C3920E84
:100DC000120435900DE0E0FEA3E0FF74216F4E7039
:100DD0000C7526DB752737C3920E120435900DE093
:100DE000E0FEA3E0FF74206F4E700C7526DB7527C4
:100DF000EBC3920E120435900DE0E0FEA3E0FF7409
:100E0000546F4E700C7526DC75279FC3920E12042A
:100E100035900DE0E0FEA3E0FF74376F4E600302F3
:100E20000EC4900DC8E060097524DF75254F1201CE
:100E30003B7554127555D075560E75573512F98D90
:100E40009012B7E4F09012B7E0D3940750249012B8
:100E5000B7E09012D012FF17E0C39430FE9012B7A3
:100E6000E090127A12FF17EEF09012B7E02401F032
:100E700050D3901280E06020901280E09012DBF05E
:100E80009012DBE0F52C120ACF9012D9E0FEA3E01D
:100E9000FF8E238F24120484901281E09012DBF0E5
:100EA0009012DBE0F52C120ACF9012D9E0FEA3E0FD
:100EB000FF8E238F241204847526CC752773C3926A
:100EC0000E120435900DD9E4F002107B900DC8E0AD
:100ED00060437524DF75255F12013B900DDEE0FE57
:100EE000A3E0FF8E268F277401F5287402F529757B
:100EF0002AE1752B0D12015A900DE0E0FEA3E0FFF0
:100F00008E268F277401F5287402F529752AE1755C
:100F10002B0A12015A900DE0E0FEA3E0FF74806FEF
:100F20004E600674FF6F4E7033900DDEE0FCA3E060
:100F3000FD7A017B00EC520AED520BEB4A600E7514
:100F400026C47527B7C3920E120435800C7526C7C8
:100F5000752787C3920E120435021053900DDEE000
:100F6000FEA3E0FF7401520F7E00EF4E60030210FB
:100F70002B900DC8E060437524DF75258112013B7D
:100F8000900DDEE0FEA3E0FF8E268F277401F5288A
:100F90007402F529752AE1752B0D12015A900DE0A6
:100FA000E0FEA3E0FF8E268F277401F5287402F57A
:100FB00029752AE1752B0A12015A900DE0E0FEA373
:100FC000E0FF740A6F4E701D900DC8E06009752433
:100FD000DF7525AB12013B7526C575276BC3920ED5
:100FE0001204358044900DE0E0FEA3E0FF740E6F24
:100FF0004E700E7526DD752753C3920E1204358090
:1010000028900DE0E0FEA3E0FF74156F4E700E75A2
:1010100026C675271FC3920E120435800C7526C98B
:101020007527A3C3920E1204358028900DE0E0FED0
:10103000A3E0FF740F6F4E700E7526DE752707C391
:10104000920E120435800C7526C67527D3C3920EF6
:10105000120435900DD9E4F08021900DD9E4F08090
:101060001A900DD9E4F08013900DD9E4F0800C9023
:101070000DD9E4F08005900DD9E4F022741B900E98
:1010800028F0C2C675F9F075E900D2C6900DCCE023
:1010900090DFC212FEA6783112FF20783112FE2FA7
:1010A000900DB2E0FEA3E0FFEF4E6008D20F900D6E
:1010B000B212FEB5900DC8E0B4040C900DB2E0FE83
:1010C000A3E0FFEF4E7002801D900DB2E0FEA3E0A2
:1010D000FF8E268F277401F5287406F529752AE1FD
:1010E000752B0A12015A300F03021541900EDAE0F7
:1010F000FE900EDBE06E6012900DD9E0700C900D4A
:10110000C6E0FEA3E0FFEF4E600302152D900EDA5D
:10111000E07F07900EDD12FE86E0F8A3E0900DDE82
:10112000C8F0A3C8F07410F52475230012008EC017
:10113000D0900DDEE0FEA3E0FF7402520F7E00EFC0
:101140004E6003D38001C392F0D0D082F0500302EE
:10115000152D900EDAE07F07900EDC12FE86E090EF
:101160000DD9F0900EDAE07F07900EDF12FE86E0D8
:10117000900DE0F8E4F0E8A3F0900EDAE07F07903D
:101180000EE012FE86AE83AF828E548F5575560DDB
:101190007557E212F94A900EDAE004541F900EDA05
:1011A000F0900DCDE06003021284900DC8E0B4040D
:1011B000028003021284E4A20F33F527752600751E
:1011C00028007401F529752AE1752B0F12015A9038
:1011D0000DD9E0F5277526007528007402F52975EC
:1011E0002AE1752B0F12015A900DC6E0FEA3E0FF15
:1011F0008E268F277528007404F529752AE1752B32
:101200000F12015A900DDAE0FEA3E0FF8E268F2721
:101210007528007404F529752AE1752B0F12015AFF
:10122000900DD9E0F5277526007528007402F52980
:10123000752AE1752B0D12015A900DDEE0FEA3E038
:10124000FF8E268F277528007402F529752AE1750F
:101250002B0D12015A900DE0E0FEA3E0FF8E268FC9
:10126000277528007402F529752AE1752B0D1201E6
:101270005A752C0D752DE27400F52E752FE1753021
:101280000A12025E900DD9E0901993F82828730293
:10129000152B900DE1E0900DCCF002152B02152BD3
:1012A000900DC8E0B401417524E075253212013B70
:1012B000900DDEE0FEA3E0FF8E268F2775280174D7
:1012C00002F529752AE1752B0D12015A900DE0E007
:1012D000FEA3E0FF8E268F277528017404F529757B
:1012E0002AE1752B0A12015A02152B900DC8E060F5
:1012F000417524E075255012013B900DDEE0FEA300
:10130000E0FF8E268F277528017402F529752AE1E2
:10131000752B0D12015A900DE0E0FEA3E0FF8E2622
:101320008F277528017404F529752AE1752B0A1297
:10133000015A900DDEE0FEA3E0FF7402520F7E0022
:10134000EF4E6039900DDEE0F8A3E0900E0EC8F08D
:10135000A3C8F075540D7555E275560E75570B12EE
:10136000F94A7410F524752300120036900DE0E060
:10137000FEA3E0FFEF4E7005900DD9E4F0900DDE76
:10138000E0FEA3E0FF7401520F7E00EF4E700D7E71
:10139000107F008E238F241200368009752310756C
:1013A0002400120060900DDEE0F8A3E09012B8C8AF
:1013B000F0A3C8F0900DE0E0F8A3E09012BAC8F0F6
:1013C000A3C8F002152B900DDEE0FEA3E0FF74022F
:1013D000520F7E00EF4E6065900DE0E0FEA3E0FF4F
:1013E00074016F4E702A900DDEE0F8A3E0900E04B9
:1013F000C8F0A3C8F075540D7555E275560D7557B4
:10140000FE12F94A7420F524752300120036802854
:10141000900DDEE0F8A3E0900E06C8F0A3C8F075CA
:10142000540D7555E275560E75570112F94A744000
:10143000F524752300120036900DD9E4F002152B27
:10144000900DC8E060417524E075256E12013B9057
:101450000DDEE0FEA3E0FF8E268F277528017402C3
:10146000F529752AE1752B0D12015A900DE0E0FE69
:10147000A3E0FF8E268F277528017404F529752AAD
:10148000E1752B0A12015A900DDEE0FEA3E0FF7415
:1014900002520F7E00EF4E6038900DE0E0FEA3E0B8
:1014A000FF74106F4E7028900DDEE0F8A3E0900EF0
:1014B0000EC8F0A3C8F075540D7555E275560E753B
:1014C000570B12F94A7410F5247523001200368068
:1014D0002C900DE0E0FEA3E0FF74106F4E701E90A4
:1014E0000DDEE0F8A3E0900E0EC8F0A3C8F075542E
:1014F0001075553B75560E75570B12F94A802C9096
:101500000DE0E0FEA3E0FFEF4E7005900DD9E4F092
:101510008019900DE0E0FEA3E0FFEF4E7005900D06
:10152000D9E4F080067409900DD9F08000900DCCBC
:10153000E090DFFA12FEA6783312FF20783312FE15
:101540002F900DDC120026900DDCE0FEA3E0FF746E
:10155000C8BE00039F50107523027524001200605E
:10156000900DDCE4F0A3F0901068E4F0A2B7400A1C
:10157000901068E04401901068F0A2B6400A901004
:1015800068E04402901068F0A2B5400A901068E04C
:101590004404901068F0A2B3400A901068E0440838
:1015A000901068F0A2A6400A901068E044109010D5
:1015B00068F0A2A5400A901068E04420901068F0FE
:1015C000A2A4400A901068E04440901068F0A2A3E2
:1015D000400A901068E04480901068F0901069E430
:1015E000F0A2A2400A901069E04401901069F0A2B4
:1015F000A1400A901069E04402901069F0A2A04056
:101600000A901069E04404901069F0A295400A9095
:101610001069E04408901069F0A294400A901069A3
:10162000E04410901069F0A293400A901069E044E1
:1016300020901069F0A292400A901069E044409016
:101640001069F0A291400A901069E04480901069FE
:10165000F09012C3E4F0901069E0600E74029012F2
:10166000C2F0901069E09012C3F0901068E0600E34
:101670009012C27401F0901068E09012C3F0900EC6
:10168000D1E0FE9012C3E06E603F9012C3E0900E76
:10169000D1F0900E1FE004F0900DC8E0B4032A755D
:1016A00024E075258D12013B900E1FE0F52775266D
:1016B000007401F5287403F529752AE1752B0A12C7
:1016C000015A742EF5231200D1900E1FE070030210
:1016D0001840900ED1E0FE9012C3E0B50E028003D8
:1016E00002183B900E1FE004F0900DC8E0600774F4
:1016F0002CF5231200D1900E1FE0FE900004E0D3E1
:101700009E4003021834900E1FE4F09012C2E0B421
:1017100002067402900E1EF09012C2E0B401069010
:101720000E1E7401F0900ED1E0900E21F0900DC8C5
:10173000E0B4030280030217F07524E175250A1254
:10174000013B7524E075259F12013B900E1FE0F5CB
:10175000277526007400F5287402F529752AE175AD
:101760002B0D12015A900E1EE0F52775260074000D
:10177000F5287402F529752AE1752B0D12015A908E
:101780000E23E0F5277526007400F5287402F5296C
:10179000752AE1752B0D12015A900E21E0F527757F
:1017A00026007400F5287402F529752AE1752B0AC4
:1017B00012015A7524E07525D712013B9012C2E040
:1017C000F5277526007400F5287402F529752AE1BD
:1017D000752B0D12015A9012C3E0F527752600747F
:1017E00000F5287402F529752AE1752B0A12015AB1
:1017F000900DC8E0603C9012C2E0B401077447F558
:10180000231200D19012C2E0B402077467F52312CC
:1018100000D1900E21E0F52775260075280074028E
:10182000F529752AE1752B0A12015A743EF5231227
:1018300000D18005900E1EE4F08005900E1FE4F0AC
:10184000900E21E06008A2A74002D2A78007A2A7BD
:10185000B34002C2A775540E7555417556107557A1
:101860003B12F907B4010975540E75554112F96719
:10187000901282120026901282E0FEA3E0FF740113
:101880006F4E7002D2A7901282E0FEA3E0FF746454
:101890006F4E7002C2A7901282E0FEA3E0FFEFD36A
:1018A0009488EE94134007901282E4F0A3F07554EC
:1018B0000D7555B412FA139012B7E4F09012B7E018
:1018C000D39401503575540D7555B49012B7E07F1F
:1018D00003900DB712FE86AE83AF828E568F5712DD
:1018E000F907700D9012B7E0900DBD12FF1774014B
:1018F000F09012B7E02401F050C2C2C72202029C4D
:101900000202E902030302030502030702030902BC
:10191000030B02030D02030F0203110205CA0205A5
:10192000D80205E60205F402060202061002061EAF
:1019300002062C02063A02064802066E02067102F0
:1019400006DB0206EF020931020A0E020A16020A3B
:101950001E020A26020A2E020AFF020B0D020B1BB0
:10196000020B29020B37020B45020B53020B6102DB
:101970000B6F020B7D020BA3020BA6020C02020CE2
:101980003F020ECC02105A02106102106802106F62
:1019900002107602128F02129202129D0212A0020F
:1019A00012EB0213C60214400214FF0215120215B4
:1019B00025020A74020A76020A84020A92020AAF17
:1019C000020ABD75A220A84CA94D854E83854F8281
:1019D0008550E012FFF075A2002285A8E0854CA892
:1019E00032854E83854F82E0F8A3E0F9A3E0FA85C3
:1019F0004C83854D82E0FBA3E0FCA3E02AFAEC399E
:101A0000F9EB38854C83854D82F0A3E9F0A3EAF029
:101A100022E4F8F9FAAF50854C83854D82E0A3C3E8
:101A20009430F5F05003021AC7200047940AB350CF
:101A300003021AC7E8FCE9FDEAFEC3CA33CAC93388
:101A4000C9C833C8C3CA33CAC933C9C833C8CA2E00
:101A5000CAC93DC9C83CC8C3CA33CAC933C9C833D7
:101A6000C8E5F0CA2ACAC93400C9C83400C8DFAD05
:101A7000021AB8940AE5F0400D9411404A9406B356
:101A80004045E5F09407C3CA33CAC933C9C833C84F
:101A9000C3CA33CAC933C9C833C8C3CA33CAC933AE
:101AA000C9C833C8C3CA33CAC933C9C833C84AFA54
:101AB000DF03021AB8021A1D854E83854F82E8F0B3
:101AC000A3E9F0A3EAF0C322854C83854D82E0F8B8
:101AD000A3E0F9A3E0FA854E83854F8275F000E01C
:101AE0006830E70375F003E0C39840157018A3E071
:101AF000C399400D7010A3E0C39A400570087400AC
:101B000022740165F022740265F022854C83854DB4
:101B100082E0F8A3E0F9A3E0FA854E83854F82E8DE
:101B2000F0A3E9F0A3EAF022854C83854D82E0F82A
:101B3000A3E0F9A3E0C39401FAE99400F9E8940062
:101B4000854C83854D82F0A3E9F0A3EAF022854E0F
:101B500083854F82E0A3F8E0A3F9E0FA854C838502
:101B60004D827C987D967E80121D4FE5532430F087
:101B7000A37C0F7D427E40121D4FE5532430F0A31D
:101B80007C017D867EA0121D4FE5532430F0A37C9E
:101B9000007D277E10121D4FE5532430F0A37C00FA
:101BA0007D037EE8121D4FE5532430F0A37C007DB9
:101BB000007E64121D4FE5532430F0A37C007D00AD
:101BC0007E0A121D4FE5532430F0A3EA2430F0A31F
:101BD0007400F022854C83854D82E0F8A3E0F9A3E0
:101BE000E02401FAE93400F9E83400854C83854D9E
:101BF00082F0A3E9F0A3EAF022854C83854D82E0D0
:101C0000F8A3E0F9A3E0F42401FAE9F43400F9E8D8
:101C1000F43400854C83854D82F0A3E9F0A3EAF00B
:101C200022854E83854F82E0F8A3E0F9A3E0FAAB6A
:101C30004CAC4DEA8CF0A485F05375520075510000
:101C4000E98CF0A42553F553E5F03552F552E551F2
:101C50003400F551EA8BF0A42553F553E5F03552E5
:101C6000F552E5513400F551E98BF0A42552F552B7
:101C7000E5F03551854E83854F82F0A3E552F0A300
:101C8000E553F022854C83854D82E0540FFBA3E0A1
:101C9000540375F00AA42BFEA3E0540FFBA3E054F9
:101CA0000775F00AA42BFDA3E0540FFBA3E0540733
:101CB00075F00AA42BFCA3E0540FFBA3E0540375BA
:101CC000F00AA42BFAC0E0780079007B3C121DB525
:101CD000ECCA2ACAC93400C9C83400C8121DB5EDFF
:101CE000CA2ACAC93400C9C83400C87B1E121DB52F
:101CF000EECA2ACAC93400C9C83400C8D0E0021DDF
:101D00000FC394174009C3E9948DF9E89427F88527
:101D10004E83854F82E8F0A3E9F0A3EAF022854ED6
:101D200083854F82E0F8A3E0F9A3E0FA854C838530
:101D30004D82E0FBA3E0FCA3E0C39AFAEC99F9EB37
:101D400098854C83854D82F0A3E9F0A3EAF02288C0
:101D50005189528A53780079007A007F19C3CA9E4C
:101D6000CAC99DC9C89CC8401ED3C55333C553C5F5
:101D70005233C552C55133C551CA33CAC933C9C814
:101D800033C8DFD9021DABCA2ECAC93DC9C83CC879
:101D9000C3C55333C553C55233C552C55133C5515D
:101DA000CA33CAC933C9C833C8DFB2C813C8C913D4
:101DB000C9CA13CA22EA8BF0A4FAAFF0E98BF0A4E7
:101DC0002FF9E5F03400FFE88BF0A42FF82210AFD4
:101DD000028003D38001C39213900925E0B4010A65
:101DE000900925E4F0854399802C900DABE0FEA38B
:101DF000E0FF0FBF00010E7C037DFFEE5214EF5297
:101E000015900DABECF0A3EDF08C168D179009A991
:101E100012FF02E543F0A21392AF22854483854569
:101E200082E4936014854483854582E493F54312EC
:101E30001DCE784412FF4280E2229012F1E4F0E5D8
:101E40004745467003021EC8E5487038AE46AF47A6
:101E500074108E148F15FF12FEEB8C168D1790E008
:101E6000FA12FF02FEE493FFEE9012F1E09012E00E
:101E700012FF17EFF0AE46AF47740412FEC38E4652
:101E80008F47803BAE46AF47740A8E148F15FF1202
:101E9000FEEB8C168D1790E0FA12FF02FEE493FF22
:101EA000EE9012F1E09012E012FF17EFF0AE46AFA5
:101EB00047740A8E148F15FF12FE768C468D47905C
:101EC00012F1E004F0021E3F9012F1E09012E012D5
:101ED000FF177430F0E548700B9012F1E00454FEE7
:101EE0009012F1F09012F1E0C3954950279012F052
:101EF0007401F09012F0E0FE9012F1E0F404254934
:101F0000C39E40107430F543121DCE9012F0E024B1
:101F100001F050DF9012F1E060189012F1E014F03F
:101F20009012F1E09012E012FF17E0F543121DCE7F
:101F300080E2AE4AAF4B8E448F45121E1B22854372
:101F40008175430022309849C298E599B41B0890E6
:101F50000926E064016002801EC2AF90FE4E12FEB0
:101F60001F90FE4E12FE1F90FE4E12FE1F900DADF2
:101F7000E0F58175D000229009A8E004547F900913
:101F8000A8F09009A8E090092712FF17E599F080C2
:101F9000B4309949C299900DA9E0FEA3E0FF900DDD
:101FA000ABE0FCA3E0FDEF6D7004EE6C60290FBFA9
:101FB00000010E7A037BFFEE5212EF5213900DA92F
:101FC000EAF0A3EBF08A168B179009A912FF02E042
:101FD000F54385439980069009257401F022C0E0FD
:101FE000C0F0C083C082C0D075D01812FB32D0D0F0
:101FF000D082D083D0F0D0E032FFFFFFFFFFFFFFA1
:102000000FFFFF0132047909303905FF040078FF22
:1020100053545550FFFFFFFFFFFFFFFFFFFFFFFF80
:10202000FFFFFFFFFFFFFFFFFFFFFFFFFFFFFFFFC0
:10203000FFFFFFFFFFFFFFFFFFFFFFFFFFFFFFFFB0
:10204000FFFFFFFFFFFFFFFFFFFFFFFFFFFFFFFFA0
:10205000FFFFFFFFFFFFFFFFFFFFFFFFFFFFFFFF90
:10206000FFFFFFFFFFFFFFFFFFFFFFFFFFFFFFFF80
:10207000FFFFFFFFFFFFFFFFFFFFFFFFFFFFFFFF70
:10208000FFFFFFFFFFFFFFFFFFFFFFFFFFFFFFFF60
:10209000044E554C4CFFFFFFFFFFFFFFFFFFFFFF0C
:1020A000FFFFFFFFFFFFFFFFFFFFFFFFFFFFFFFF40
:1020B000FFFFFFFFFFFFFFFFFFFFFFFFFFFFFFFF30
:1020C000FFFFFFFFFFFFFFFFFFFFFFFFFFFFFFFF20
:1020D000FFFFFFFFFFFFFFFFFFFFFFFFFFFFFFFF10
:1020E000FFFFFFFFFFFFFFFFFFFFFFFFFFFFFFFF00
:1020F000FFFFFFFFFFFFFFFFFFFFFFFFFFFFFFFFF0
:10210000FFFFFFFFFFFFFFFFFFFFFFFFFFFFFFFFDF
:10211000FF045354444EFFFFFFFFFFFFFFFFFFFF8D
:10212000FFFFFFFFFFFFFFFFFFFFFFFFFFFFFFFFBF
:10213000FFFFFFFFFFFFFFFFFFFFFFFFFFFFFFFFAF
:10214000FFFFFFFFFFFFFFFFFFFFFFFFFFFFFFFF9F
:10215000FFFFFFFFFFFFFFFFFFFFFFFFFFFFFFFF8F
:10216000FFFFFFFFFFFFFFFFFFFFFFFFFFFFFFFF7F
:10217000FFFFFFFFFFFFFFFFFFFFFFFFFFFFFFFF6F
:10218000FFFFFFFFFFFFFFFFFFFFFFFFFFFFFFFF5F
:10219000FFFF0453544C46FFFFFFFFFFFFFFFFFF0D
:1021A000FFFFFFFFFFFFFFFFFFFFFFFFFFFFFFFF3F
:1021B000FFFFFFFFFFFFFFFFFFFFFFFFFFFFFFFF2F
:1021C000FFFFFFFFFFFFFFFFFFFFFFFFFFFFFFFF1F
:1021D000FFFFFFFFFFFFFFFFFFFFFFFFFFFFFFFF0F
:1021E000FFFFFFFFFFFFFFFFFFFFFFFFFFFFFFFFFF
:1021F000FFFFFFFFFFFFFFFFFFFFFFFFFFFFFFFFEF
:10220000FFFFFFFFFFFFFFFFFFFFFFFFFFFFFFFFDE
:10221000FFFFFF0453545254FFFFFFFFFFFFFFFF78
:10222000FFFFFFFFFFFFFFFFFFFFFFFFFFFFFFFFBE
:10223000FFFFFFFFFFFFFFFFFFFFFFFFFFFFFFFFAE
:10224000FFFFFFFFFFFFFFFFFFFFFFFFFFFFFFFF9E
:10225000FFFFFFFFFFFFFFFFFFFFFFFFFFFFFFFF8E
:10226000FFFFFFFFFFFFFFFFFFFFFFFFFFFFFFFF7E
:10227000FFFFFFFFFFFFFFFFFFFFFFFFFFFFFFFF6E
:10228000FFFFFFFFFFFFFFFFFFFFFFFFFFFFFFFF5E
:10229000FFFFFFFF04454E5452FFFFFFFFFFFFFF0C
:1022A000FFFFFFFFFFFFFFFFFFFFFFFFFFFFFFFF3E
:1022B000FFFFFFFFFFFFFFFFFFFFFFFFFFFFFFFF2E
:1022C000FFFFFFFFFFFFFFFFFFFFFFFFFFFFFFFF1E
:1022D000FFFFFFFFFFFFFFFFFFFFFFFFFFFFFFFF0E
:1022E000FFFFFFFFFFFFFFFFFFFFFFFFFFFFFFFFFE
:1022F000FFFFFFFFFFFFFFFFFFFFFFFFFFFFFFFFEE
:10230000FFFFFFFFFFFFFFFFFFFFFFFFFFFFFFFFDD
:10231000FFFFFFFFFF0450524556FFFFFFFFFFFF87
:10232000FFFFFFFFFFFFFFFFFFFFFFFFFFFFFFFFBD
:10233000FFFFFFFFFFFFFFFFFFFFFFFFFFFFFFFFAD
:10234000FFFFFFFFFFFFFFFFFFFFFFFFFFFFFFFF9D
:10235000FFFFFFFFFFFFFFFFFFFFFFFFFFFFFFFF8D
:10236000FFFFFFFFFFFFFFFFFFFFFFFFFFFFFFFF7D
:10237000FFFFFFFFFFFFFFFFFFFFFFFFFFFFFFFF6D
:10238000FFFFFFFFFFFFFFFFFFFFFFFFFFFFFFFF5D
:10239000FFFFFFFFFFFF044E455854FFFFFFFFFF05
:1023A000FFFFFFFFFFFFFFFFFFFFFFFFFFFFFFFF3D
:1023B000FFFFFFFFFFFFFFFFFFFFFFFFFFFFFFFF2D
:1023C000FFFFFFFFFFFFFFFFFFFFFFFFFFFFFFFF1D
:1023D000FFFFFFFFFFFFFFFFFFFFFFFFFFFFFFFF0D
:1023E000FFFFFFFFFFFFFFFFFFFFFFFFFFFFFFFFFD
:1023F000FFFFFFFFFFFFFFFFFFFFFFFFFFFFFFFFED
:10240000FFFFFFFFFFFFFFFFFFFFFFFFFFFFFFFFDC
:10241000FFFFFFFFFFFFFF044E554C4CFFFFFFFF88
:10242000FFFFFFFFFFFFFFFFFFFFFFFFFFFFFFFFBC
:10243000FFFFFFFFFFFFFFFFFFFFFFFFFFFFFFFFAC
:10244000FFFFFFFFFFFFFFFFFFFFFFFFFFFFFFFF9C
:10245000FFFFFFFFFFFFFFFFFFFFFFFFFFFFFFFF8C
:10246000FFFFFFFFFFFFFFFFFFFFFFFFFFFFFFFF7C
:10247000FFFFFFFFFFFFFFFFFFFFFFFFFFFFFFFF6C
:10248000FFFFFFFFFFFFFFFFFFFFFFFFFFFFFFFF5C
:10249000FFFFFFFFFFFFFFFF045245544EFFFFFF0A
:1024A000FFFFFFFFFFFFFFFFFFFFFFFFFFFFFFFF3C
:1024B000FFFFFFFFFFFFFFFFFFFFFFFFFFFFFFFF2C
:1024C000FFFFFFFFFFFFFFFFFFFFFFFFFFFFFFFF1C
:1024D000FFFFFFFFFFFFFFFFFFFFFFFFFFFFFFFF0C
:1024E000FFFFFFFFFFFFFFFFFFFFFFFFFFFFFFFFFC
:1024F000FFFFFFFFFFFFFFFFFFFFFFFFFFFFFFFFEC
:10250000FFFFFFFFFFFFFFFFFFFFFFFFFFFFFFFFDB
:10251000FFFFFFFFFFFFFFFFFF044E554D4231FF5E
:10252000FFFFFFFFFFFFFFFFFFFFFFFFFFFFFFFFBB
:10253000FFFFFFFFFFFFFFFFFFFFFFFFFFFFFFFFAB
:10254000FFFFFFFFFFFFFFFFFFFFFFFFFFFFFFFF9B
:10255000FFFFFFFFFFFFFFFFFFFFFFFFFFFFFFFF8B
:10256000FFFFFFFFFFFFFFFFFFFFFFFFFFFFFFFF7B
:10257000FFFFFFFFFFFFFFFFFFFFFFFFFFFFFFFF6B
:10258000FFFFFFFFFFFFFFFFFFFFFFFFFFFFFFFF5B
:10259000FFFFFFFFFFFFFFFFFFFF054E554D4232DC
:1025A000FFFFFFFFFFFFFFFFFFFFFFFFFFFFFFFF3B
:1025B000FFFFFFFFFFFFFFFFFFFFFFFFFFFFFFFF2B
:1025C000FFFFFFFFFFFFFFFFFFFFFFFFFFFFFFFF1B
:1025D000FFFFFFFFFFFFFFFFFFFFFFFFFFFFFFFF0B
:1025E000FFFFFFFFFFFFFFFFFFFFFFFFFFFFFFFFFB
:1025F000FFFFFFFFFFFFFFFFFFFFFFFFFFFFFFFFEB
:10260000FFFFFFFFFFFFFFFFFFFFFFFFFFFFFFFFDA
:10261000FFFFFFFFFFFFFFFFFFFFFF054E554D428E
:1026200033FFFFFFFFFFFFFFFFFFFFFFFFFFFFFF86
:10263000FFFFFFFFFFFFFFFFFFFFFFFFFFFFFFFFAA
:10264000FFFFFFFFFFFFFFFFFFFFFFFFFFFFFFFF9A
:10265000FFFFFFFFFFFFFFFFFFFFFFFFFFFFFFFF8A
:10266000FFFFFFFFFFFFFFFFFFFFFFFFFFFFFFFF7A
:10267000FFFFFFFFFFFFFFFFFFFFFFFFFFFFFFFF6A
:10268000FFFFFFFFFFFFFFFFFFFFFFFFFFFFFFFF5A
:10269000FFFFFFFFFFFFFFFFFFFFFFFF054E554D51
:1026A0004234FFFFFFFFFFFFFFFFFFFFFFFFFFFFC2
:1026B000FFFFFFFFFFFFFFFFFFFFFFFFFFFFFFFF2A
:1026C000FFFFFFFFFFFFFFFFFFFFFFFFFFFFFFFF1A
:1026D000FFFFFFFFFFFFFFFFFFFFFFFFFFFFFFFF0A
:1026E000FFFFFFFFFFFFFFFFFFFFFFFFFFFFFFFFFA
:1026F000FFFFFFFFFFFFFFFFFFFFFFFFFFFFFFFFEA
:10270000FFFFFFFFFFFFFFFFFFFFFFFFFFFFFFFFD9
:10271000FFFFFFFFFFFFFFFFFFFFFFFFFF054E551E
:102720004D4235FFFFFFFFFFFFFFFFFFFFFFFFFFF2
:10273000FFFFFFFFFFFFFFFFFFFFFFFFFFFFFFFFA9
:10274000FFFFFFFFFFFFFFFFFFFFFFFFFFFFFFFF99
:10275000FFFFFFFFFFFFFFFFFFFFFFFFFFFFFFFF89
:10276000FFFFFFFFFFFFFFFFFFFFFFFFFFFFFFFF79
:10277000FFFFFFFFFFFFFFFFFFFFFFFFFFFFFFFF69
:10278000FFFFFFFFFFFFFFFFFFFFFFFFFFFFFFFF59
:10279000FFFFFFFFFFFFFFFFFFFFFFFFFFFF054EF4
:1027A000554D4236FFFFFFFFFFFFFFFFFFFFFFFF1B
:1027B000FFFFFFFFFFFFFFFFFFFFFFFFFFFFFFFF29
:1027C000FFFFFFFFFFFFFFFFFFFFFFFFFFFFFFFF19
:1027D000FFFFFFFFFFFFFFFFFFFFFFFFFFFFFFFF09
:1027E000FFFFFFFFFFFFFFFFFFFFFFFFFFFFFFFFF9
:1027F000FFFFFFFFFFFFFFFFFFFFFFFFFFFFFFFFE9
:10280000FFFFFFFFFFFFFFFFFFFFFFFFFFFFFFFFD8
:10281000FFFFFFFFFFFFFFFFFFFFFFFFFFFFFF05C2
:102820004E554D4237FFFFFFFFFFFFFFFFFFFFFF4A
:10283000FFFFFFFFFFFFFFFFFFFFFFFFFFFFFFFFA8
:10284000FFFFFFFFFFFFFFFFFFFFFFFFFFFFFFFF98
:10285000FFFFFFFFFFFFFFFFFFFFFFFFFFFFFFFF88
:10286000FFFFFFFFFFFFFFFFFFFFFFFFFFFFFFFF78
:10287000FFFFFFFFFFFFFFFFFFFFFFFFFFFFFFFF68
:10288000FFFFFFFFFFFFFFFFFFFFFFFFFFFFFFFF58
:10289000FFFFFFFFFFFFFFFFFFFFFFFFFFFFFFFF48
:1028A000054E554D4238FFFFFFFFFFFFFFFFFFFFC3
:1028B000FFFFFFFFFFFFFFFFFFFFFFFFFFFFFFFF28
:1028C000FFFFFFFFFFFFFFFFFFFFFFFFFFFFFFFF18
:1028D000FFFFFFFFFFFFFFFFFFFFFFFFFFFFFFFF08
:1028E000FFFFFFFFFFFFFFFFFFFFFFFFFFFFFFFFF8
:1028F000FFFFFFFFFFFFFFFFFFFFFFFFFFFFFFFFE8
:10290000FFFFFFFFFFFFFFFFFFFFFFFFFFFFFFFFD7
:10291000FFFFFFFFFFFFFFFFFFFFFFFFFFFFFFFFC7
:10292000FF05FFFFFFFFFFFFFFFFFFFFFFFFFFFFB1
:10293000FFFFFFFFFFFFFFFFFFFFFFFFFFFFFFFFA7
:10294000FFFFFFFFFFFFFFFFFFFFFFFFFFFFFFFF97
:10295000FFFFFFFFFFFFFFFFFFFFFFFFFFFFFFFF87
:10296000FFFFFFFFFFFFFFFFFFFFFFFFFFFFFFFF77
:1040000010AF028003D38001C39208900DDAE0FE66
:10401000A3E0FFAC35AD36EE4204EF4205900DDA79
:10402000ECF0A3EDF0A20892AF2210AF028003D310
:104030008001C39208900DDAE0FEA3E0FFE535F4BD
:10404000FCE536F4FDEE5204EF5205900DDAECF08B
:10405000A3EDF0A20892AF22900DDAE0FEA3E0FFFC
:10406000AC35AD36EE5204EF5205ED4C6002D32272
:10407000C322900DDAE0FEA3E0FFAC35AD36EE5280
:1040800004EF5205AA35AB36EDB50306ECB50202D6
:10409000D322C32210AF028003D38001C3920875DC
:1040A0004C0D754DC3754E10754F8D121B0BA2082C
:1040B00092AF7E107F8D22E539C394025027E539F7
:1040C00020E003C38001D3B39200AE35AF368E4CEF
:1040D0008F4DAC37AD388C4E8D4FE53AF550121AF6
:1040E00011C200D322740090109EF090109DF090A9
:1040F000109CF090109BF090109AF0AE35AF36E522
:104100003A2FFF50010E1FBFFF011E8E358F36E57F
:104110003A700302419F853583853682E090109F77
:10412000F0783512FF4A153A90109FE0B43A0280B9
:10413000DE90109FE0C39430FE90109AE090109BA8
:1041400012FF17EEF0E53A7002805485358385360C
:1041500082E090109FF0783512FF4A153A90109F38
:10416000E0B43A0280DF90109FE0C3943075F00A0B
:10417000A4FFAEF090109AE090109B12FF17EFFF93
:10418000E0FCEF2CFE90109AE090109B12FF17EECF
:10419000F090109AE004540390109AF002410F90AE
:1041A000109EE0D39423501290109DE0D3943B5086
:1041B0000990109CE0D3943B4002C32290109EE0F3
:1041C00075F00A84FF7E00EF901097F090109EE04B
:1041D00075F00A84ADF07C00ED901096F090109D83
:1041E000E075F00A84FF7E00EF901095F090109D2E
:1041F000E075F00A84ADF07C00ED901094F0901022
:104200009CE075F00A84FF7E00EF901093F0901010
:104210009CE075F00A84ADF07C00ED901092F09077
:10422000109BE075F00A84FF7E00EF901091F090F3
:10423000109BE075F00A84ADF07C00ED901090F0DA
:10424000E539B4021A90109BE0D3941D4002C322BA
:10425000754C10754D9085374E85384F121C84D3A0
:1042600022900DA9E0FEA3E0FF900DABE0FCA3E0DF
:10427000FDEF6D7004EE6C600280E622853583856B
:104280003682E4936016853583853682E493F5990A
:1042900074FF12FE66783512FF4280E080FE221025
:1042A000AF028003D38001C39208900925E0B401D6
:1042B0000A900925E4F0853599802C900DABE0FE3D
:1042C000A3E0FF0FBF00010E7C037DFFEE5204EF61
:1042D0005205900DABECF0A3EDF08C068D07900924
:1042E000A912FF02E535F0A20892AF228536838538
:1042F0003782E06013853683853782E0F5351242D8
:104300009F783612FF4280E422853683853782E427
:10431000936014853683853782E493F53512429F86
:10432000783612FF4280E222E538601585368385B3
:104330003782E0F53512429F783612FF42153880F9
:10434000E722E5386016853683853782E493F535B4
:1043500012429F783612FF42153880E6229010B143
:10436000E4F0E539453870030243EBE53A7038AEC6
:1043700038AF3974108E048F05FF12FEEB8C068D5A
:104380000790E0FA12FF02FEE493FFEE9010B1E016
:104390009010A012FF17EFF0AE38AF39740412FE80
:1043A000C38E388F39803BAE38AF39740A8E048F94
:1043B00005FF12FEEB8C068D0790E0FA12FF02FE5D
:1043C000E493FFEE9010B1E09010A012FF17EFF011
:1043D000AE38AF39740A8E048F05FF12FE768C3822
:1043E0008D399010B1E004F00243629010B1E0907A
:1043F00010A012FF177430F0E53A700B9010B1E086
:104400000454FE9010B1F09010B1E0C3953B5027DA
:104410009010B07401F09010B0E0FE9010B1E0F494
:1044200004253BC39E40107430F53512429F901016
:10443000B0E02401F050DF9010B1E060189010B1AE
:10444000E014F09010B1E09010A012FF17E0F535E5
:1044500012429F80E2AE3CAF3D8E368F3712430949
:1044600022853E4C853F4D754E10754FC2121B0B79
:10447000900DCDE07024754C10754D3BAE3EAF3FB6
:104480008E4E8F4F121AC8B40110742DF53512429A
:104490009F754C10754DC2121BF9E54090A017F89E
:1044A0002828739010C2E0F5397538007400F53A89
:1044B0007402F53B753CE1753D1512435D9010C3E8
:1044C000E0F5397538007400F53A7402F53B753C37
:1044D000E1753D1512435D9010C4E0F53975380063
:1044E0007400F53A7402F53B753CE1753D151243D5
:1044F0005D8079900DCDE0B4014A754C10754D3B4F
:10450000AE3EAF3F8E4E8F4F121AC8B40136754C77
:1045100010754DC2121BF9754C10754D35754E1046
:10452000754FC5121B0B754C10754DC5754E10752A
:104530004FC2121D1E754C10754DC5754E10754F2E
:10454000C2121B0B754C10754DB2754E10754FC2D3
:10455000121B4E7536107537B21242EC800E800C6D
:10456000800A80088006800480028000AE41AF424D
:104570008E368F371243092210AE028003D380019A
:10458000C39208AE36AF37748052077E00EF4E609C
:104590005B900EDAE014541F900EDAF0900EDAE021
:1045A0007F07900EDC12FE86E535F0900EDAE07F94
:1045B00007900EDD12FE86E536F0A3E537F0900E8B
:1045C000DAE07F07900EDF12FE86E539F0853A4C7F
:1045D000853B4D900EDAE07F07900EE012FE86AE2E
:1045E00083AF828E4E8F4F121B0B8059900EDBE0F3
:1045F0007F07900EDC12FE86E535F0900EDBE07F43
:1046000007900EDD12FE86E536F0A3E537F0900E3A
:10461000DBE07F07900EDF12FE86E539F0853A4C2D
:10462000853B4D900EDBE07F07900EE012FE86AEDC
:1046300083AF828E4E8F4F121B0B900EDBE0045423
:104640001F900EDBF0A20892AE2274009010C8F00A
:104650009010C9E535F0A3E536F0744D9010CBF815
:10466000E4F0E8A3F09010CBE0FEA3E0FF8E4C8FC7
:104670004D754E10754FC8121C21754C10754DC8E4
:10468000121BD410AF028003D38001C39208754C73
:104690000D754DB4E5377F03900DB712FE86AE83DE
:1046A000AF828E4E8F4F121B0BE5377F03900DB7F5
:1046B00012FE86AE83AF828E4C8F4D754E10754FB5
:1046C000C81219E1E537900DBD12FF177400F0A272
:1046D0000892AF22AE38AF398E358F367400F53779
:1046E00012464A900DBDE0700280F82275350275C1
:1046F0003610124072C0D0900EDAE0FE900EDBE071
:10470000B50603C38001D392F0D0D072F0500B7580
:1047100039647538001246D480D29010CDE4F0A3ED
:1047200004F09010CDE0FEA3E0FF900DEAE0BE00A3
:104730003E9F403B7539C87538001246D475361017
:10474000753500124058C0D07535027536001240DC
:1047500058B392F0D0D0B382F05002D3229010CE52
:10476000E02401F050079010CDE03400F050B37415
:1047700012900DCAF0124094C006C007D007D006B0
:104780008E4C8F4D754E10754F78121B0BC32290B7
:1047900010CFE4F0A304F09010CFE0FEA3E0FF9070
:1047A0000DE9E0BE002B9F402875350275360012DA
:1047B00040585002D3227539647538001246D4909F
:1047C00010D0E02401F050079010CFE03400F050FA
:1047D000C674FC900DCAF0124094C006C007D00702
:1047E000D0068E4C8F4D754E10754F78121B0BC333
:1047F0002274199010D3F09010D17401F09010D160
:10480000E0D39404504FD2A79010D27401F09010CE
:10481000D2E0FE9010D3E0C39E400E74FA12FE6602
:104820009010D2E02401F050E5C2A79010D274019C
:10483000F09010D2E0FE9010D3E0C39E400E74FAC8
:1048400012FE669010D2E02401F050E59010D1E005
:104850002401F050A8C2A722E535642C6023E53579
:104860006420601DE53564086017E535647F6011DC
:10487000E5356409600BE535640D6005E535B40A7E
:1048800002D322C322740E90120DF090120EE4F0A7
:1048900090120FE4F0A3F090120DE0F54C90120E80
:1048A000E0F54D90120FE0FEA3E0FF8E4E8F4F908B
:1048B0001211E0F5501219C3901212F07536E1751D
:1048C000372B124309901212E0F539753800753A0A
:1048D000007402F53B753CE1753D0A12435D901290
:1048E0000FE4F0A304F090120DE0F54C90120EE0EE
:1048F000F54D90120FE0FEA3E0FF8E4E8F4F901209
:1049000011E0F5501219C3901212F07536E17537A7
:104910003A124309901212E0F539753800753A00E1
:104920007402F53B753CE1753D0A12435D740290DB
:10493000120FF8E4F0E8A3F090120DE0F54C90129D
:104940000EE0F54D90120FE0FEA3E0FF8E4E8F4F6C
:10495000901211E0F5501219C3901212F07536E161
:1049600075374C124309901212E0F539753800750D
:104970003A007402F53B753CE1753D0A12435D2235
:10498000222222223003139011FBE090A035F82858
:10499000287380048002800080002222C2AFE5815B
:1049A00014901213F0901213E0F8760008760022AB
:1049B0003003119011FAE0F8A3E0901086C8F0A33C
:1049C000C8F0801F901086E0FEA3E0FF8E388F397C
:1049D00090120CE0F53A7404F53B753CE1753D0A24
:1049E00012435D223003129011FBE0900DC8F0904D
:1049F0000DC8E0900003F08038900DC8E0F53975DF
:104A0000380090120CE0F53A7401F53B753CE17505
:104A10003D0D12435D900003E0F5397538009012AA
:104A20000CE0F53A7401F53B753CE1753D0A124323
:104A30005D229011FAE0F8A3E0901214C8F0A3C828
:104A4000F0901217E4F0901217E0D39403506A909C
:104A50001214E0FEA3E0FF8E388F39753A0074041B
:104A6000F53B753CE1753D1112435D901216E4F083
:104A7000901216E0D3940F502B90121412FEDFE028
:104A8000F539753800753A007402F53B753CE175EF
:104A90003D0D12435D901214120026901216E02470
:104AA00001F050CC7536E175370A124309124261A4
:104AB000901217E02401F0508D2230030A9011FB70
:104AC000E09011EFF0801C9011EFE0F5397538009F
:104AD00090120CE0F53A7401F53B753CE1753D0A26
:104AE00012435D229011EFE4F0229011EF7401F077
:104AF00022900DCEE070277404F5357E017F008E84
:104B0000368F377480F539753800753A10753B2F3C
:104B10001245787539C87538001246D4805C124049
:104B200094C006C007754C11754DF9D007D0068E9C
:104B30004E8F4F121AC8C0E0D006EE90A041F82860
:104B4000287380367404F535753702753600741590
:104B5000F539753800753A11753BF9124578801AA8
:104B60007404F5357537037536007415F5397538E5
:104B700000753A11753BF912457822300311A209EC
:104B8000B34006A209B3B35004A2099202801CE408
:104B9000A20233F53975380090120CE0F53A740131
:104BA000F53B753CE1753D0A12435D2230030A90E6
:104BB00011FBE0900DCAF08045900DCAE0F5397503
:104BC000380090120CE0F53A7405F53B753CE17540
:104BD0003D0D12435D753E10753F7890120CE0F567
:104BE000407541E175420A124461900DCAE4F075C6
:104BF0004C10754D3B754E10754F78121B0B2230C3
:104C0000030A9011FBE0900DCAF08039900DCAE0C4
:104C1000F53975380090120CE0F53A7405F53B75DE
:104C20003CE1753D0A12435D74009011EBF0900D6C
:104C3000CBF0900DCAF0754C10754D3B754E10754C
:104C40004F78121B0B22C2AFE58114901218F0901E
:104C50001218E0F8760008760022900DCEE0B4013C
:104C60001D7404F5357537007536007415F5397502
:104C70003800753A10753B2F124578024D057404C3
:104C8000F5357E017F008E368F377480F5397538A3
:104C900000753A10753B2F124578753964753800E8
:104CA0001246D4300345124094C006C007754C111B
:104CB000754DF9D007D0068E4E8F4F121AC8C0E03E
:104CC000D006EE6402601C7404F535753702753643
:104CD000007415F539753800753A11753BF91245B0
:104CE0007880067404900DCAF0801A7404F5357546
:104CF00037007536007415F539753800753A10753A
:104D00003B2F124578223003219011FBE06419609B
:104D1000079011FBE0B41E0A9011FBE0900DD1F05A
:104D200080067404900DCAF0801C900DD1E0F53916
:104D300075380090120CE0F53A7401F53B753CE1D2
:104D4000753D0A12435D2230033E754C11754DF9D5
:104D5000754E10754F5C121B0B754C11754DF97526
:104D60004E0D754FC3121B0B754C11754DF9754ED9
:104D700010754F59121B0B754C11754DF9754E0D71
:104D8000754FBF121B0B801E124094C006C007D087
:104D900007D0068E3E8F3F90120CE0F5407541E142
:104DA00075420A1244612230030A9011FBE0900020
:104DB00004F0801C900004E0F53975380090120C66
:104DC000E0F53A7402F53B753CE1753D0A12435D2E
:104DD0002230030A9011FBE0900ED7F0801C900E59
:104DE000D7E0F53975380090120CE0F53A7401F50A
:104DF0003B753CE1753D0A12435D2230030E901174
:104E0000FBE090106AF0900ED3F0801C900ED3E07F
:104E1000F53975380090120CE0F53A7401F53B75E0
:104E20003CE1753D0A12435D227536E175375E122D
:104E30004309900E1EE0F5397538007401F53A7497
:104E400001F53B753CE1753D0D12435D900E21E08F
:104E5000F5397538007400F53A7401F53B753CE19D
:104E6000753D0D12435D900E22E0F53975380074E2
:104E700000F53A7401F53B753CE1753D0D12435D5B
:104E8000900E24E0F5397538007400F53A7401F598
:104E90003B753CE1753D0A12435D22901219E4F026
:104EA000901219E0D394FF501A901219E090106AF2
:104EB000F07539647538001246D4901219E0240157
:104EC000F050DD740090106AF0900ED3F02222743E
:104ED000009011EBF0900DCBF0900DCAF0740090A3
:104EE0000DD4F0900DD7F0900DD8F0900DD5F09036
:104EF0000DCDE070767401F535753700753600908C
:104F00000DCCE0F539753800753A10753B2F124518
:104F1000787536E17537901243097538077539D0C1
:104F20001246D4900DCCE0F5397538007401F53A8D
:104F30007402F53B900DCFE0FEA3E0FF8E3C8F3D69
:104F400012435D7536E17537A31243097402F535D6
:104F5000753700753600900DCCE0F5397538007561
:104F60003A10753B2F124578025007900DCAE0B4F5
:104F70001E237403F5357537007536007401F53955
:104F8000753800753A10753B2F12457875380175E4
:104F900039F41246D4900DCAE4F0900DCBE4F074CD
:104FA00004F535753700753600740AF53975380023
:104FB000753A10753B2F12457812478F40061247FD
:104FC0008F40012275381275391A1246D47538127D
:104FD00075391A1246D47404F5357E017F008E3679
:104FE0008F377480F539753800753A10753B2F127C
:104FF0004578900DD5E0700674FD900DCAF0900EC6
:10500000D8E0B4010280F722227403F53575370029
:105010007536007450F539753800753A10753B2FA8
:10502000124578229009A8E004547F90121DF8E4FC
:10503000F0E8A3F090121DE0FEA3E0FF9009A7E0C6
:105040006F4E603F90092712FF02E090121FF09010
:10505000121FE0F53512429F90121FE0B40D077445
:105060000AF53512429F90121DE0FEA3E0FF0FBF2C
:1050700000010E747F52077E0090121DEEF0A3EF28
:10508000F080B17536E175370A12430922222222D7
:105090003003519011FBE0901223F0901223E0B402
:1050A0000121D2A79012237401F0901223E0D3942F
:1050B00064500E74FA12FE66901223E02401F05040
:1050C000E9801FC2A79012237401F0901223E0D34D
:1050D0009464500E74FA12FE66901223E02401F0DC
:1050E00050E980031247F122754C12754D09754E37
:1050F00010754F3B121AC8B40111754C12754D0949
:10510000121B28901208E0900EC6F02230033F7563
:105110004C11754DF9754E12754F09121B0B754CDC
:1051200012754D09121B28900DC8E06012753E12D1
:10513000753F097540017541E175420A124461905D
:105140000EC6E0901207F8E4F0E8A3F08015753E73
:1051500012753F0990120CE0F5407541E175420A65
:10516000124461227536E17537A61243097535017F
:10517000753600124058E433F53975380090120C3A
:10518000E0F53A7401F53B753CE1753D0D12435D68
:10519000753502753600124058E433F5397538001C
:1051A00090120CE0F53A7401F53B753CE1753D0D4C
:1051B00012435D753510753600124058E433F539E9
:1051C00075380090120CE0F53A7401F53B753CE13E
:1051D000753D0D12435D900DCDE0F53975380090A9
:1051E000120CE0F53A7401F53B753CE1753D0D128A
:1051F000435D7536E17537DF12430990000CE0F529
:1052000039753800753A017402F53B753CE1753D1E
:105210000D12435D900E1DE0F539753800753A01A9
:105220007402F53B753CE1753D0D12435D900E3CFB
:10523000E0F539753800753A017401F53B753CE1CC
:10524000753D0A12435D22754C11754DF3754E1173
:10525000754FF91219E122754C11754DF6754E1105
:10526000754FF91219E122900DC8E070030252FF48
:105270007441F53512429F745FF53512429F9012CA
:1052800024E4F0901224E0D3941E5019901224E0EC
:10529000900FE212FF17E0F53512429F901224E0C2
:1052A0002401F050DE740DF53512429F740AF53575
:1052B00012429F7453F53512429F745FF5351242C6
:1052C0009F901224E4F0901224E0D3941E50199081
:1052D0001224E090100212FF17E0F53512429F9061
:1052E0001224E02401F050DE740DF53512429F7453
:1052F0000AF53512429F7536E27537091243099057
:105300000EC9E0F53512429F742CF53512429F907C
:105310000ECAE0F53512429F742CF53512429F906B
:105320000ECBE0F53512429F742CF53512429F905A
:105330000ECCE0F53512429F742CF53512429F9049
:105340000ECDE0F53512429F742CF53512429F9038
:105350000ECEE0F53512429F742CF53512429F9027
:105360000ECFE0F53512429F740DF53512429F7451
:105370000AF53512429F22753502753600124058E3
:10538000500B7536E275372A12430980097536E2EB
:105390007537331243092230031C7403F535753712
:1053A000007536009011FBE0F539753800753A103C
:1053B000753B2F1245782230031C7404F535753780
:1053C000007536009011FBE0F539753800753A101C
:1053D000753B2F1245782230031A7403F535753763
:1053E000007536007453F539753800753A10753B01
:1053F0002F1245782230031A7403F535753700757E
:1054000036007445F539753800753A10753B2F1222
:10541000457822300329754C11754DF9754E0E757E
:105420004F3E121B0B900E3EE0900005F0900E3F99
:10543000E0900006F0900E40E0900007F080557577
:105440003E0E753F3E90120CE0F5407541E175420D
:105450000D124461900DC8E0603A753E0E753F41F3
:1054600090120CE0F5407541E175420D12446190D7
:105470000E44E0F53975380090120CE0F53A7401ED
:10548000F53B753CE1753D0D12435D7536E17537B1
:105490000A12430922900DC8E060227536E2753782
:1054A0003C124309900E3CE0F539753800753A011D
:1054B0007401F53B753CE1753D0A12435D300337DD
:1054C0009011FBE0901225F0901225E07011754CC0
:1054D00010754D3B754E0E754F35121B0B80169097
:1054E0001225E0B4010F754C10754D41754E0E75C7
:1054F0004F35121B0B800F754C10754D2F754E0ECE
:10550000754F35121B0B7403F53575370075360072
:10551000744AF539753800753A0E753B3512457881
:10552000227403F5357537007536007452F53975F8
:105530003800753A10753B2F12457822900DC8E05F
:1055400060097536E27537621243097403F53575E3
:105550003700753600744DF539753800753A107599
:105560003B2F12457822900DC8E060097536E27530
:1055700037731243097403F53575370075360074B7
:105580004EF539753800753A10753B2F1245782263
:10559000900DC8E060097536E275378412430974CE
:1055A00003F5357537007536007416F53975380012
:1055B000753A10753B2F124578227403F53575370F
:1055C000007536007417F539753800753A10753B5B
:1055D0002F12457822900DC8E060097536E27537C4
:1055E000951243097403F535753700753600744F0D
:1055F000F539753800753A10753B2F1245782274CD
:1056000003F5357537007536007424F539753800A3
:10561000753A10753B2F124578227403F5357537AE
:10562000007536007425F539753800753A10753BEC
:105630002F124578227403F53575370075360074DE
:1056400049F539753800753A10753B2F12457822A7
:10565000900DCCE0B4081C7404F535753700753630
:1056600000740AF539753800753A10753B2F1245EC
:1056700078801A7403F535753700753600741CF59B
:1056800039753800753A10753B2F1245782274032E
:10569000F5357537007536007418F53975380075AD
:1056A0003A10753B2F124578227403F53575370093
:1056B0007536007419F539753800753A10753B2F39
:1056C000124578227403F535753700753600741A63
:1056D000F539753800753A10753B2F1245782274EC
:1056E00003F535753700753600741BF539753800CC
:1056F000753A10753B2F124578227403F5357537CE
:1057000000753600743DF539753800753A10753BF3
:105710002F124578227403F53575370075360074FD
:1057200034F539753800753A10753B2F12457822DB
:10573000900DC8E060097536E27537A6124309304E
:10574000030A9011FAE0F53CA3E0F53D7409F53544
:10575000753700753600AE3CAF3D8E388F39753ADF
:1057600010753B2F12457822300371754C11754D21
:10577000F9754E0E754F35121B0B7403F5357537E1
:10578000027536007446F539753800753A10753B68
:105790002F1245787539C87538001246D47403F550
:1057A000357537027536007437F539753800753A36
:1057B0000E753B351245787538077539D01246D4C9
:1057C0007403F5357537007536007413F53975387F
:1057D00000753A10753B2F124578801A7403F53521
:1057E0007537007536007446F539753800753A100E
:1057F000753B2F12457822754C10754D3B754E0E3A
:10580000754F35121B0B754C11754DF9754E0E7594
:105810004F35121B0B7403F5357537007536007460
:1058200037F539753800753A0E753B3512457822D3
:10583000754C11754DF9754E0E754F35121B0B7465
:1058400003F535753700753600747FF53975380006
:10585000753A0E753B3512457822300306A209923F
:1058600002802BE4A20233F53975380090120CE067
:10587000F53A7401F53B753CE1753D0A12435D90C4
:105880000DC8E060097536E27537BC1243092290F5
:105890000DC8E0601375994E743212FE6675990D4D
:1058A000743212FE6675990A743212FE66222290D4
:1058B0000DCEE0B4011D7404F53575370075360062
:1058C0007480F539753800753A10753B2F1245789C
:1058D00002596230034B124094C006C007754C1148
:1058E000754DF9D007D0068E4E8F4F121AC8C0E002
:1058F000D006EE64026022900DC27401F07404F5CB
:10590000357537027536007480F539753800753A8B
:1059100011753BF912457880067404900DCAF08029
:1059200041753502753600124058501C7404F53527
:105930007537007536007480F539753800753A1082
:10594000753B2F124578801A7404F535753700754C
:10595000360074FFF539753800753A10753B2F1213
:105960004578229011FBE0C39480C4540F90A04A64
:10597000F8282873805A9011FBE0540790A062F831
:10598000282873C290801AC2918016C2928012C2D7
:1059900093800EC294800AC2958006C2968002C28D
:1059A00097802D802B9011FBE0540790A07AF82867
:1059B0002873C2B0801AC2B18016C2B28012C2B3BC
:1059C000800EC2B4800AC2B58006C2B68002C2B7D9
:1059D000229011FA12FEDFE0F53975380090120CB2
:1059E000E0F53A7401F53B753CE1753D0A12435D03
:1059F00022E580F5397538007400F53A7402F53BFC
:105A0000753CE2753DE212435DE590F5397538006D
:105A10007400F53A7402F53B753CE2753DEC1243B7
:105A20005DE5A0F5397538007400F53A7402F53B70
:105A3000753CE2753DF612435DE5B0F53975380009
:105A40007400F53A7402F53B753CE3753D00124372
:105A50005D7536E375370B124309E4A29133F539CE
:105A60007538007400F53A7402F53B753CE1753DFC
:105A70000D12435DE4A29233F5397538007400F5D8
:105A80003A7402F53B753CE1753D0D12435DE4A2AD
:105A90009333F5397538007400F53A7402F53B75A7
:105AA0003CE1753D0D12435DE4A29433F539753840
:105AB000007400F53A7402F53B753CE1753D0D123A
:105AC000435DE4A29533F5397538007400F53A74F6
:105AD00002F53B753CE1753D0D12435DE4A2A03338
:105AE000F5397538007400F53A7402F53B753CE100
:105AF000753D0D12435DE4A2A133F539753800748C
:105B000000F53A7402F53B753CE1753D0D12435DBD
:105B1000E4A2A233F5397538007400F53A7402F541
:105B20003B753CE1753D0D12435D7536E175370DF2
:105B30001243097536E175370D124309E4A2A33308
:105B4000F5397538007400F53A7402F53B753CE19F
:105B5000753D0D12435DE4A2A433F5397538007428
:105B600000F53A7402F53B753CE1753D0D12435D5D
:105B7000E4A2A533F5397538007400F53A7402F5DE
:105B80003B753CE1753D0D12435DE4A2A633F5394A
:105B90007538007400F53A7402F53B753CE1753DCB
:105BA0000D12435DE4A2B333F5397538007400F586
:105BB0003A7402F53B753CE1753D0D12435DE4A27C
:105BC000B533F5397538007400F53A7402F53B7554
:105BD0003CE1753D0D12435DE4A2B633F5397538ED
:105BE000007400F53A7402F53B753CE1753D0D1209
:105BF000435DE4A2B733F5397538007400F53A74A3
:105C000002F53B753CE1753D0D12435D7536E1755E
:105C1000370A12430922300345124094C006C007D8
:105C2000754C11754DF9D007D0068E4E8F4F121A54
:105C3000C8C0E0D006EE6402601C7404F535753708
:105C400002753600740AF539753800753A11753BDE
:105C5000F912457880067404900DCAF0801A740415
:105C6000F535753700753600740AF53975380075E5
:105C70003A10753B2F124578229011FA12FEDFA8D8
:105C800083A9829011F9E088838982F02230031180
:105C90009011FAE0F8A3E0900DB2C8F0A3C8F0802C
:105CA0001D900DB2E0FEA3E0FF8E388F397401F530
:105CB0003A7406F53B753CE1753D0A12435D22904E
:105CC0001068E4F0227536E37537401243097536E3
:105CD000E3753756124309E580F5397538007400CD
:105CE000F53A7402F53B753CE1753D0D12435DE5F7
:105CF00090F5397538007400F53A7402F53B753C3F
:105D0000E1753D0D12435DE5A0F53975380074006D
:105D1000F53A7402F53B753CE1753D0D12435DE5C6
:105D2000B0F5397538007400F53A7402F53B753CEE
:105D3000E1753D0D12435DE5A8F539753800740035
:105D4000F53A7402F53B753CE1753D0D12435D7407
:105D500020F53512429FE598F5397538007400F545
:105D60003A7402F53B753CE1753D0D12435D7536A5
:105D7000E3753796124309E588F5397538007400E4
:105D8000F53A7402F53B753CE1753D0D12435D75C6
:105D900036E3753799124309E5C8F539753800744B
:105DA00000F53A7402F53B753CE1753D0D12435D1B
:105DB0007536E375379D124309E589F53975380065
:105DC0007400F53A7402F53B753CE1753D0D1243E4
:105DD0005D7536E37537A1124309E5C9F5397538A4
:105DE000007400F53A7402F53B753CE1753D0D1207
:105DF000435D7536E37537A5124309E4A2AD33F56B
:105E0000397538007400F53A7401F53B753CE1755D
:105E10003D0D12435D7536E37537A8124309E4A2C0
:105E2000E833F5397538007400F53A7401F53B75BF
:105E30003CE1753D0D12435D7536E37537AB12439A
:105E400009E5B8F5397538007400F53A7402F53B88
:105E5000753CE1753D0D12435D7536E37537AC1247
:105E60004309E5B7F5397538007400F53A7402F561
:105E70003B753CE1753D1512435D7536E37537AEF4
:105E8000124309E4A2AE33F5397538007400F53ACF
:105E90007401F53B753CE1753D0D12435D7536E1CE
:105EA00075370A1243097536E37537B0124309E5B1
:105EB000C1F5397538007400F53A7402F53B753C4C
:105EC000E1753D0D12435D7536E37537BE1243092A
:105ED000E5C0F5397538007400F53A7402F53B7584
:105EE0003CE1753D0D12435D7536E175370A12438D
:105EF00009125CBF2230030A9011FBE090000AF007
:105F0000803D7536E37537C112430990000AE0F50C
:105F1000397538007401F53A7402F53B753CE1754A
:105F20003D0D12435D901084E0F539753800740121
:105F3000F53A7402F53B753CE1753D0A12435D226A
:105F40007403F5357537007536007401F539753809
:105F500000753A10753B2F1245787536E175370A92
:105F6000124309229011FBE0F8863975380090122F
:105F70000CE0F53A7401F53B753CE1753D0A1243BE
:105F80005D2230030A900E49E09011F2F0801290E9
:105F900011F2E0F53512429F7536E175370A12436A
:105FA0000922300311754C11754DF9754E0D754F61
:105FB000F5121B0B8015753E0D753FF590120CE028
:105FC000F5407541E175420A12446122900DC8E026
:105FD000B4010280030260649011FAE0F8A3E0903B
:105FE0001228C8F0A3C8F090122BE4F090122BE016
:105FF000D39403506D901228E0FEA3E0FF8E388FFB
:10600000397400F53A7404F53B753CE1753D1112A5
:10601000435D90122AE4F090122AE0D3940F502DA1
:1060200090122812FEDFE493F5397538007400F5FC
:106030003A7402F53B753CE1753D0D12435D9012DB
:106040002812002690122AE02401F050CA7536E189
:1060500075370A12430912426190122BE02401F0B5
:10606000508A80209011FA12FEDFE493F5397538DA
:106070000090120CE0F53A7401F53B753CE1753D7A
:106080000D12435D229011FBE0C39480C4540F9025
:10609000A056F8282873805A9011FBE0540790A06E
:1060A00092F8282873D290801AD2918016D29280CA
:1060B00012D293800ED294800AD2958006D2968016
:1060C00002D297802D802B9011FBE0540790A0AA5C
:1060D000F8282873D2B0801AD2B18016D2B28012BA
:1060E000D2B3800ED2B4800AD2B58006D2B6800276
:1060F000D2B7223003119011FAE0F8A3E0900FBC60
:10610000C8F0A3C8F0801F900FBCE0FEA3E0FF8E94
:10611000388F3990120CE0F53A7401F53B753CE18B
:10612000753D0A12435D223003119011FAE0F8A385
:10613000E090000DC8F0A3C8F0801D90000DE0FEB7
:10614000A3E0FF8E388F397401F53A7405F53B757D
:106150003CE1753D0A12435D22900DC8E06009756F
:1061600036E37537D7124309300345124094C00611
:10617000C007754C11754DF9D007D0068E4E8F4F64
:10618000121AC8C0E0D006EE6402601C7406F53531
:106190007537027536007410F539753800753A1187
:1061A000753BF912457880067404900DCAF0802979
:1061B000900DC8E060097536E37537E41243097441
:1061C00006F5357537007536007410F539753800E9
:1061D000753A10753B2F12457822A203B340117512
:1061E0004C11754DF9754E11754FF3121B0B80153F
:1061F000753E11753FF390120CE0F5407541E17565
:10620000420A12446122A203B34011754C11754D2C
:10621000F9754E11754FF6121B0B8015753E1175F1
:106220003FF690120CE0F5407541E175420A1244C8
:1062300061227403F535753700753600740CF53935
:10624000753800753A10753B2F12457822300312CD
:106250009011FBE090000CF09011FBE0901070F0BA
:106260008038901070E0F53975380090120CE0F528
:106270003A7402F53B753CE1753D0D12435D9000AB
:106280000CE0F53975380090120CE0F53A7402F51F
:106290003B753CE1753D0A12435D22900DCEE0B4A2
:1062A000011D7404F5357537017536007415F5391F
:1062B000753800753A10753B2F12457802634674A5
:1062C00004F5357E017F008E368F377480F5397581
:1062D0003800753A10753B2F1245787539C87538F6
:1062E000001246D4300345124094C006C007754CD6
:1062F00011754DF9D007D0068E4E8F4F121AC8C0B7
:10630000E0D006EE6401601C7404F5357537037542
:1063100036007415F539753800753A11753BF91268
:10632000457880067404900DCAF0801A7404F5351F
:106330007537017536007415F539753800753A10E2
:10634000753B2F124578227404F535753700753684
:106350000074FFF539753800753A10753B2F1245FA
:106360007822753E0E753F0B90120CE0F54075419A
:10637000E175420A12446122741490122CF0754C9B
:1063800010754D3B754E0E754F35121B0B90108AD4
:10639000E0900E37F0753E0E753F35754001754142
:1063A000E175420A1244617403F53575370075369C
:1063B000007437F539753800753A0E753B3512455E
:1063C0007890108AE004F090108AE0FE90122CE0A1
:1063D000C39E500690108A7401F022124261C2AF2F
:1063E0007400F54C7401F54D754E20754F007550D5
:1063F000001219C3900DAEF0D2AF22124261C2AFAB
:10640000740EF54C7402F54DAE35AF368E4E8F4F8F
:106410008537501219C390122DF0D2AF90122DE093
:1064200022900DC8E0900003F0900DCCE0900000A9
:10643000F0900E3EE0900005F0900E3FE0900006D8
:10644000F0900E40E0900007F07536E37537F612D5
:1064500043091263DB7536E4753705124309753657
:10646000E475371712430990122EE4F0A3F090124E
:106470002EE0FEA3E0FF7424C39F74099E50030224
:10648000651E7C007D00ED2FFFEC3EFE7866A606C3
:1064900008A60790122EE0FCA3E0FD8C068D079065
:1064A000200012FF02AA83AB828A358B367866867B
:1064B00083088682E0F5371263FB60287536E47541
:1064C000372612430990122EE0FEA3E0FF8E388F8C
:1064D000397400F53A7404F53B753CE1753D0A12D8
:1064E000435D803A900DC8E0B4031E786686830849
:1064F0008682E0F5397538007400F53A7401F53B91
:10650000753CE1753D0D12435D90122FE02401F0C2
:10651000500790122EE03400F0400302646E75368E
:10652000E475373A12430922755C20755D00755E8B
:1065300000755F0075600975612512FD94223003B6
:10654000649012327401F0901232E0D394055053EB
:10655000901232E090E11C12FEA6E493FC740193C9
:10656000FD9011FAE0FEA3E0FFEDB50724ECB506BF
:1065700020C28E901232E090E11693F58BF58DD209
:106580008E901232E090000FF090106BF0126421A8
:10659000227536E475374B124309901232E024011C
:1065A000F050A4803990106BE090E11C12FEA678A8
:1065B0003812FF20753A017401F53B753CE1753DD9
:1065C0000D12435D900DC8E0600B7536E475375FC2
:1065D00012430980097536E175370A12430922749E
:1065E00004F5357537007536007416F539753800C1
:1065F000753A10753B2F12457822753E10753F593C
:1066000090120CE0F5407541E475428D12446175BD
:106610003E0D753FBF90120CE0F5407541E47542A8
:106620009C124461753E10753F5F90120CE0F5407E
:106630007541E47542AB124461753E10753F35906B
:10664000120CE0F5407541E47542BB124461753EA1
:1066500010753F5C90120CE0F5407541E47542CA3C
:10666000124461753E10753F6290120CE0F5407562
:1066700041E47542D9124461901233E4F090123330
:10668000E0D394145030901233E0F4042414900FAB
:10669000E212FF17E0C39430F539753800753A00FF
:1066A0007402F53B753CE1753D0D12435D9012336C
:1066B000E02401F050C77536E47537E9124309222A
:1066C00022900DC8E060097536E47537FB12430966
:1066D0007404F5357537007536007433F53975383F
:1066E00000753A11753BF912457822900DC8E060AB
:1066F000097536E575370C1243097403F53575379E
:1067000000753600744CF539753800753A10753BD4
:106710002F12457822900DC8E060097536E575376F
:10672000211243097403F535753700753600744B33
:10673000F539753800753A10753B2F12457822905F
:106740000DC8E060097536E57537361243097403E4
:10675000F5357537007536007451F53975380075A3
:106760003A10753B2F1245782230031A7535117592
:1067700036F9740BF5377538117539F9753A0B74AC
:1067800000F53B1266C0227536E575374B1243099A
:106790007536E575375D124309900E3DE0F53975A4
:1067A0003800753A017401F53B753CE1753D0A12FC
:1067B000435D7536E575376A124309900E3CE0F586
:1067C00039753800753A017401F53B753CE1753D4A
:1067D0000A12435D7536E5753776124309900E440B
:1067E000E0F539753800753A017401F53B753CE107
:1067F000753D0A12435D7536E57537831243097599
:106800003E0E753F3E90120CE0F5407541E1754239
:106810000A1244617536E575378F124309753E0ECD
:10682000753F4190120CE0F5407541E175420A1246
:1068300044617536E575379B124309900DB2E0FE51
:10684000A3E0FF8E388F39753A017406F53B753C2D
:10685000E1753D0A12435D7536E57537A7124309A8
:1068600090107FE0F539753800753A017401F53BF9
:10687000753CE1753D0A12435D22124094C006C08A
:1068800007D007D0068E3E8F3F90120CE0F5407582
:1068900041E175420F1244617535027536001240B0
:1068A0005850097431F53512429F80077430F53520
:1068B00012429F742CF53512429F900E10E0F5396C
:1068C00075380090120CE0F53A7402F53B753CE126
:1068D000753D0F12435D900DCAE0F53975380075AE
:1068E0003A017405F53B753CE1753D1512435D7544
:1068F00036E57537B4124309900DCAE4F0900DCB1C
:10690000E4F09011EBE4F022300A1C7404F53575C4
:1069100037117536007401F539753800753A107500
:106920003B2F124578801A7404F53575371075368B
:10693000007401F539753800753A10753B2F124512
:106940007822A20AB340247404F5357537217536D0
:10695000009011FBE075F002A4FFAEF08E388F3985
:10696000753A10753B2F12457880227404F5357501
:1069700037207536009011FBE075F002A4FFAEF0F1
:106980008E388F39753A10753B2F12457822754C29
:1069900011754DF9754E12754F37121B0B900DCEB8
:1069A000E0B4013D900DC8E0601B7536E57537B762
:1069B000124309753E12753F377540017541E17507
:1069C000420A1244617404F5357537027536007455
:1069D00048F539753800753A12753B37124578809D
:1069E000002230030A9011FBE0900DEAF0801C9029
:1069F0000DEAE0F53975380090120CE0F53A7403B1
:106A0000F53B753CE1753D0A12435D2230034712A8
:106A10004094C006C007754C11754DF9D007D006DB
:106A20008E4E8F4F121AC8C0E0D006EE6402601E70
:106A30007404F5357E017F028E368F377480F53908
:106A4000753800753A11753BF91245788006740463
:106A5000900DCAF080277E017F008E358F36124060
:106A60002A7404F5357E017F008E368F377480F5E9
:106A700039753800753A10753B2F12457822E4A21B
:106A80008033F53975380090120CE0F53A7401F551
:106A90003B753CE1753D0A12435D22200303026B06
:106AA000B1755CE5755DCB901201E0FEA3E0FF904F
:106AB0000E4512FF02AC83AD828C5E8D5F75610462
:106AC00075600012FCEEEFB4FF0DEEB4FF097536F1
:106AD000E57537CF124309755CE5755DE4901201E9
:106AE000E0FEA3E0FF900E4512FF02AC83AD828C66
:106AF0005E8D5F75610475600012FCEEEFB4FF0DF2
:106B0000EEB4FF097536E57537E8124309755CE5A3
:106B1000755DFD901201E0FEA3E0FF900E4512FFAF
:106B200002AC83AD828C5E8D5F756104756000126E
:106B3000FCEEEFB4FF0DEEB4FF097536E6753701D4
:106B4000124309755CE6755D16901201E0FEA3E044
:106B5000FF900E4512FF02AC83AD828C5E8D5F7597
:106B6000610475600012FCEEEFB4FF0DEEB4FF0996
:106B70007536E675371A124309755CE6755D2F9018
:106B80001201E0FEA3E0FF900E4512FF02AC83ADC0
:106B9000828C5E8D5F75610475600012FCEEEFB44F
:106BA000FF0DEEB4FF097536E675373312430980E1
:106BB000097536E675374812430922222230030A46
:106BC0009011FBE0900DC2F0801C900DC2E0F539F1
:106BD00075380090120CE0F53A7401F53B753CE114
:106BE000753D0A12435D229011FAE0F8A3E0900E81
:106BF00038C8F0A3C8F090123AE4F0A304F0901261
:106C00003AE0FEA3E0FF900E38E0FCA3E0FDEDC308
:106C10009FEC9E402E7539C87538001246D49012EC
:106C20003AE0FEA3E0FF7401BE0006D39F4002805D
:106C30001290123BE02401F0500790123AE0340029
:106C4000F050BB22300303026D98900EDAE0F53964
:106C50007538007400F53A7402F53B753CE1753DFA
:106C60000D12435D900EDBE0F5397538007400F5C8
:106C70003A7402F53B753CE1753D0D12435D900D94
:106C8000D9E0F5397538007400F53A7402F53B75B2
:106C90003CE1753D0D12435D900DC6E0FEA3E0FFA3
:106CA0008E388F397400F53A7404F53B753CE675FF
:106CB0003D6312435D900EDAE090123CF8E4F0E898
:106CC000A3F090123CE0FEA3E0FF900EDBE06F4EDD
:106CD0007003026D988E048F057F07900EDC12FE04
:106CE00096E0F5397538007400F53A7402F53B7595
:106CF0003CE1753D0D12435D90123CE0FEA3E0FFC8
:106D00008E048F057F07900EDD12FE96E0F538A306
:106D1000E0F5397400F53A7402F53B753CE1753DD8
:106D20000D12435D90123CE0FEA3E0FF8E048F0540
:106D30007F07900EDF12FE96E0F53975380074007B
:106D4000F53A7402F53B753CE1753D0D12435D90DB
:106D5000123CE0FEA3E0FF8E048F057F07900EE05B
:106D600012FE96AE83AF828E3E8F3F90120CE0F5FE
:106D7000407541E175420A12446190123CE0FEA365
:106D8000E0FF0FBF00010E741F52077E0090123CFF
:106D9000EEF0A3EFF0026CC222300345124094C023
:106DA00006C007754C11754DF9D007D0068E4E8F71
:106DB0004F121AC8C0E0D006EE6402601C7405F5DC
:106DC000357537027536007401F539753800753A36
:106DD00011753BF912457880067404900DCAF08055
:106DE0001A7405F5357537007536007401F5397577
:106DF0003800753A10753B2F124578223003451242
:106E00004094C006C007754C11754DF9D007D006E7
:106E10008E4E8F4F121AC8C0E0D006EE6402601C7E
:106E20007405F5357537027536007400F539753817
:106E300000753A11753BF912457880067404900D7F
:106E4000CAF0801A7405F535753700753600740080
:106E5000F539753800753A10753B2F1245782212B6
:106E60004261C2CA7400F5CCF5CDD2CAD2CF45E09A
:106E7000900DAEF0C2CAE5CD90123EF0E5CC901276
:106E80003FF0D2CA90123EE0FEA3E0FF740E120063
:106E9000038E388F3990120CE0F53A7401F53B758A
:106EA0003CE1753D1512435D7536E675378E12432C
:106EB00009900DB0E0FEA3E0FF8E388F3990120CE0
:106EC000E0F53A7401F53B753CE1753D0A12435D0E
:106ED000223003539011FBE0900DCCF09011FBE0B9
:106EE00060397401F535753700753600900DCCE0CA
:106EF000F539753800753A10753B2F1245787400D6
:106F0000900DCBF0900DCAF07538017539F412462A
:106F1000D47400900DCBF0900DCAF07400900DCB9E
:106F2000F0900DCAF0804F900DC8E0602D7536E1ED
:106F300075370A124309900DCCE0F5397538009089
:106F4000120CE0F53A7402F53B900DCFE0FEA3E0A1
:106F5000FF8E3C8F3D12435D801C900DCCE0F539D7
:106F600075380090120CE0F53A7402F53B753CE17F
:106F7000753D0A12435D2222222230030A9011FB42
:106F8000E090000BF0801A90000BE0F539753800A6
:106F90007401F53A7402F53B753CE1753D0A124304
:106FA0005D2230032F9011FBE090126DF090126D76
:106FB000E07007D3920692A5801890126DE0FE90C3
:106FC000000BE06E6007C3920692A58005D392067F
:106FD00092A58028A2A5B3B35006A206B3B340027F
:106FE000801A90000BE0F5397538007401F53A7499
:106FF00002F53B753CE1753D0A12435D2230032AE0
:107000009011FBE090126EF030A50890126EE090A7
:1070100011EDF090126EE0FE9011EDE06E6007C38E
:10702000920692A58002D206801F30A51C9011ED19
:10703000E0F53975380090120CE0F53A7401F53B33
:10704000753CE6753D9712435D223003569012045D
:10705000E0FE901202E0F4042EC39404900090F03D
:10706000900090E0C3947F5032901201E0FEA3E0C4
:10707000FF900E4912FF02AC83AD828C5C8D5D7572
:107080005E00755F10900090E0F56175600012FD84
:10709000BF901204E0900EC6F080067404900DCAF2
:1070A000F08027900090E060217536E675379A12DF
:1070B0004309753600753710900090E0F53812439B
:1070C000287536E175370A124309223003469012BB
:1070D00004E0FE901202E0F4042EC3940490011127
:1070E000F0900111E0C3947F5022755C0E755D49EC
:1070F000755E00755F91900111E0F5617560001299
:10710000FDBF901204E0900EC6F080067404900D4E
:10711000CAF08027900111E060217536E67537A02E
:10712000124309753600753791900111E0F5381258
:1071300043287536E175370A124309223003469019
:107140001204E0FE901202E0F4042EC394049001B5
:1071500092F0900192E0C3947F5022755C0E755DB1
:1071600049755E01755F12900192E0F561756000EE
:1071700012FDBF901204E0900EC6F08006740490D9
:107180000DCAF08027900192E060217536E67537D0
:10719000A6124309753601753712900192E0F53851
:1071A0001243287536E175370A1243092230034627
:1071B000901204E0FE901202E0F4042EC3940490B6
:1071C0000213F0900213E0C3947F5022755C0E7599
:1071D0005D49755E01755F93900213E0F56175601E
:1071E0000012FDBF901204E0900EC6F080067404F9
:1071F000900DCAF08027900213E060217536E67585
:1072000037AC124309753601753793900213E0F5D8
:10721000381243287536E175370A124309223003C4
:1072200046901204E0FE901202E0F4042EC394048F
:10723000900294F0900294E0C3947F5022755C0E0B
:10724000755D49755E02755F14900294E0F5617595
:10725000600012FDBF901204E0900EC6F08006742C
:1072600004900DCAF08027900294E060217536E604
:107270007537B2124309753602753714900294E0DF
:10728000F5381243287536E175370A124309223062
:107290000346901204E0FE901202E0F4042EC39420
:1072A00004900315F0900315E0C3947F5022755CA1
:1072B0000E755D49755E02755F95900315E0F56189
:1072C00075600012FDBF901204E0900EC6F08006BB
:1072D0007404900DCAF08027900315E06021753684
:1072E000E67537B812430975360275379590031560
:1072F000E0F5381243287536E175370A1243092242
:10730000300346901204E0FE901202E0F4042EC313
:107310009404900396F0900396E0C3947F502275F6
:107320005C0E755D49755E03755F16900396E0F51A
:107330006175600012FDBF901204E0900EC6F080EF
:10734000067404900DCAF08027900396E0602175C2
:1073500036E67537BE124309753603753716900346
:1073600096E0F5381243287536E175370A1243095D
:1073700022300346901204E0FE901202E0F4042E44
:10738000C39404900417F0900417E0C3947F502234
:10739000755C0E755D49755E03755F97900417E027
:1073A000F56175600012FDBF901204E0900EC6F00A
:1073B00080067404900DCAF08027900417E06021C5
:1073C0007536E67537C412430975360375379790DD
:1073D0000417E0F5381243287536E175370A124371
:1073E0000922300346901204E0FE901202E0F404F9
:1073F0002EC39404900498F0900498E0C3947F50B6
:1074000022755C0E755D49755E04755F1890049871
:10741000E0F56175600012FDBF901204E0900EC6A9
:10742000F080067404900DCAF08027900498E06004
:10743000217536E67537CA12430975360475371853
:10744000900498E0F5381243287536E175370A1232
:10745000430922300346901204E0FE901202E0F449
:10746000042EC39404900519F0900519E0C3947F8D
:107470005022755C0E755D49755E04755F999005C7
:1074800019E0F56175600012FDBF901204E0900EE6
:10749000C6F080067404900DCAF08027900519E0AC
:1074A00060217536E67537D0124309753604753795
:1074B00099900519E0F5381243287536E175370AB9
:1074C00012430922300346901204E0FE901202E0BB
:1074D000F4042EC3940490059AF090059AE0C394A6
:1074E0007F5022755C0E755D49755E05755F1A905B
:1074F000059AE0F56175600012FDBF901204E090FE
:107500000EC6F080067404900DCAF0802790059A8C
:10751000E060217536E67537D61243097536057574
:10752000371A90059AE0F5381243287536E1753719
:107530000A12430922300346901204E0FE90120220
:10754000E0F4042EC3940490061BF090061BE0C3E5
:10755000947F5022755C0E755D49755E05755F9B65
:1075600090061BE0F56175600012FDBF901204E00B
:10757000900EC6F080067404900DCAF08027900625
:107580001BE060217536E67537DC12430975360558
:1075900075379B90061BE0F5381243287536E17568
:1075A000370A12430922300346901204E0FE90127B
:1075B00002E0F4042EC3940490069CF090069CE034
:1075C000C3947F5022755C0E755D49755E06755FCC
:1075D0001C90069CE0F56175600012FDBF901204DE
:1075E000E0900EC6F080067404900DCAF0802790DB
:1075F000069CE060217536E67537E2124309753660
:107600000675371C90069CE0F5381243287536E164
:1076100075370A12430922300346901204E0FE90A7
:107620001202E0F4042EC3940490071DF090071D8D
:10763000E0C3947F5022755C0E755D49755E0675DA
:107640005F9D90071DE0F56175600012FDBF90120F
:1076500004E0900EC6F080067404900DCAF08027F6
:1076600090071DE060217536E67537E8124309750D
:10767000360675379D90071DE0F53812432875369C
:10768000E175370A12430922300346901204E0FEE6
:10769000901202E0F4042EC3940490079EF0900729
:1076A0009EE0C3947F5022755C0E755D49755E0740
:1076B000755F1E90079EE0F56175600012FDBF903A
:1076C0001204E0900EC6F080067404900DCAF0809B
:1076D0002790079EE060217536E67537EE12430964
:1076E00075360775371E90079EE0F53812432875EA
:1076F00036E175370A12430922300346901204E03E
:10770000FE901202E0F4042EC3940490081FF0903F
:10771000081FE0C3947F5022755C0E755D49755E4D
:1077200007755F9F90081FE0F56175600012FDBF4F
:10773000901204E0900EC6F080067404900DCAF01A
:10774000802790081FE060217536E67537F41243F4
:107750000975360775379F90081FE0F538124328E2
:107760007536E175370A1243092230034690120438
:10777000E0FE901202E0F4042EC394049008A0F0FE
:107780009008A0E0C3947F5022755C0E755D49752A
:107790005E08755F209008A0E0F56175600012FD3D
:1077A000BF901204E0900EC6F080067404900DCADB
:1077B000F080279008A0E060217536E67537FA1250
:1077C00043097536087537209008A0E0F538124354
:1077D000287536E175370A124309223003469012A4
:1077E00004E0FE901202E0F4042EC39404900921F8
:1077F000F0900921E0C3947F5022755C0E755D49BD
:10780000755E08755FA1900921E0F5617560001251
:10781000FDBF901204E0900EC6F080067404900D37
:10782000CAF08027900921E060217536E77537009E
:107830001243097536087537A1900921E0F5381211
:1078400043287536E175370A12430922C2031270C4
:107850004A1270CB12713C1271AD12721E12728FED
:107860001273001273711274531274C412753512AC
:1078700075A61276171276881276F912776A127741
:10788000DB1273E222901204E0FE901202E0F40494
:107890002EC39404900090F0900090E0C3947F5029
:1078A00020755C0E755D49755E00755F10900090E7
:1078B000E0F56175600012FDBF901204E0900EC605
:1078C000F022755CE7755D06755E00755F10756189
:1078D0000475600012FD947404900090F0755CE7EC
:1078E000755D0B755E00755F9175610475600012C2
:1078F000FD947404900111F0755CE7755D10755E80
:1079000001755F1275610475600012FD9474049036
:107910000192F0755CE7755D15755E01755F937595
:10792000610475600012FD947404900213F0755C9C
:10793000E7755D1A755E02755F1475610475600008
:1079400012FD947404900294F0755CE7755D1F75E8
:107950005E02755F9575610475600012FD94740494
:10796000900315F0755CE7755D24755E03755F1611
:1079700075610475600012FD947404900396F075AF
:107980005CE7755D29755E03755F977561047560C9
:107990000012FD947404900417F0755CE7755D2E79
:1079A000755E04755F9975610475600012FD9474CD
:1079B00004900519F0755CE7755D33755E05755FBC
:1079C0001A75610575600012FD94740590059AF0B2
:1079D000755CE7755D39755E05755F9B756105754D
:1079E000600012FD94740590061BF0755CE7755DF0
:1079F0003F755E06755F1C75610575600012FD942C
:107A0000740590069CF0755CE7755D45755E0675BE
:107A10005F9D75610575600012FD94740590071DEA
:107A2000F0755CE7755D4B755E07755F1E756105EA
:107A300075600012FD94740590079EF0755CE77503
:107A40005D51755E07755F9F75610575600012FD7C
:107A500094740590081FF0755CE7755D57755E08B6
:107A6000755F2075610575600012FD9474059008BE
:107A7000A0F0755CE7755D5D755E08755FA1756169
:107A80000575600012FD947405900921F0755CE79E
:107A9000755D63755E00755F9175610475600012B8
:107AA000FD947404900111F0755CE7755D68755E76
:107AB00004755F1875610475600012FD947404907C
:107AC0000498F07432900004F022300353901203B3
:107AD000E0FEA3E0FF901201E0FCA3E0FD12FF3204
:107AE00074041200039010D6EEF0A3EFF07404BEFD
:107AF00000039F5023755C0E755D49755E10755FC0
:107B0000D89010D6E0F560A3E0F56112FDBF9012A9
:107B100004E0900EC6F080067404900DCAF0803F19
:107B20009010D6E0FEA3E0FF7404BE00039F502F28
:107B30007536107537D87404F538124328743DF53E
:107B40003512429F7536107537DC9010D7E0C3941C
:107B500004F5381243287536E175370A12430922B5
:107B6000300353901203E0FEA3E0FF901201E0FC0B
:107B7000A3E0FD12FF3274041200039011D8EEF05E
:107B8000A3EFF07404BE00039F5023755C0E755D77
:107B900049755E11755F589011D8E0F560A3E0F566
:107BA0006112FDBF901204E0900EC6F080067404CE
:107BB000900DCAF0803F9011D8E0FEA3E0FF74045E
:107BC000BE00039F502F7536117537587404F53871
:107BD000124328743DF53512429F75361175375C96
:107BE0009011D9E0C39404F5381243287536E17535
:107BF000370A12430922900DCCE090126FF07536CF
:107C0000E77537751243097536E175370A1243096E
:107C10007536E77537B71243097536E775376D1254
:107C200043097536FD7537671243097536E77537B1
:107C3000BB124309900DCCE0F539753800753A0157
:107C40007402F53B900DCFE0FEA3E0FF8E3C8F3D2C
:107C500012435D900DC8E060227536E77537CC128F
:107C60004309900000E0F539753800753A01740257
:107C7000F53B753CE1753D0A12435D900DC8E0B4DB
:107C80000A028003027D749011DB7401F09011DB15
:107C9000E0FE900E28E0C39E5003027D719011DB40
:107CA000E0F539753800753A017402F53B753CE131
:107CB000753D0D12435D7401F5357537007536005D
:107CC0009011DBE0F539753800753A10753B2F12CD
:107CD00045787400900DCBF0900DCAF075380175A1
:107CE00039F41246D4900DCCE060347536E7753720
:107CF000E3124309900DCCE0F53975380090120C71
:107D0000E0F53A7402F53B900DCFE0FEA3E0FF8E64
:107D10003C8F3D12435D7538017539F41246D474B9
:107D200001F5357537007536007400F53975380082
:107D3000753A10753B2F1245787538017539F41274
:107D400046D47400900DCBF0900DCAF09011DBE09A
:107D500075F00A84AFF07E00EF4E70097536E1755C
:107D6000370A1243099011DBE02401F04003027C42
:107D70008D124C467400900DCBF0900DCAF0753802
:107D8000017539F41246D47400900DCBF0900DCAF1
:107D9000F0223003239011FBE0641E60079011FB7A
:107DA000E0B4190280087404900DCAF080089011A4
:107DB000FBE0900DD1F0801C900DD1E0F5397538C5
:107DC0000090120CE0F53A7402F53B753CE1753D0C
:107DD0000A12435D22900E3B7401F022900E3BE4A8
:107DE000F02222754C10754D3B754E11754FF912EE
:107DF0001B0BD203124D47754C10754D3B754E1140
:107E0000754FF9121B0BD203124D477403F53575EC
:107E100037007536007405F539753800753A1075F8
:107E20003B2F124578227536F67537441243099078
:107E3000107EE0F539753800753A017403F53B752D
:107E40003CE1753D0A12435D7536F675374E1243B7
:107E500009900E32E0FEA3E0FF8E388F39753A01AB
:107E60007403F53B753CE1753D0A12435D22900DAC
:107E7000CAE0603F900DCAE09011EBF0124094C050
:107E800006C007D007D0068E4C8F4D754E10754F2B
:107E90003B121AC8C0E0D006EE7018124094C0061B
:107EA000C007D007D0068E4C8F4D754E10754F7899
:107EB000121B0B9011EBE0600E9011EBE0642A6056
:107EC00006900DC8E07002806090107FE0B401352C
:107ED0009011EBE0F5397538007401F53A7403F54B
:107EE0003B753CE1753D0D12435D9011EBE090F464
:107EF0004412FEA6783612FF201243097536E1754A
:107F0000370A1243099011EBE4F0900DCAE4F090A7
:107F10000DCBE4F0754C10754D3B754E10754F78D8
:107F2000121B0B9011F07401F07400901085F0900A
:107F30001086F8E4F0E8A3F0900003E0900DC8F09C
:107F400090107FE06003028288741A900E28F090EF
:107F50000DC8E060767536E175370A12430975364B
:107F6000E175370A1243097536F675375C12430915
:107F70007536F675376E12430990107FE0F5397546
:107F800038007401F53A7401F53B753CE1753D0A22
:107F900012435D7536F675377D124309900008E08F
:107FA000FEA3E0FF8E388F397401F53A7401F53B7A
:107FB000753CE1753D0A12435D7536F675378E12D4
:107FC00043097536F67537A21243091247F190112D
:107FD000DB7401F09011DBE0D39450500E74FF126B
:107FE000FE669011DBE02401F050E9900008E0FE0D
:107FF000A3E0FFEF64397005EE64306026900DC891
:10800000E060097536F67537B01243091278C290F0
:1080100000087430F0A37439F07401900003F090FC
:108020000DC8F0900E1FE4F0900E1EE4F0900E21AB
:10803000E4F0900E23E4F0900E3CE4F0900E3DE46A
:10804000F0900E44E4F0901083E4F0900E25E4F0FC
:10805000900E26E4F0900E31E4F0D2C6900000E0DD
:10806000900DCCF0747890000DF8E4F0E8A3F09057
:108070000DCCE0FE900E28E0C39E5005900DCCE4A0
:10808000F07536F67537D7124309900E28E0F539AA
:108090007538007401F53A7402F53B753CE1753DA5
:1080A0000A12435D7536F67537E5124309900000F4
:1080B000E0F5397538007401F53A7402F53B753C0A
:1080C000E1753D0A12435D7536F67537F6124309C0
:1080D000900DCCE0F5397538007401F53A7402F56D
:1080E0003B753CE1753D0A12435D900DC8E060238D
:1080F0007536F7753703124309900DCCE0F53975E5
:1081000038007401F53A7402F53B753CE1753D0A9F
:1081100012435D7401F535753700753600900DCC4E
:10812000E0F539753800753A10753B2F1245789097
:1081300011DB7401F09011DBE0D3940A501F753904
:10814000FA7538001246D4900DC8E06007742DF51A
:108150003512429F9011DBE02401F050D87536E1D2
:1081600075370A124309900DC8E0604C7536F775F3
:10817000371A124309900DCCE0F5397538007401B7
:10818000F53A7402F53B900DCFE0FEA3E0FF8E3C84
:108190008F3D12435D7536F77537281243099000FD
:1081A00000E0F5397538007401F53A7402F53B7555
:1081B0003CE1753D0A12435D90000CE0FE901070AA
:1081C000E06E600990000CE0C394054002800A90C4
:1081D000000CE0901070F08008901070E090000C9F
:1081E000F0901089E0B40172901089E4F0900DC80D
:1081F000E060097536F775373E124309900498E040
:10820000C394805055900DCCE0604F755C04755D53
:1082100018901201E0FEA3E0FF900E4512FF02ACA1
:1082200083AD828C5E8D5F900498E0F5617560008F
:1082300012FDBF901201E0FEA3E0FF900498E02F32
:10824000FF50010E901203EEF0A3EFF0900E4512D6
:10825000FF02743BF0900E3AE4F090107F7401F04E
:10826000900DC8E060227536F775375312430990B8
:10827000107FE0F539753800753A017401F53B75EA
:108280003CE1753D0A12435D900E1EE0B40106907C
:108290000E21E07003028963900DC8E0B4030280F0
:1082A0000302833C7536E175370A1243097536F7C8
:1082B000753766124309900E1FE0F5397538007561
:1082C0003A017401F53B753CE1753D0D12435D903B
:1082D0000E1EE0F539753800753A017401F53B75ED
:1082E0003CE1753D0D12435D901068E0F53975383D
:1082F00000753A007401F53B753CE1753D0D124384
:108300005D900E21E0F539753800753A007401F57D
:108310003B753CE1753D0D12435D900E23E0F53950
:10832000753800753A007401F53B753CE1753D0AFE
:1083300012435D7536E175370A124309900E1EE44B
:10834000F0900E21E0B401028003028400900E3B05
:10835000E07006900E25E060030283F6900E26740E
:1083600001F0900DC8E060317407F53512429F7539
:1083700036F77537A21243097536E175370A12438D
:1083800009753600753710900090E0F538124328D3
:108390007536E175370A124309901201E4F0A3F033
:1083A000901203E4F0A3F0755C00755D109012016B
:1083B000E0FEA3E0FF900E4512FF02AC83AD828C7D
:1083C0005E8D5F900090E0F56175600012FDBF90DA
:1083D0001201E0FEA3E0FF900090E02FFF50010E9D
:1083E000901203EEF0A3EFF0900E4512FF02743BE3
:1083F000F0900E3AE4F0900E21E054FE900E21F041
:10840000900E21E0B4020280030284C6900E3BE08D
:10841000700D900E3AE0B40106900E25E060030264
:1084200084BC900E267401F0900DC8E06031740792
:10843000F53512429F7536F77537B0124309753618
:10844000E175370A124309753601753712900192AA
:10845000E0F5381243287536E175370A1243099062
:108460001201E4F0A3F0901203E4F0A3F0755C01B4
:10847000755D12901201E0FEA3E0FF900E4512FF21
:1084800002AC83AD828C5E8D5F900192E0F56175E8
:10849000600012FDBF901201E0FEA3E0FF90019288
:1084A000E02FFF50010E901203EEF0A3EFF0900EBC
:1084B0004512FF02743BF0900E3AE4F0900E21E07A
:1084C00054FD900E21F0900E21E0B40402800302CE
:1084D000858C900E3BE0700D900E3AE0B401069052
:1084E0000E25E06003028582900E267401F0900D47
:1084F000C8E060317407F53512429F7536F775375D
:10850000BE1243097536E175370A12430975360103
:10851000753793900213E0F5381243287536E175EC
:10852000370A124309901201E4F0A3F0901203E419
:10853000F0A3F0755C01755D93901201E0FEA3E07D
:10854000FF900E4512FF02AC83AD828C5E8D5F9072
:108550000213E0F56175600012FDBF901201E0FEAC
:10856000A3E0FF900213E02FFF50010E901203EEE4
:10857000F0A3EFF0900E4512FF02743BF0900E3A1C
:10858000E4F0900E21E054FB900E21F0900E21E0DB
:10859000B408028003028652900E3BE0700D900EEC
:1085A0003AE0B40106900E25E06003028648900E82
:1085B000267401F0900DC8E060317407F535124261
:1085C0009F7536F77537CC1243097536E175370A52
:1085D000124309753602753714900294E0F538128B
:1085E00043287536E175370A124309901201E4F009
:1085F000A3F0901203E4F0A3F0755C02755D149093
:108600001201E0FEA3E0FF900E4512FF02AC83AD25
:10861000828C5E8D5F900294E0F56175600012FDC2
:10862000BF901201E0FEA3E0FF900294E02FFF5004
:10863000010E901203EEF0A3EFF0900E4512FF0230
:10864000743BF0900E3AE4F0900E21E054F7900E57
:1086500021F0900E21E0B410028003028718900EE2
:108660003BE0700D900E3AE0B40106900E25E060FC
:108670000302870E900E267401F0900DC8E0603161
:108680007407F53512429F7536F77537DA124309CC
:108690007536E175370A12430975360275379590BC
:1086A0000315E0F5381243287536E175370A124391
:1086B00009901201E4F0A3F0901203E4F0A3F07526
:1086C0005C02755D95901201E0FEA3E0FF900E45FF
:1086D00012FF02AC83AD828C5E8D5F900315E0F5D6
:1086E0006175600012FDBF901201E0FEA3E0FF90F3
:1086F0000315E02FFF50010E901203EEF0A3EFF0F0
:10870000900E4512FF02743BF0900E3AE4F0900E8A
:1087100021E054EF900E21F0900E21E0B420028071
:10872000030287DE900E3BE0700D900E3AE0B4013C
:1087300006900E25E060030287D4900E267401F0A7
:10874000900DC8E060317407F53512429F7536F719
:108750007537E81243097536E175370A1243097512
:108760003603753716900396E0F5381243287536B0
:10877000E175370A124309901201E4F0A3F0901258
:1087800003E4F0A3F0755C03755D16901201E0FE42
:10879000A3E0FF900E4512FF02AC83AD828C5E8D8C
:1087A0005F900396E0F56175600012FDBF901201C5
:1087B000E0FEA3E0FF900396E02FFF50010E901221
:1087C00003EEF0A3EFF0900E4512FF02743BF09021
:1087D0000E3AE4F0900E21E054DF900E21F0900E5E
:1087E00021E0B4400280030288A4900E3BE0700DAB
:1087F000900E3AE0B40106900E25E0600302889ADC
:10880000900E267401F0900DC8E060317407F535C4
:1088100012429F7536F77537F61243097536E175C2
:10882000370A124309753603753797900417E0F538
:10883000381243287536E175370A12430990120140
:10884000E4F0A3F0901203E4F0A3F0755C03755D0F
:1088500097901201E0FEA3E0FF900E4512FF02ACDC
:1088600083AD828C5E8D5F900417E0F561756000CA
:1088700012FDBF901201E0FEA3E0FF900417E02F6D
:10888000FF50010E901203EEF0A3EFF0900E451290
:10889000FF02743BF0900E3AE4F0900E21E054BFDA
:1088A000900E21F0900E21E0B480028003028963D3
:1088B000900E3BE0700D900E3AE0B40106900E254C
:1088C000E06003028959900E267401F0900DC8E013
:1088D000602A7536F87537041243097536E1753725
:1088E0000A124309753604753799900519E0F53871
:1088F0001243287536E175370A124309901201E4D4
:10890000F0A3F0901203E4F0A3F0755C04755D9998
:10891000901201E0FEA3E0FF900E4512FF02AC832F
:10892000AD828C5E8D5F900519E0F5617560001277
:10893000FDBF901201E0FEA3E0FF900519E02FFFBC
:1089400050010E901203EEF0A3EFF0900E4512FFCF
:1089500002743BF0900E3AE4F0900E21E0547F90C8
:108960000E21F0900E1EE0B40206900E21E070037E
:10897000028F64900E21E0B401028003028A2B90E2
:108980000E3BE07006900E25E06003028A21900EF7
:10899000267401F0900DC8E0602A7536F87537121C
:1089A0001243097536E175370A12430975360575A4
:1089B000371A90059AE0F5381243287536E1753775
:1089C0000A124309901201E4F0A3F0901203E4F0BC
:1089D000A3F0755C05755D1A901201E0FEA3E0FF3F
:1089E000900E4512FF02AC83AD828C5E8D5F9005C8
:1089F0009AE0F56175600012FDBF901201E0FEA3E0
:108A0000E0FF90059AE02FFF50010E901203EEF068
:108A1000A3EFF0900E4512FF02743BF0900E3AE483
:108A2000F0900E21E054FE900E21F0900E21E0B463
:108A300002028003028AEA900E3BE0700D900E3A2B
:108A4000E0B40106900E25E06003028AE0900E2655
:108A50007401F0900DC8E0602A7536F87537201261
:108A600043097536E175370A1243097536057537BE
:108A70009B90061BE0F5381243287536E175370ADE
:108A8000124309901201E4F0A3F0901203E4F0A362
:108A9000F0755C05755D9B901201E0FEA3E0FF9010
:108AA0000E4512FF02AC83AD828C5E8D5F90061B7B
:108AB000E0F56175600012FDBF901201E0FEA3E0D9
:108AC000FF90061BE02FFF50010E901203EEF0A363
:108AD000EFF0900E4512FF02743BF0900E3AE4F076
:108AE000900E21E054FD900E21F0900E21E0B40490
:108AF000028003028BA9900E3BE0700D900E3AE0CD
:108B0000B40106900E25E06003028B9F900E267440
:108B100001F0900DC8E0602A7536F875372F1243C2
:108B2000097536E175370A12430975360675371C23
:108B300090069CE0F5381243287536E175370A1225
:108B40004309901201E4F0A3F0901203E4F0A3F0C3
:108B5000755C06755D1C901201E0FEA3E0FF900EAF
:108B60004512FF02AC83AD828C5E8D5F90069CE067
:108B7000F56175600012FDBF901201E0FEA3E0FFF9
:108B800090069CE02FFF50010E901203EEF0A3EF31
:108B9000F0900E4512FF02743BF0900E3AE4F09014
:108BA0000E21E054FB900E21F0900E21E0B408025B
:108BB0008003028C68900E3BE0700D900E3AE0B49A
:108BC0000106900E25E06003028C5E900E26740173
:108BD000F0900DC8E0602A7536F875373E124309EB
:108BE0007536E175370A12430975360675379D905B
:108BF000071DE0F5381243287536E175370A124330
:108C000009901201E4F0A3F0901203E4F0A3F075D0
:108C10005C06755D9D901201E0FEA3E0FF900E459D
:108C200012FF02AC83AD828C5E8D5F90071DE0F574
:108C30006175600012FDBF901201E0FEA3E0FF909D
:108C4000071DE02FFF50010E901203EEF0A3EFF08E
:108C5000900E4512FF02743BF0900E3AE4F0900E35
:108C600021E054F7900E21F0900E21E0B410028024
:108C700003028D27900E3BE0700D900E3AE0B40198
:108C800006900E25E06003028D1D900E267401F003
:108C9000900DC8E0602A7536F875374D1243097596
:108CA00036E175370A12430975360775371E900786
:108CB0009EE0F5381243287536E175370A124309EC
:108CC000901201E4F0A3F0901203E4F0A3F0755CBD
:108CD00007755D1E901201E0FEA3E0FF900E4512A5
:108CE000FF02AC83AD828C5E8D5F90079EE0F561E4
:108CF00075600012FDBF901201E0FEA3E0FF900737
:108D00009EE02FFF50010E901203EEF0A3EFF090C3
:108D10000E4512FF02743BF0900E3AE4F0900E21E3
:108D2000E054EF900E21F0900E21E0B42002800379
:108D3000028DE6900E3BE0700D900E3AE0B4010615
:108D4000900E25E06003028DDC900E267401F090F9
:108D50000DC8E0602A7536F875375C124309753620
:108D6000E175370A12430975360775379F90081F5A
:108D7000E0F5381243287536E175370A1243099039
:108D80001201E4F0A3F0901203E4F0A3F0755C0785
:108D9000755D9F901201E0FEA3E0FF900E4512FF6B
:108DA00002AC83AD828C5E8D5F90081FE0F561752B
:108DB000600012FDBF901201E0FEA3E0FF90081FCB
:108DC000E02FFF50010E901203EEF0A3EFF0900E93
:108DD0004512FF02743BF0900E3AE4F0900E21E051
:108DE00054DF900E21F0900E21E0B4400280030287
:108DF0008EA5900E3BE0700D900E3AE0B401069007
:108E00000E25E06003028E9B900E267401F0900DFB
:108E1000C8E0602A7536F875376B1243097536E17C
:108E200075370A1243097536087537209008A0E097
:108E3000F5381243287536E175370A124309901246
:108E400001E4F0A3F0901203E4F0A3F0755C087560
:108E50005D20901201E0FEA3E0FF900E4512FF029C
:108E6000AC83AD828C5E8D5F9008A0E0F56175608B
:108E70000012FDBF901201E0FEA3E0FF9008A0E009
:108E80002FFF50010E901203EEF0A3EFF0900E456D
:108E900012FF02743BF0900E3AE4F0900E21E05481
:108EA000BF900E21F0900E21E0B480028003028F6B
:108EB00064900E3BE0700D900E3AE0B40106900E07
:108EC00025E06003028F5A900E267401F0900DC8C1
:108ED000E0602A7536F875377A1243097536E17500
:108EE000370A1243097536087537A1900921E0F554
:108EF000381243287536E175370A1243099012017A
:108F0000E4F0A3F0901203E4F0A3F0755C08755D43
:108F1000A1901201E0FEA3E0FF900E4512FF02AC0B
:108F200083AD828C5E8D5F900921E0F561756000F4
:108F300012FDBF901201E0FEA3E0FF900921E02F97
:108F4000FF50010E901203EEF0A3EFF0900E4512C9
:108F5000FF02743BF0900E3AE4F0900E21E0547F53
:108F6000900E21F0900E3AE0B4010280030291AB22
:108F70009011F1E070059011F0E4F09011F0E0B480
:108F8000010E9011F2E0F53512429F9011F0E4F0DD
:108F90009009A7E0FE9009A8E06E70030291A890E6
:108FA00011EEE4F09009A7E004547F9009A7F09037
:108FB00009A7E090092712FF17E09011DAF090114D
:108FC000DAE0B45F07901088E4F08098901088E0B1
:108FD000B4011F9011DAE0C3946140099011DAE006
:108FE000D3947A4002800B9011DAE0C39420901160
:108FF000DAF09011DAE0640860079011DAE0B47FEB
:1090000031901203E0FEA3E0FFEF4E6022901203C6
:1090100012FEB59011EFE0B401157408F535124257
:109020009F7420F53512429F7408F53512429F0255
:1090300091A89011DAE0B40A030291A89011DAE045
:10904000B42E08901088E0640160028006740D90D0
:1090500011DAF09011DAE0B41302D2C69011DAE01E
:10906000B4121F901201E0FEA3E0FFEF4E600D1F4F
:10907000BFFF011E901203EEF0A3EFF0740D9011EC
:10908000DAF0901088E070279011DAE0B4200674CE
:109090005E9011DAF09011DAE0B42E06747E901131
:1090A000DAF09011DAE0B42C0674409011DAF09006
:1090B00011EFE0B401099011DAE0F53512429F900A
:1090C0001203E0FEA3E0FF900E4512FF02A883A961
:1090D000829011DAE088838982F00FBF00010E745C
:1090E0007F52077E00901203EEF0A3EFF09011DAAA
:1090F000E0B40D0280030291A89010887401F090F2
:1091000011EFE0B40107740AF53512429F74009024
:109110000EC6F0901201F8E4F0E8A3F0901201E01E
:10912000FEA3E0FF901203E0FCA3E0FDEDD39FEC73
:109130009E403A900E4512FF02E0F5351248584025
:1091400024901201E0FEA3E0FF900E4512FF02FC06
:10915000E0FDEC900EC6E0900E4512FF17EDF0908A
:109160000EC6E004F090120112002680AF901201AA
:10917000E4F0A3F0900EC6E0901203F8E4F0E8A348
:10918000F09011F1E0B401069011F07401F090122A
:1091900003E0FEA3E0FFEF4E600E900E4512FF02CB
:1091A000743BF0900E3AE4F0029A5F901201E0FEF8
:1091B000A3E0FF900E4512FF02AC83AD828C5C8D64
:1091C0005D755E10755FD875610475600012FD2BCA
:1091D0009010D6E0FCA3E0FD7404BC00039D500396
:1091E000D38001C392F0EF64FF7005EE64FF60036B
:1091F000C38001D382F05060755C10755DDC901205
:1092000001E0FEA3E0FF900E4512FF02AC83AD82A9
:109210008C5E8D5F9010D6E0FEA3E0FF7404120018
:10922000038E608F6112FDBF901201E0FEA3E0FF8C
:109230009010D6E0FCA3E0FDEF2DFDEE3CFC7404A5
:109240008C068D07120003901203EEF0A3EFF0904E
:109250000E4512FF02743BF0901201E0FEA3E0FF06
:10926000900E4512FF02AC83AD828C5C8D5D755E05
:1092700011755F5875610475600012FD2B9011D84F
:10928000E0FCA3E0FD7404BC00039D5003D3800107
:10929000C392F0EF64FF7005EE64FF6003C38001CA
:1092A000D382F05060755C11755D5C901201E0FE38
:1092B000A3E0FF900E4512FF02AC83AD828C5E8D61
:1092C0005F9011D8E0FEA3E0FF74041200038E60EB
:1092D0008F6112FDBF901201E0FEA3E0FF9011D854
:1092E000E0FCA3E0FDEF2DFDEE3CFC74048C068D4C
:1092F00007120003901203EEF0A3EFF0900E451258
:10930000FF02743BF0901202E02404900EC5F0902E
:109310001202E0900EC6F0900EC6E0900E4512FFCD
:1093200017E0643B6008900EC6E004F080E9900E00
:10933000C6E0FE900EC5E0D39E4009900DCA7401B0
:10934000F0029A2DC20AC20B90120C7401F0900E1A
:10935000C5E0900E4512FF17E0B4240D90120CE406
:10936000F0900EC5E004F080E5900EC5E0900E454B
:1093700012FF17E0B44E0E740290120CF0900EC55E
:10938000E004F080C9900EC5E0900E4512FF17E092
:10939000B4500E740390120CF0900EC5E004F080EF
:1093A000AD900EC5E0900E4512FF17E0B4490E7463
:1093B0000590120CF0900EC5E004F08091900EC55F
:1093C000E0900E4512FF17E0B43A0F740290120CB1
:1093D000F0900EC5E004F002934E900EC5E0900EA2
:1093E0004512FF17E0B4230BD20B900EC5E004F03A
:1093F00002934E900EC5E0900E4512FF17E0B42D7B
:109400000BD20A900EC5E004F002934E900EC5E018
:10941000900E4512FF17E0B42B09900EC5E004F042
:1094200002934E900EC5E0900E4512FF17E0B42156
:10943000159011EE7401F090120C7401F0900EC5AD
:10944000E004F002934E900EC5E0900E4512FF1717
:10945000E0B4261574029011EEF0740290120CF034
:10946000900EC5E004F002934E900EC5E0FE900E03
:10947000C6E06E6004D2038002C2039011DCE4F007
:10948000A3F074939011E0F8E4F0E8A3F09011DCFD
:10949000E0FEA3E0FF9011E0E0FCA3E0FDEDC39F40
:1094A000EC9E5003029A27EF2DFDEE3CFC74018CDC
:1094B000068D0712FEC39011DEEEF0A3EFF09011BF
:1094C000DBE4F09011DBE0D3940340030295859038
:1094D00011DBE0FF7E009011DEE0FCA3E0FD8E02D8
:1094E0008F037F1090E7E612FE968A068B0712FE26
:1094F000F7E493901201FAE0FEA3E0FF9011DBE0A5
:109500002FFF50010E900E4512FF02EAFEE0FFEE23
:10951000D39F40101DBDFF011C9011E0ECF0A3EDA6
:10952000F0029A249011DBE0FF7E009011DEE0FC57
:10953000A3E0FD8E028F037F1090E7E612FE968A6D
:10954000068B0712FEF7E493901201FAE0FEA3E007
:10955000FF9011DBE02FFF50010E900E4512FF022D
:10956000EAFEE0FFEEC39F50100DBD00010C90110C
:10957000DCECF0A3EDF0029A249011DBE02401F082
:1095800040030294C3A203B3501A9011DEE0FEA37D
:10959000E0FF8E048F057F1090E7EC12FE96E493B7
:1095A0006402600280097402900DCAF0029A2D30A4
:1095B00003189011DEE0FEA3E0FF8E048F057F10FC
:1095C00090E7EC12FE96E493600280097409900D16
:1095D000CAF0029A2D3003199011DEE0FEA3E0FFDD
:1095E0008E048F057F1090E7EC12FE96E493B4038F
:1095F000030298819011DEE0FEA3E0FF8E048F0548
:109600007F1090E7ED12FE96AE83AF828E5C8F5D89
:10961000755E11755FE275610375600012FD9490CF
:1096200011DEE0FEA3E0FF8E048F057F1090E7F0CF
:1096300012FE96AE83AF828E5C8F5D755E11755F94
:10964000E575610375600012FD949011DEE0FEA3E4
:10965000E0FF8E048F057F1090E7F312FE96AE8335
:10966000AF828E5C8F5D755E11755FE87561037505
:10967000600012FD94754C10754D3B754E11754F81
:10968000F9121B0B755CF8755D89900EC5E0900EA4
:109690004512FF17AE83AF828E5E8F5F75610475D2
:1096A000600012FCEEEFB4FF16EEB4FF12754C1121
:1096B000754DF3754E11754FF9121B0B0297E3753B
:1096C0005CF8755D8D900EC5E0900E4512FF17AEEB
:1096D00083AF828E5E8F5F75610475600012FCEE51
:1096E000EFB4FF16EEB4FF12754C11754DF6754EC2
:1096F00011754FF9121B0B0297E3755CF8755D91BC
:10970000900EC5E0900E4512FF17AE83AF828E5EBD
:109710008F5F75610375600012FCEEEFB4FF16EE0B
:10972000B4FF12754C10754D3B754E11754FF91203
:109730001B0B0297E3755CF8755D94900EC5E09085
:109740000E4512FF17AE83AF828E5E8F5F7561028A
:1097500075600012FCEEEFB4FF15EEB4FF11754C0E
:1097600010754D41754E11754FF9121B0B807475B4
:109770005CF8755D96900EC5E0900E4512FF17AE31
:1097800083AF828E5E8F5F75610275600012FCEEA2
:10979000EFB4FF15EEB4FF11754C10754D56754EB4
:1097A00011754FF9121B0B803A900EC5E0900E45D3
:1097B00012FF17AE83AF828E358F3675371175382D
:1097C000F990120CE0F539900EC6E0FE900EC5E05F
:1097D000F4042EF53A1240B740097404900DCAF013
:1097E000029A2D754C11754DF9754E10754F3B123F
:1097F0001AC87004C2098002D209754C11754DE275
:10980000754E10754F3B121AC864026003C3800185
:10981000D3820A5009754C11754DF9121BF9300BA2
:1098200018124094C006C007754C11754DF9D00749
:10983000D0068E4E8F4F1219E1754C11754DE5759E
:109840004E11754FF9121AC8C0E0754C11754DE2F2
:10985000754E11754FF9121AC8C0E0D006EE6401BA
:109860006003C38001D392F0D006EEB40203D3802C
:1098700001C372F050097404900DCAF0029A2D8051
:109880002B9011DEE0FEA3E0FF8E048F057F109089
:10989000E7F312FE96AE83AF828E5C8F5D755E112C
:1098A000755FF975610375600012FD949011DEE03B
:1098B000FEA3E0FF8E048F057F1090E7EA12FE966C
:1098C000E493F8740193901205C8F0A3C8F0300631
:1098D00014901205E0FEA3E0FF7A4E7BCEEF6B7092
:1098E00004EE6A600302998E30030302998C753688
:1098F000F875379D1243099011DB7401F09011DB6C
:10990000E0D39492507D9011DBE07F1090E7E61257
:10991000FE86E493F53512429F9011DBE07F1090B4
:10992000E7E712FE86E493F53512429F9011DBE0E3
:109930007F1090E7E812FE86E493F53512429F907F
:1099400011DBE07F1090E7E912FE86E493F5351213
:10995000429F9011DBE075F01084AFF07E00EF4E77
:10996000700E7536E175370A12430912426180079D
:109970007420F53512429F9011DBE02401F0400382
:109980000298FD7536E175370A12430980382006C2
:109990002C901205E0FEA3E0FF7C6F7D79EF6D70E7
:1099A00004EE6C60187C6F7DA2EF6D7004EE6C604D
:1099B0000C7C6F7DFDEFB5050DEEB504091242611B
:1099C00090120512FE28753630753500124058C0C9
:1099D000D0753502753600124058C0D0900E3BE06D
:1099E000B40103D38001C392F0D0D082F092F0D0C2
:1099F000D082F0500280CF9011DEE0FEA3E0FF8E17
:109A0000048F057F1090E7E612FE96AE83AF828E3C
:109A10005C8F5D755E11755FFC7561047560001289
:109A2000FD94800902948D900DCA7401F0900EC6C9
:109A3000E004901201F8E4F0E8A3F0901201E0FED7
:109A4000A3E0FF901203E0FCA3E0FDEFC39DEE9CBA
:109A5000400D900E3A7401F0901203E4F0A3F0224E
:109A60007400901203F8E4F0E8A3F0901201F8E417
:109A7000F0E8A3F0900E3A7401F09011F07401F048
:109A80009011F17401F09011EF7401F09011EEE477
:109A9000F0900E3BE4F09011ECE4F09011ECE070EB
:109AA00004D2068002C206A208B3407090108974E6
:109AB00001F0743E9011F2F0754C10754D3B754EEF
:109AC00011754FF3121B0B754C10754D3B754E11F4
:109AD000754FF6121B0B754C10754D3B754E0D7581
:109AE0004FB2121B0B755CF8755DC1755E11755F29
:109AF000FC75610575600012FD949012057458F0B4
:109B0000A3748FF09010D6E4F0A3F09011D8E4F095
:109B1000A3F09011EBE4F09011EDE4F07E7E7F6E07
:109B200022D20C901275E4F0758E01755C20755D83
:109B300000755E00755F0075600975612512FD9402
:109B400075A8007580FF7590FF75A0FF75B0FFC206
:109B5000C6C2AEC2C775C18175F9F075E90075C29C
:109B60000075C30075C40075C50075C60075B702E1
:109B7000D2AED2AEC2CAC2E875C902C2CF75C800A1
:109B800074FFF5CBF5CD7448F5CAF5CCD2CAC28CBA
:109B9000C2A9C28DD2B9E58954F04405F589D2A98C
:109BA000C29CC2ACC392999298759840758780D236
:109BB0009CD2BCD2ACC28EC2ABC28FC2BBC297C257
:109BC00096E589540F4420F589A280B34033900074
:109BD0000FE0600990000FE0C394064002800A90F5
:109BE000000FE090106BF08006740390106BF0C2D1
:109BF0008E90106BE090E11693F58BF58DD28E80F0
:109C00004B9012737401F0901273E0D394055032AC
:109C1000859965901273E090E11693F58BF58DD2DE
:109C20008E20980280FB859965E565B40D0280144D
:109C300074FF12FE66C298C28E901273E02401F087
:109C400050C580BD901273E090106BF074009010BE
:109C50006AF0900ED3F0755CF8755DC6755E107590
:109C60005F2C75610375600012FD94755CF8755D7D
:109C7000C9755E10755F2F75610375600012FD94E4
:109C8000755CF8755DCC755E10755F29756103753F
:109C9000600012FD94755CF8755DCF755E10755FA0
:109CA0005675610375600012FD94755CF8755DD2A0
:109CB000755E10755F3275610375600012FD9475F5
:109CC0005CF8755DD5755E10755F357561037560FF
:109CD0000012FD94755CF8755DD8755E10755F387F
:109CE00075610375600012FD94755CF8755DDB7538
:109CF0005E10755F3B75610375600012FD94755CC5
:109D0000F8755DDE755E10755F4175610375600005
:109D100012FD94755CF8755DE1755E10755F4475B4
:109D2000610375600012FD94755CF8755DE4755E05
:109D300010755F4775610375600012FD94755CF8DE
:109D4000755DE7755E10755F4A7561037560001299
:109D5000FD94755CF8755DEA755E10755F50756110
:109D60000375600012FD94755CF8755DED755E100D
:109D7000755F5375610375600012FD94755CF8752D
:109D80005DF0755E0D755FF275610375600012FD23
:109D900094754C10754D3B754E10754F5C121B0B36
:109DA000754C10754D3B754E0D754FC3121B0B75E1
:109DB0004C10754D3B754E10754F59121B0B754C61
:109DC00010754D3B754E0D754FBF121B0B740090F7
:109DD0000EDBF0900EDAF0901273E4F0901273E064
:109DE000D394015016901273E0900DBD12FF1774BA
:109DF00001F0901273E02401F050E1900DD9E4F0ED
:109E0000754C10754D3B754E0D754FB2121B0B9076
:109E10000DC6E4F0A3F0901027E4F0901028E4F0D1
:109E2000901026E4F090106FE4F0901071E4F0A32D
:109E3000F0901073E4F0A3F0C204C205754C1075E5
:109E40004D4A754E10754F4D121B0BC202300C540B
:109E5000900DCAE4F0900DD7E4F0900DD4E4F090AA
:109E600009A8E4F09009A8E0D3947F50169009A8BF
:109E7000E090092712FF17742AF09009A8E0240146
:109E8000F050E1754C10754D3B754E10754F5912E1
:109E90001B0B7EFF7FFF8E358F3612402A900DC23E
:109EA000E4F0800B7ECD7FFF8E358F3612402A7412
:109EB00005900DE8F0900DCDE4F07464900DE9F09C
:109EC000900DEAF0900ED4E4F0900ED5E4F0900EF0
:109ED000D6E4F0901068E0900ED1F0900ED77401A7
:109EE000F0900E32E4F0A3F07400900E24F0900E87
:109EF00022F0900E21F0900E1EF07400900ED1F022
:109F0000900ED2F0740590000AF0901084E4F09066
:109F100010887401F0900EC7E4F0741A900E28F0C7
:109F200090108A7401F090108B7401F090108C7472
:109F300001F09009257401F074009009A8F09009CF
:109F4000A7F07400900DABF8E4F0E8A3F0900DA931
:109F5000F8E4F0E8A3F0A20C9208901274E0F53552
:109F6000129A609010D4EEF0A3EFF09010D4E0F8C5
:109F7000A3E0900DE5C8F0A3C8F09009267401F0A5
:109F80007536E175370A124309D206754C10754DC6
:109F900059754E0D754FBF121B0B7EFF7FFF8E351F
:109FA0008F3612402AE581900DADF0D2AF900DC8EA
:109FB000E4F09012757401F090107FE4F090127547
:109FC000E0B4011474FF12FE66900DC8E0600975DC
:109FD00036F87537F3124309901068E0900ED1F00F
:109FE000900DE512FE2880F822D207754C00121958
:109FF000DA900DAEF0754C001219DA900DAEF075D6
:10A000004C001219DA900DAEF075D000A207920C38
:10A01000129B21C20780D40244A30244F302455E8E
:10A0200002456002456202456402456602456802D7
:10A03000456A02456C0249920249940249960249D6
:10A0400098024B42024B44024B600259740259760B
:10A050000259A30259A50260960260980260C502E7
:10A0600060C702598302598702598B02598F0259DE
:10A070009302599702599B02599F0259B20259B64D
:10A080000259BA0259BE0259C20259C60259CA023D
:10A0900059CE0260A50260A90260AD0260B1026003
:10A0A000B50260B90260BD0260C10260D40260D82E
:10A0B0000260DC0260E00260E40260E80260EC0240
:10A0C00060F000FCF8F0E1C2000096004B00258033
:10A0D00012C0096068A8E820776169745F6972201E
:10A0E00000204E6F206465636B2074797065207367
:10A0F000656C65637465640D0A0053414E3201005E
:10A10000008E0048001200120011003600110013EA
:10A1100000110013001100130011001300100013B0
:10A12000001000140010001400100014001000149F
:10A13000001000140010001400100038001000146B
:10A140000010001400100015000F0015000F00157E
:10A15000000F0015000F0039000F0039000F001527
:10A16000000F0039000F0015000F0015000F00153B
:10A17000000F0015000F0015000F0015000E001550
:10A18000000F0015000F0039000E0016000E0039F8
:10A19000000F0039000E0039000F0039000F0015C4
:10A1A000000E0016000E0039000F0016000E0039D8
:10A1B000000E0039000E0016000E0016000E0016EC
:10A1C000000E003A000E0C04000000000000000029
:10A1D000000000000000000000000000000000007F
:10A1E000000000000000000000000000000000006F
:10A1F000008D0048001200120012003600110013FA
:10A2000000110013001100130011001300100014BE
:10A2100000100013001000140010001400100014AF
:10A22000001000140010001400100038001000147A
:10A23000000F0015000F0015000F0015000F00158E
:10A24000000F0015000F0039000F0039000F001536
:10A25000000F0039000F0015000F0015000F00154A
:10A26000000F0015000E0015000F0015000F00155F
:10A27000000F0015000F0015000F0015000E00164E
:10A28000000E0016000E0016000E0016000E00163E
:10A29000000E0016000E0016000E0016000E00162E
:10A2A000000E0016000E003A000E003A000E0016D6
:10A2B000000E003A000E0C04000000000000000038
:10A2C000000000000000000000000000000000008E
:10A2D000000000000000000000000000000000007E
:10A2E000008E004800120012001200360011001308
:10A2F00000110013001100130011001300110013CE
:10A3000000100014001000140010001400100014BD
:10A3100000100014000F001400100038001000148A
:10A32000000F0014000F001400100014000F00159F
:10A33000000F0015000F0039000F0039000F001545
:10A34000000F0039000F0015000F0015000F001559
:10A35000000F0015000F0015000E0015000F00156E
:10A36000000F0015000F0015000F0039000F001638
:10A37000000E0039000E0016000E0015000E00162B
:10A38000000E0016000E0016000E003A000E001619
:10A39000000E003A000E003A000E003A000E0016C1
:10A3A000000E003A000E0C04000000000000000047
:10A3B000000000000000000000000000000000009D
:10A3C000000000000000000000000000000000008D
:10A3D000008D004800120012001200360011001318
:10A3E00000110013001100130010001400100014DD
:10A3F00000100014001000140010001400100015CC
:10A40000000F0016000E0016000E0039000F001697
:10A41000000E0016000E0016000E0016000E0016AC
:10A42000000E0016000E003A000E003A000E001654
:10A43000000E003A000E0016000D0017000D001768
:10A44000000D0017000D0017000D0017000D00177C
:10A45000000D0017000D003B000D0017000D003B24
:10A46000000D0017000D0017000D0017000D00175C
:10A47000000D0017000D003B000D0017000C003B05
:10A48000000D0017000D003B000D003B000D0017F4
:10A49000000D003B000D0C23000000000000000038
:10A4A00000000000000000000000000000000000AC
:10A4B000000000000000000000000000000000009C
:10A4C000008D00470015000F001200370014001027
:10A4D00000110013001100130010001400100014EC
:10A4E00000100014001000140010001400100014DC
:10A4F00000100015000F0016000E003A000E0015A7
:10A50000000F0016000E0016000E0016000E0016BA
:10A51000000E0016000E003A000E003A000E001663
:10A52000000E003A000E0016000E0016000E001677
:10A53000000E0016000E0016000E0016000E00178A
:10A54000000D0017000D0017000D0017000D003B57
:10A55000000D0017000D0017000D0017000D00176B
:10A56000000D0017000D0017000D0017000D003B37
:10A57000000D0017000D003B000D003B000D001703
:10A58000000D003B000D0C23000000000000000047
:10A5900000000000000000000000000000000000BB
:10A5A00000000000000000000000000000000000AB
:10A5B0000090004500110013001100370011001336
:10A5C00000110013001100130010001400100014FB
:10A5D00000100014001000140010001400100014EB
:10A5E00000100014000F0015000E0039000F0015B8
:10A5F000000F0016000E0016000E0016000E0016CA
:10A60000000E0016000E003A000E003A000E001672
:10A61000000E003A000E0016000E0016000E001686
:10A62000000E0016000E0016000E0017000D001799
:10A63000000D0017000D0017000D003B000D003B42
:10A64000000D0017000D0017000D0017000D00177A
:10A65000000D0017000D0017000D003B000D003B22
:10A66000000D0017000D003B000D003B000D001712
:10A67000000D003B000D0C23000000000000000056
:10A6800000000000000000000000000000000000CA
:10A6900000000000000000000000000000000000BA
:10A6A000008D004800130011001000380013001145
:10A6B000001000140010001400100014001000140A
:10A6C00000100014001000140010001400100014FA
:10A6D00000100014000F0015000F003A000E0015C6
:10A6E000000F0015000F0016000E0016000E0016D9
:10A6F000000E0016000E003A000E003A000E001682
:10A70000000E003A000E0016000E0016000E001695
:10A71000000E0016000E0016000E0016000E0016A9
:10A72000000E0016000D0017000D003B000D003B51
:10A73000000D0017000D0017000D0017000D001789
:10A74000000D0017000D0017000D003B000D003B31
:10A75000000D0017000D003B000D003B000D001721
:10A76000000D003B000D0C23000000000000000065
:10A7700000000000000000000000000000000000D9
:10A7800000000000000000000000000000000000C9
:10A79000008E004600100014001000380010001455
:10A7A0000010001400100014001000140010001419
:10A7B0000010001400100014001000140010001409
:10A7C0000010001400100015000F003A000E0015D4
:10A7D000000F0016000E0016000E0016000E0016E8
:10A7E000000E0016000E003A000E003A000E001691
:10A7F000000E003A000E0016000E0016000E0016A5
:10A80000000E0016000E0016000E0016000E0016B8
:10A81000000E0017000D0017000D0017000D0017A7
:10A82000000D0017000D0017000D0017000D001798
:10A83000000D0017000D0017000D0017000D001788
:10A84000000D0017000D003B000D003B000D001730
:10A85000000D003B000D0C23000000000000000074
:10A8600000000000000000000000000000000000E8
:10A8700000000000000000000000000000000000D8
:10A88000008C004800120012001100370011001364
:10A890000011001300110013001100140010001427
:10A8A0000010001400100014001000140010001418
:10A8B00000100014000F0015000F0039000F0015E4
:10A8C000000F0015000F0015000F0015000F0015F8
:10A8D000000F0015000F0039000F0039000F0015A0
:10A8E000000F0039000F0016000E0016000E0016B3
:10A8F000000E0016000D0017000D0017000D0017C8
:10A90000000D0017000D003B000D0017000D003B6F
:10A91000000D0017000D0017000D0017000D0017A7
:10A92000000D0017000D003B000D0017000D003B4F
:10A93000000D0017000D003B000D003B000D00173F
:10A94000000D003B000D0C23000000000000000083
:10A9500000000000000000000000000000000000F7
:10A9600000000000000000000000000000000000E7
:10A97000008E004800120012001100370011001371
:10A980000011001300110013001000140010001437
:10A990000010001400100014001000140010001427
:10A9A00000100014000F0015000F0039000F0015F3
:10A9B000000F0015000F0015000F0015000F001507
:10A9C000000F0015000F0039000F003A000E0016AE
:10A9D000000E003A000E0016000E0016000D0017C3
:10A9E000000D0017000D0017000D0017000D0017D7
:10A9F000000D0017000D0017000D003B000D0017A3
:10AA0000000D003B000D0017000D0017000D003B6E
:10AA1000000D0017000D0017000D003B000D001782
:10AA2000000D003B000D003B000D003B000D003B06
:10AA3000000D003B000D0C23000000000000000092
:10AA40000000000000000000000000000000000006
:10AA500000000000000000000000000000000000F6
:10AA6000008D004800120012001100370011001381
:10AA70000011001300110013001000140010001446
:10AA80000010001400100014001000140010001436
:10AA9000000F0015000F0015000F0039000F001502
:10AAA000000F0015000F0015000F0015000F001516
:10AAB000000F0015000F003A000E003A000E0016BD
:10AAC000000E003A000E0016000E0016000E0016D2
:10AAD000000E0017000D0017000D0017000D0017E5
:10AAE000000D0017000D003B000D0017000D0017B2
:10AAF000000D003B000D0017000D0017000D003B7E
:10AB0000000D0017000D003B000D0017000D001791
:10AB1000000D003B000D003B000D003B000D003B15
:10AB2000000D003B000D0C230000000000000000A1
:10AB30000000000000000000000000000000000015
:10AB40000000000000000000000000000000000005
:10AB5000008D004800120012001100370011001390
:10AB60000011001300110013001000140010001455
:10AB70000010001400100014001000140010001445
:10AB8000000F0015000F0015000F0039000F001511
:10AB9000000F0015000F0015000F0015000F001525
:10ABA000000F0015000F003A000E0039000F0016CC
:10ABB000000E003A000E0016000E0016000E0016E1
:10ABC000000D0017000D0017000D0017000D0017F5
:10ABD000000D0017000D003B000D0017000D0017C1
:10ABE000000D0017000D0017000D0017000D0017D5
:10ABF000000D003B000D003B000D0017000D00177D
:10AC0000000D0017000D003B000D003B000D00176C
:10AC1000000D0017000C0C240000000000000000D4
:10AC20000000000000000000000000000000000024
:10AC30000000000000000000000000000000000014
:10AC4000008E00480012001200110037001100139E
:10AC50000011001300110013001000140010001464
:10AC60000010001400100014001000140010001454
:10AC700000100015000F0015000F0039000F00151F
:10AC8000000F0015000F0015000F0015000F001534
:10AC9000000F0015000F0039000F003A000E0016DB
:10ACA000000E003A000E0016000E0016000E0016F0
:10ACB000000E0017000D0017000D0017000D001703
:10ACC000000D0017000D0017000D003B000D0017D0
:10ACD000000D0017000D0017000D0017000D0017E4
:10ACE000000D003B000D0017000D003B000D00178C
:10ACF000000D0017000D003B000D003B000D00177C
:10AD0000000D0017000D0C240000000000000000E2
:10AD10000000000000000000000000000000000033
:10AD20000000000000000000000000000000000023
:10AD3000008E0048001200120012003700110013AC
:10AD40000011001300110013001000140010001473
:10AD50000010001400100014001000140010001463
:10AD600000100015000F0015000F0039000F00152E
:10AD7000000F0015000F0015000F0015000F001543
:10AD8000000F0015000F0039000F003A000E0016EA
:10AD9000000E003A000E0016000E0016000E0017FE
:10ADA000000D0017000D0017000D0017000D001713
:10ADB000000D0017000D003B000D0017000D003BBB
:10ADC000000D0017000D0017000D0017000D0017F3
:10ADD000000D003B000D003B000D0017000D003B77
:10ADE000000D0017000D003B000D003B000D00178B
:10ADF000000D0017000D0C230000000000000000F3
:10AE00000000000000000000000000000000000042
:10AE10000000000000000000000000000000000032
:10AE2000008D0048001200120011003700110013BD
:10AE30000011001300110013001000140010001482
:10AE40000010001400100014001000140010001472
:10AE5000000F0015000F0015000F0039000F00153E
:10AE6000000F0015000F0015000F0015000F001552
:10AE7000000F0015000F003A000E003A000E0016F9
:10AE8000000E003A000E0016000E0016000E00160E
:10AE9000000D0017000D0017000D0017000D001722
:10AEA000000D0017000D0017000D003B000D003BCA
:10AEB000000D0017000D0017000D0017000D001702
:10AEC000000D003B000D0017000D003B000D003B86
:10AED000000D0017000D003B000D003B000D00179A
:10AEE000000D0017000D0C23000000000000000002
:10AEF0000000000000000000000000000000000052
:10AF00000000000000000000000000000000000041
:10AF1000008E0048001200120011003700110013CB
:10AF20000011001300110013001000140010001491
:10AF30000010001400100014001000140010001481
:10AF4000000F0015000F0015000F0039000F00154D
:10AF5000000F0015000F0015000F0015000F001561
:10AF6000000F0015000F003A000E003A000E001608
:10AF7000000E003A000E0016000E0017000D00171C
:10AF8000000E0017000D0017000D0017000D001730
:10AF9000000D0017000D0017000D0017000D001721
:10AFA000000D003B000D0017000D0017000D0017ED
:10AFB000000D003B000D0017000D0017000D0017DD
:10AFC000000D003B000D003B000D003B000D001785
:10AFD000000D0017000D0C24000000000000000010
:10AFE0000000000000000000000000000000000061
:10AFF0000000000000000000000000000000000051
:10B00000008E0048001200120012003600110013DA
:10B0100000110013001100130010001400100014A0
:10B020000010001400100014001000140010001490
:10B03000000F0015000F0015000F0039000F00155C
:10B04000000F0015000F0015000F0015000F001570
:10B05000000F0015000F003A000E003A000E001617
:10B06000000E003A000E0016000E0016000E00162C
:10B07000000D0017000D0017000D0017000D001740
:10B08000000D0017000D003B000D003B000D003BC4
:10B09000000D0017000D0017000D0017000D001720
:10B0A000000D003B000D003B000D003B000D003B80
:10B0B000000D0017000D003B000D003B000D0017B8
:10B0C000000D0017000D0C23000000000000000020
:10B0D0000000000000000000000000000000000070
:10B0E0000000000000000000000000000000000060
:10B0F000008D0047001200120011003700110013EC
:10B1000000110013001100130010001400100014AF
:10B11000001000140010001400100014001000149F
:10B12000000F0015000F0015000F0039000F00156B
:10B13000000F0015000F0015000F0015000F00157F
:10B14000000F0015000F003A000E003A000E001626
:10B15000000E003A000E0016000E0016000D00163C
:10B16000000D0017000D0017000D0017000D00174F
:10B17000000D0017000D0017000D0017000D00173F
:10B18000000D0017000D0017000D0017000D00172F
:10B19000000D003B000D0017000D0017000D0017FB
:10B1A000000D0017000D003B000D003B000D0017C7
:10B1B000000C0017000D0C2400000000000000002F
:10B1C000000000000000000000000000000000007F
:10B1D000000000000000000000000000000000006F
:10B1E000008D0048001200120012003600110013FA
:10B1F00000110013001100130010001400100014BF
:10B2000000100014001000140010001400100014AE
:10B21000000F0015000F0015000F0039000F00157A
:10B22000000F0015000F0015000F0015000F00158E
:10B23000000F0015000F003A000E003A000E001635
:10B24000000E003A000E0016000E0017000D001749
:10B25000000D0017000D0017000D0017000D00175E
:10B26000000D0017000D003B000D003B000D001706
:10B27000000D003B000D003B000D0017000D0017F6
:10B28000000D003B000D003B000D003B000D0017C2
:10B29000000D003B000D0017000D003B000D0017D6
:10B2A000000D0017000D0C2400000000000000003D
:10B2B000000000000000000000000000000000008E
:10B2C000000000000000000000000000000000007E
:10B2D0000088004500120011001100340011001216
:10B2E00000110012001100120011001200100012D3
:10B2F00000100013001000130010001300100013C2
:10B30000001000130010001300100036001000138E
:10B3100000100013000F0014000F0014000F0014A1
:10B32000000F0014000F0037000F0037000F00144B
:10B33000000F0037000F0014000F0014000F00145E
:10B34000000F0014000F0014000F0014000F001471
:10B35000000E0015000D0037000E0015000D001541
:10B36000000D0038000E0038000E0015000D00160C
:10B37000000D0016000D0038000E0016000D00161E
:10B38000000D0038000E0016000D0038000E0016EB
:10B39000000D0038000E0BB100000000000000009E
:10B3A000000000000000000000000000000000009D
:10B3B000000000000000000000000000000000008D
:10B3C000008A004500120011001100340011001223
:10B3D00000110012001100120011001200100012E2
:10B3E00000100013001000130010001300100013D1
:10B3F000001000130010001300100036001000139E
:10B4000000100013000F0014000F0014000F0014B0
:10B41000000F0014000F0037000F0037000F00145A
:10B42000000F0037000F0014000F0014000F00146D
:10B43000000F0014000F0014000F0014000F00157F
:10B44000000E0015000D0015000D0016000D001671
:10B45000000D0016000D0038000E0016000D00163D
:10B46000000D0016000D0016000D0016000D001650
:10B47000000D0016000D0016000D0038000E00161D
:10B48000000D0038000E0BAD0000000000000000B1
:10B4900000000000000000000000000000000000AC
:10B4A000000000000000000000000000000000009C
:10B4B000008A004500120011001100340011001232
:10B4C00000110012001100120011001200100012F1
:10B4D00000100013001000130010001300100013E0
:10B4E00000100013001000130010003600100013AD
:10B4F00000100013000F0014000F0014000F0014C0
:10B50000000F0014000F0037000F0037000F001469
:10B51000000F0037000F0014000F0014000F00147C
:10B52000000F0014000F0014000F0014000F00158E
:10B53000000E0015000D0037000E0015000D00155F
:10B54000000D0016000D0038000E0016000D00164C
:10B55000000D0016000D0038000E0016000D00163C
:10B56000000D0016000D0016000D0038000E00162C
:10B57000000D0038000E0BB90000000000000000B4
:10B5800000000000000000000000000000000000BB
:10B5900000000000000000000000000000000000AB
:10B5A0000089004600120011001100350011001240
:10B5B00000110012001100120011001200100013FF
:10B5C00000100013001000130010001300100013EF
:10B5D00000100013000F00130010003600100014BC
:10B5E000000F0014000F0014000F0014000F0014CF
:10B5F000000F0014000F0037000F0037000F001479
:10B60000000F0037000F0014000F0014000F00148B
:10B61000000F0014000F0015000E0015000E00159D
:10B62000000E0015000D0016000D0038000E00166B
:10B63000000D0016000D0038000E0016000D00165B
:10B64000000D0016000D0016000D0038000E00164B
:10B65000000D0016000D0016000D0038000E00163B
:10B66000000D0038000E0BB90000000000000000C3
:10B6700000000000000000000000000000000000CA
:10B6800000000000000000000000000000000000BA
:10B690000089004500120011001100350011001250
:10B6A000001100120011001200110012001000120F
:10B6B00000100013001000130010001300100013FE
:10B6C00000100013001000130010003600100013CB
:10B6D000000F0014000F0014000F0014000F0014DE
:10B6E000000F0014000F0037000F0037000F001488
:10B6F000000F0037000F0014000F0014000F00149B
:10B70000000F0014000F0014000E0015000E0015AD
:10B71000000E0015000E0037000F0037000E001558
:10B72000000E0016000D0038000E0016000D001669
:10B73000000D0016000D0038000E0038000E001637
:10B74000000D0016000D0016000D0038000E00164A
:10B75000000D0038000E0BB10000000000000000DA
:10B7600000000000000000000000000000000000D9
:10B7700000000000000000000000000000000000C9
:10B78000008A00460012001100110035001100125D
:10B79000001100120011001200110012001100121D
:10B7A000001000130010001300100013001000130D
:10B7B0000010001300100013000F003600100013DB
:10B7C000000F0014000F0014000F0014000F0014ED
:10B7D000000F0014000F0037000F0037000F001497
:10B7E000000F0037000F0014000F0014000F0014AA
:10B7F000000F0014000F0014000E0015000E0015BD
:10B80000000E0015000E0015000D0016000D00388A
:10B81000000E0016000D0038000E0016000D001678
:10B82000000D0016000D0016000D0016000D00386A
:10B83000000E0016000D0016000D0038000E001658
:10B84000000D0038000E0BB90000000000000000E1
:10B8500000000000000000000000000000000000E8
:10B8600000000000000000000000000000000000D8
:10B87000008900460012001100110034001100126E
:10B88000001100120011001200110012001000132C
:10B89000001000130010001300100013001000131C
:10B8A00000100013001000130010003600100013E9
:10B8B000000F0013000F0014000F0014000F0014FD
:10B8C000000F0014000F0037000F0037000F0014A6
:10B8D000000F0037000F0014000F0014000F0014B9
:10B8E000000F0014000F0014000F0014000F0014CC
:10B8F000000E0015000D0037000E0015000E003779
:10B90000000E0015000D0038000E0015000D001689
:10B91000000D0016000D0038000E0016000D003856
:10B92000000E0016000D0016000D0038000E001667
:10B93000000D0038000E0BB10000000000000000F8
:10B9400000000000000000000000000000000000F7
:10B9500000000000000000000000000000000000E7
:10B96000008900460012001100110034001100127D
:10B97000001100120011001200110012001100123B
:10B98000001000130010001300100013001000132B
:10B9900000100013001000130010003600100013F8
:10B9A000000F0013000F0014000F0014000F00140C
:10B9B000000F0014000F0037000F0037000F0014B5
:10B9C000000F0037000F0014000F0014000F0014C8
:10B9D000000F0014000F0014000F0014000F0014DB
:10B9E000000E0015000E0015000D0038000E003787
:10B9F000000E0015000D0038000E0015000D001699
:10BA0000000D0016000D0016000D0038000E003865
:10BA1000000E0016000D0016000D0038000E001676
:10BA2000000D0038000E0BB1000000000000000007
:10BA30000000000000000000000000000000000006
:10BA400000000000000000000000000000000000F6
:10BA5000008900460012001100110035001100128B
:10BA6000001100120011001200110012001000134A
:10BA7000001000130010001300100013001000133A
:10BA80000010001300100014000F00360010001307
:10BA9000000F0014000F0014000F0014000F00141A
:10BAA000000F0014000F0037000F0037000F0014C4
:10BAB000000F0037000F0014000F0014000F0014D7
:10BAC000000F0014000E0015000E0015000E0015EA
:10BAD000000E0015000D0038000E0038000E003773
:10BAE000000E0015000D0038000E0015000D0016A8
:10BAF000000D0016000D0038000E0038000E003852
:10BB0000000E0016000D0016000D0038000E001685
:10BB1000000D0038000E0BBD00000000000000000A
:10BB20000000000000000000000000000000000015
:10BB30000000000000000000000000000000000005
:10BB4000008900460012001100110035001100129A
:10BB5000001100120011001200110012001000125A
:10BB60000010001300100013001000130010001349
:10BB7000001000130010001300100036000F001317
:10BB8000000F0014000F0014000F0014000F001429
:10BB9000000F0014000F0037000F0037000F0014D3
:10BBA000000F0037000F0014000F0014000F0014E6
:10BBB000000F0014000F0014000F0014000E0015F9
:10BBC000000E0015000D0015000D0016000D0016EA
:10BBD000000D0038000E0038000E0016000D001693
:10BBE000000D0016000D0016000D0016000D0016C9
:10BBF000000D0038000E0016000D0038000E001673
:10BC0000000D0038000E0BB900000000000000001D
:10BC10000000000000000000000000000000000024
:10BC20000000000000000000000000000000000014
:10BC3000008E00480012001200110037001100139E
:10BC40000011001300110013001000140010001464
:10BC50000010001400100014001000140010001553
:10BC6000000F0015000F0015000F0039000F001520
:10BC7000000F0015000F0015000F0015000F001534
:10BC8000000F0015000F003A000E003A000E0016DB
:10BC9000000E003A000E0016000E0016000D0017F0
:10BCA000000D0017000D0017000D0017000D001704
:10BCB000000D0017000D003B000D0017000D0017D0
:10BCC000000D0017000D003B000D003B000D00179C
:10BCD000000D003B000D003B000D0017000D00178C
:10BCE000000D0017000D0017000D0017000D0017C4
:10BCF000000D0017000D0C240000000000000000E3
:10BD00000000000000000000000000000000000033
:10BD10000000000000000000000000000000000023
:10BD2000007E0048001200120012003600120012BD
:10BD30000011001300100014001000130010001474
:10BD4000001000130010001400100014000F001465
:10BD500000100014000F0015000F0039000F00152F
:10BD6000000F0015000F0015000F0016000F001542
:10BD7000000F0015000F003A000E003A000E0016EA
:10BD8000000E003A000D0017000D0017000D0017FF
:10BD9000000D0017000D0017000D0017000D001713
:10BDA000000D0017000C0017000D0017000D001704
:10BDB000000D003B000D003B000D003B000C001887
:10BDC000000D003B000D0017000C0014000C0018C3
:10BDD000000C003C000C0017000D0017000C0017B1
:10BDE000000D0017000C107400000000000000009F
:10BDF0000000000000000000000000000000000043
:10BE00000000000000000000000000000000000032
:10BE1000007D0048001200120012003600120012CD
:10BE20000011001300110013001000140010001482
:10BE3000001000140010001400100014000F001473
:10BE4000000F0015000F0014000F0039000F001440
:10BE5000000C0015000F0015000F0015000F001555
:10BE6000000F0015000F0039000F0039000F0015FA
:10BE7000000F0039000F0015000F0016000F00160C
:10BE8000000E0016000E0017000D0017000D001721
:10BE9000000E0017000D003A000D0017000D0017EE
:10BEA000000D003B000D003A000D003B000D001797
:10BEB000000D003B000D003B000D0017000D0017AA
:10BEC000000D003B000D0017000D0017000C0017BF
:10BED000000D0017000D14E000000000000000003D
:10BEE0000000000000000000000000000000000052
:10BEF0000000000000000000000000000000000042
:10BF0000007E0048001200120011003600120012DC
:10BF10000011001300110013001100130010001491
:10BF20000010001400100014001000110010001484
:10BF3000001000140010001400100039001000144C
:10BF40000010001400100015000F0015000F001560
:10BF5000000F0015000F0039000F003A000F001508
:10BF6000000F0039000F0015000F0015000F00151D
:10BF7000000F0016000E0016000F0015000F001530
:10BF8000000F0015000F0016000E003A000E0016FC
:10BF9000000E003A000F003A000E003A000E0017A3
:10BFA000000D003A000E0017000D003A000F0017B8
:10BFB000000D003A000E0017000D0017000D0017CD
:10BFC000000D0017000D14E000000000000000004C
:10BFD0000000000000000000000000000000000061
:10BFE0000000000000000000000000000000000051
:10BFF000007F004700120012001200360012000FEE
:10C0000000110013001100130011001300100014A0
:10C010000010001400100014001000140010001490
:10C020000010001400100014000F0039000F00155C
:10C03000000F0015000F0015000F0015000F001570
:10C04000000F0015000F0039000F0039000F001518
:10C05000000F0039000F0015000F0015000F00162B
:10C06000000D0017000D0016000D0017000D001642
:10C07000000D0017000D003B000E003A000E0017E7
:10C08000000D003A000D003B000D003B000D0017B5
:10C09000000D003B000D003B000D003B000D0017A4
:10C0A000000C003B000D0018000C0017000D0017DD
:10C0B000000D0017000D14E000000000000000005B
:10C0C0000000000000000000000000000000000070
:10C0D0000000000000000000000000000000000060
:10C0E000007D0047001200120011003700110013FC
:10C0F00000110013001000140010001400100014B0
:10C10000001000140010001400100014001000149F
:10C110000010001400100014000F0039000F00156B
:10C12000000F0015000F0015000F0015000F00157F
:10C13000000F0015000F003A000E003A000E001626
:10C14000000D003B000D0016000D0016000E00163D
:10C15000000D0017000D0016000D0017000D001750
:10C16000000D0016000D0014000D0018000C003B1F
:10C17000000D003B000D003B000C003B000D0017C4
:10C18000000D003B000C0018000C0017000D003BD8
:10C19000000D003B000C0018000D0017000D0017EB
:10C1A000000D0017000D10740000000000000000DA
:10C1B000000000000000000000000000000000007F
:10C1C000000000000000000000000000000000006F
:10C1D0000089004500120011001100350011001205
:10C1E00000110012001100120011001200100012C4
:10C1F00000100013001000130010001300100013B3
:10C20000001000130010001300100036001000137F
:10C2100000100013000F0014000F0014000F001492
:10C22000000F0014000F0037000F0037000F00143C
:10C23000000F0037000F0014000F0014000F00144F
:10C24000000F0014000F0015000E0014000F001561
:10C25000000E0015000E0037000E0015000D001531
:10C26000000D0038000E0016000D0016000D00161F
:10C27000000D0038000E0038000E0016000D0016EC
:10C28000000D0038000E0038000E0038000E0016B9
:10C29000000D0016000D0BB10000000000000000B2
:10C2A000000000000000000000000000000000008E
:10C2B000000000000000000000000000000000007E
:10C2C0000088004500110011001100340011001217
:10C2D00000100012001000120010001200100013D5
:10C2E00000100013001000130010001300100013C2
:10C2F000000F0013000F0013000F0036000F001492
:10C30000000F0014000F0014000F0014000E0014A2
:10C31000000E0014000E0036000F0036000E001450
:10C32000000E0037000F0014000E0014000E001461
:10C33000000E0014000E0014000E0014000E001475
:10C34000000E0015000E0037000E0014000E001540
:10C35000000E0015000E0015000E0015000E001551
:10C36000000E0015000D0037000E0015000E001520
:10C37000000D0015000D0038000D0038000D0015EF
:10C38000000D0037000E0B9B0000000000000000B5
:10C39000000000000000000000000000000000009D
:10C3A000000000000000000000000000000000008D
:10C3B000202069725F6E756D203D20002050616EF7
:10C3C00061736F6E6963204456442047656E6572E1
:10C3D000616C20495220285459504520313629207B
:10C3E000303430383230200D0A002050616E6173D5
:10C3F0006F6E696320445644204456502D43563591
:10C4000031204368616E6765722028545950452079
:10C41000313729200D0A0050414E2047656E657264
:10C42000616C204952204D4F44454445462061727D
:10C4300067756D656E74203D200050414E20435657
:10C440003531204368616E676572204952204D4F37
:10C45000444544454620617267756D656E74203DA4
:10C46000200050414E204952204D4F7645444546CC
:10C4700020617267756D656E74203D200050414EDD
:10C48000204358353120495220444E554D444546AD
:10C4900020617267756D656E74203D200050414EBD
:10C4A0002069722E64697363335F636D64200D0AC3
:10C4B0000053414E32010000620016001B001700BD
:10C4C0001A0017001A001700310019003100190076
:10C4D00030001A0017001A0017001A0030001A0066
:10C4E00017001A002F001B002F001B002F001B003D
:10C4F00016001B0016001B002F001B0016001B005F
:10C5000016001C002F001B00160224000000000073
:10C51000000000000000000000000000000000001B
:10C52000000000000000000000000000000000000B
:10C5300000000000000000000000000000000000FB
:10C5400000000000000000000000000000000000EB
:10C5500000000000000000000000000000000000DB
:10C560000000000000000000000000006100160054
:10C570001A001800310019001800190018001900DD
:10C5800030001A002F001A0017001A0017001A00B6
:10C590002F001B0014001B002D001B002D001B0092
:10C5A0002D001B0014001B0014001B002D001C009C
:10C5B00013001C0013001C002D001C00130220009F
:10C5C000000000000000000000000000000000006B
:10C5D000000000000000000000000000000000005B
:10C5E000000000000000000000000000000000004B
:10C5F000000000000000000000000000000000003B
:10C60000000000000000000000000000000000002A
:10C61000000000000000000000000000000000001A
:10C62000610017001A0017001A00180031001900E5
:10C630001800190030001A0030001A0017001A0004
:10C6400017001B002F001B0016001B002F001C00F2
:10C650002E001C002E001C0015001D0015001D00E2
:10C660002D001D0015001D0015001D002D001D00D2
:10C67000150224000000000000000000000000007F
:10C6800000000000000000000000000000000000AA
:10C69000000000000000000000000000000000009A
:10C6A000000000000000000000000000000000008A
:10C6B000000000000000000000000000000000007A
:10C6C000000000000000000000000000000000006A
:10C6D000000000006200160032001800310019004E
:10C6E000190019001800190030001A0030001A0053
:10C6F00017001B0017001B002F001B0016001B005B
:10C700002F001C002E001C002E001C0015001D0018
:10C7100015001D002D001D0015001D0015001D0039
:10C720002D001D0014020C0000000000000000009D
:10C7300000000000000000000000000000000000F9
:10C7400000000000000000000000000000000000E9
:10C7500000000000000000000000000000000000D9
:10C7600000000000000000000000000000000000C9
:10C7700000000000000000000000000000000000B9
:10C7800000000000000000006200170032001800E6
:10C7900019001800190018003100190030001A00A3
:10C7A00030001A0017001A0017001B002F001B0092
:10C7B00016001B002F001C002E001C002E001C0069
:10C7C00015001D0015001D002D001D0015001D0089
:10C7D00015001D002D001D0015020C0000000000BA
:10C7E0000000000000000000000000000000000049
:10C7F0000000000000000000000000000000000039
:10C800000000000000000000000000000000000028
:10C810000000000000000000000000000000000018
:10C820000000000000000000000000000000000008
:10C830000000000000000000000000006200160080
:10C8400032001800320018001900190030001A00D8
:10C8500030001A002F001B0017001B0017001B00E0
:10C860002F001C0015001C002E001C002E001D00B7
:10C870002D001D0015001D0015001D002D001D00C0
:10C8800015001D0015001D002D001D001401F300F2
:10C890000000000000000000000000000000000098
:10C8A0000000000000000000000000000000000088
:10C8B0000000000000000000000000000000000078
:10C8C0000000000000000000000000000000000068
:10C8D0000000000000000000000000000000000058
:10C8E0000000000000000000000000000000000048
:10C8F000620017001A0017001A001800190018002B
:10C900003100190030001A0030001A0017001B0017
:10C9100017001A002F001B0016001B002F001C0020
:10C920002E001C002D001D0015001D0015001D000F
:10C930002D001D0015001D0015001D002D001D00FF
:10C9400015022400000000000000000000000000AC
:10C9500000000000000000000000000000000000D7
:10C9600000000000000000000000000000000000C7
:10C9700000000000000000000000000000000000B7
:10C9800000000000000000000000000000000000A7
:10C990000000000000000000000000000000000097
:10C9A0000000000062001600320018001900180094
:10C9B00019001800190018001800190030001A009A
:10C9C00030001A0017001A002F001B0016001B0071
:10C9D0002F001B002F001C002E001C0015001C0047
:10C9E00015001D002D001D0015001D0015001D0067
:10C9F0002D001D00150224000000000000000000B2
:10CA00000000000000000000000000000000000026
:10CA10000000000000000000000000000000000016
:10CA20000000000000000000000000000000000006
:10CA300000000000000000000000000000000000F6
:10CA400000000000000000000000000000000000E6
:10CA50000000000000000000620016003200180014
:10CA600019001800190018001900190030001A00E8
:10CA700030001A0017001A0017001B002F001B00BF
:10CA800016001B002F001C002E001C002E001D0095
:10CA900015001D0015001D002D001D0015001D00B6
:10CAA00015001D002D001D001402240000000000D0
:10CAB0000000000000000000000000000000000076
:10CAC0000000000000000000000000000000000066
:10CAD0000000000000000000000000000000000056
:10CAE0000000000000000000000000000000000046
:10CAF0000000000000000000000000000000000036
:10CB000000000000000000000000000062001600AD
:10CB10001A0017001A001800190018001900180050
:10CB20003100190030001A0017001A0017001A000F
:10CB300030001A0017001B002F001B002F001C00E4
:10CB40002E001C0015001C0015001C002D001D00EF
:10CB500015001D0015001D002D001D0015023D00D3
:10CB600000000000000000000000000000000000C5
:10CB700000000000000000000000000000000000B5
:10CB800000000000000000000000000000000000A5
:10CB90000000000000000000000000000000000095
:10CBA0000000000000000000000000000000000085
:10CBB0000000000000000000000000000000000075
:10CBC000620016001A001700320018003100190028
:10CBD00030001A0017001A0017001A0017001A0078
:10CBE00017001A002F001B0016001B002F001B004F
:10CBF0002F001C002E001D0015001C0015001D003C
:10CC00002D001D0015001D0015001D002D001D002C
:10CC100015022400000000000000000000000000D9
:10CC20000000000000000000000000000000000004
:10CC300000000000000000000000000000000000F4
:10CC400000000000000000000000000000000000E4
:10CC500000000000000000000000000000000000D4
:10CC600000000000000000000000000000000000C4
:10CC700000000000620016003200180032001800A8
:10CC80001900190030001A0017001A0017001A00C6
:10CC900017001A0017001A002F001B0016001B00B7
:10CCA0002F001C002E001C002E001C0015001D0073
:10CCB00015001D002D001D0015001D0015001D0094
:10CCC0002D001D00150224000000000000000000DF
:10CCD0000000000000000000000000000000000054
:10CCE0000000000000000000000000000000000044
:10CCF0000000000000000000000000000000000034
:10CD00000000000000000000000000000000000023
:10CD10000000000000000000000000000000000013
:10CD20000000000000000000620016003200180041
:10CD300019001800190018003100190030001A00FD
:10CD400030001A002F001B0016001B002F001C00D3
:10CD500015001C002E001C002D001D002D001D00C4
:10CD600015001D0015001D002D001D0015001D00E3
:10CD700014001D002D001D001401F3000000000030
:10CD800000000000000000000000000000000000A3
:10CD90000000000000000000000000000000000093
:10CDA0000000000000000000000000000000000083
:10CDB0000000000000000000000000000000000073
:10CDC0000000000000000000000000000000000063
:10CDD00000000000000000000000000062001700DA
:10CDE0001A0017003200180019001800310019004D
:10CDF00030001A0030001A002F001B0016001B0024
:10CE00002F001C0015001C002E001D002D001D0011
:10CE10002D001D0015001D0015001D002D001D001A
:10CE200014001D0014001D002D001D001401F4004D
:10CE300000000000000000000000000000000000F2
:10CE400000000000000000000000000000000000E2
:10CE500000000000000000000000000000000000D2
:10CE600000000000000000000000000000000000C2
:10CE700000000000000000000000000000000000B2
:10CE800000000000000000000000000000000000A2
:10CE9000620017001A0017001A001800320018006C
:10CEA0003100190030001A0030001A002F001B005A
:10CEB00016001B002F001C0015001C002E001C007B
:10CEC0002D001D002D001D0015001D0015001D006A
:10CED0002D001D0015001D0015001D002D001D005A
:10CEE0001401F3000000000000000000000000003A
:10CEF0000000000000000000000000000000000032
:10CF00000000000000000000000000000000000021
:10CF10000000000000000000000000000000000011
:10CF20000000000000000000000000000000000001
:10CF300000000000000000000000000000000000F1
:10CF400000000000620017003200180031001900D4
:10CF50001800190030001A0030001A0030001A00C2
:10CF60002F001B0016001B002F001C0015001C00CA
:10CF70002D001D002D001D002D001D0015001D00A1
:10CF800015001D002D001D0014001D0014001D00C3
:10CF90002D001D001401DB00000000000000000057
:10CFA0000000000000000000000000000000000081
:10CFB0000000000000000000000000000000000071
:10CFC0000000000000000000000000000000000061
:10CFD0000000000000000000000000000000000051
:10CFE0000000000000000000000000000000000041
:10CFF000000000000000000062001700320018006E
:10D00000310019001800190030001A0030001A0011
:10D0100017001A0017001B0017001B002F001B0031
:10D0200016001C002E001C002E001C002D001D00F0
:10D0300015001D0015001D002D001D0015001D0010
:10D0400014001D002D001D0014020D000000000042
:10D0500000000000000000000000000000000000D0
:10D0600000000000000000000000000000000000C0
:10D0700000000000000000000000000000000000B0
:10D0800000000000000000000000000000000000A0
:10D090000000000000000000000000000000000090
:10D0A0000000000000000000000000006100170008
:10D0B0001A00170032001800190019003100190079
:10D0C00030001A0017001A0017001A0017001A0083
:10D0D0002F001B0016001B002F001B002F001C0040
:10D0E0002F001C0015001D0015001D002D001D0047
:10D0F00015001D0015001D002D001D001502240047
:10D10000000000000000000000000000000000001F
:10D11000000000000000000000000000000000000F
:10D1200000000000000000000000000000000000FF
:10D1300000000000000000000000000000000000EF
:10D1400000000000000000000000000000000000DF
:10D1500000000000000000000000000000000000CF
:10D160006200170032001800190018001900190099
:10D170003100190017001A0017001A0017001A00D2
:10D1800017001A002F001B0016001B002F001B00A9
:10D190002F001C002E001D0015001C0015001D0096
:10D1A0002D001D0015001D0015001D002D001D0087
:10D1B00015023D000000000000000000000000001B
:10D1C000000000000000000000000000000000005F
:10D1D000000000000000000000000000000000004F
:10D1E000000000000000000000000000000000003F
:10D1F000000000000000000000000000000000002F
:10D20000000000000000000000000000000000001E
:10D2100000000000620017001A0017001A00180032
:10D220001900180019001900180019001800190039
:10D2300018001A0017001A0030001A0017001A0010
:10D240002F001B002F001B002F001C0016001C00CD
:10D2500015001D002D001D0015001D0015001D00EE
:10D260002D001D0015026E000000000000000000EF
:10D2700000000000000000000000000000000000AE
:10D28000000000000000000000000000000000009E
:10D29000000000000000000000000000000000008E
:10D2A000000000000000000000000000000000007E
:10D2B000000000000000000000000000000000006E
:10D2C000000000000000000060001700320018009D
:10D2D000190018001800190018001900180019008A
:10D2E00017001A0017001A0017001A002F001B0061
:10D2F00017001B002F001B002F001C002E001D001C
:10D3000015001D0015001D002D001D0015001D003D
:10D3100015001D002D001D00150256000000000024
:10D3200000000000000000000000000000000000FD
:10D3300000000000000000000000000000000000ED
:10D3400000000000000000000000000000000000DD
:10D3500000000000000000000000000000000000CD
:10D3600000000000000000000000000000000000BD
:10D370000000000000000000000000006200160035
:10D380001A001700320018001900180019001900BF
:10D39000180019001800190017001A0017001A00C9
:10D3A00030001A0017001B002F001B002F001C006C
:10D3B0002E001C0015001C0015001C002E001D0076
:10D3C00015001C0015001D002D001D001502550044
:10D3D000000000000000000000000000000000004D
:10D3E000000000000000000000000000000000003D
:10D3F000000000000000000000000000000000002D
:10D40000000000000000000000000000000000001C
:10D41000000000000000000000000000000000000C
:10D4200000000000000000000000000000000000FC
:10D4300062001600330018003200180019001900AD
:10D440001800190018001A0017001A0017001A0017
:10D4500017001A002F001B0016001B002F001B00D6
:10D460002F001C002E001C0015001C0015001D00C4
:10D470002D001D0015001D0015001D002D001D00B4
:10D4800015023D0000000000000000000000000048
:10D49000000000000000000000000000000000008C
:10D4A000000000000000000000000000000000007C
:10D4B000000000000000000000000000000000006C
:10D4C000000000000000000000000000000000005C
:10D4D000000000000000000000000000000000004C
:10D4E00000000000620016001A0017001A00180061
:10D4F00032001800190019001800190018001A004D
:10D5000017001A0017001A0030001A0017001B003D
:10D510002F001B002F001C002E001C0015001C00FB
:10D5200015001C002E001C0015001D0015001C001D
:10D530002E001D0015025500000000000000000034
:10D5400000000000000000000000000000000000DB
:10D5500000000000000000000000000000000000CB
:10D5600000000000000000000000000000000000BB
:10D5700000000000000000000000000000000000AB
:10D58000000000000000000000000000000000009B
:10D5900000000000000000006200170032001800C8
:10D5A00019001800310019001800190018001A009D
:10D5B00017001A0017001A0017001A002F001B008E
:10D5C00017001B002F001B002F001C002E001C004A
:10D5D00015001C0015001C002E001D0015001D006C
:10D5E00015001D002D001D0015023D00000000006B
:10D5F000000000000000000000000000000000002B
:10D60000000000000000000000000000000000001A
:10D61000000000000000000000000000000000000A
:10D6200000000000000000000000000000000000FA
:10D6300000000000000000000000000000000000EA
:10D640000000000000000000000000006200160062
:10D650001A001700320018003100190018001900D4
:10D6600018001A0017001A0017001A0017001A00F5
:10D670002F001B0017001B002F001C002E001C0099
:10D680002E001C0015001C0015001D002D001D00A3
:10D6900015001C0015001D002D001D0015023D0089
:10D6A000000000000000000000000000000000007A
:10D6B000000000000000000000000000000000006A
:10D6C000000000000000000000000000000000005A
:10D6D000000000000000000000000000000000004A
:10D6E000000000000000000000000000000000003A
:10D6F000000000000000000000000000000000002A
:10D7000062001600320018003100190031001900C3
:10D7100017001A0017001A0017001A0017001A0045
:10D7200017001A002F001B0016001B002F001C0002
:10D730002E001C002D001D0015001D0015001D00F1
:10D740002D001D0015001D0014001D002D001D00E2
:10D75000150224000000000000000000000000008E
:10D7600000000000000000000000000000000000B9
:10D7700000000000000000000000000000000000A9
:10D780000000000000000000000000000000000099
:10D790000000000000000000000000000000000089
:10D7A0000000000000000000000000000000000079
:10D7B00000000000620017001A0017001A0018008D
:10D7C00019001800310019001800190018001A007B
:10D7D00017001A0017001A002F001B0017001B006B
:10D7E0002F001B002F001C002E001C0015001C0029
:10D7F00015001C002E001D0015001C0015001D004A
:10D800002D001D0015025500000000000000000062
:10D810000000000000000000000000000000000008
:10D8200000000000000000000000000000000000F8
:10D8300000000000000000000000000000000000E8
:10D8400000000000000000000000000000000000D8
:10D8500000000000000000000000000000000000C8
:10D860000000000000000000550016003300170003
:10D870001A001700190018001800190018001900E4
:10D880001800190030001A0017001A0030001A00A2
:10D89000170018002F001B002F001B0016001B0094
:10D8A0002E001C0016001B0016001C0016001C0099
:10D8B0002E001C002E001C0015023B000000000082
:10D8C0000000000000000000000000000000000058
:10D8D0000000000000000000000000000000000048
:10D8E0000000000000000000000000000000000038
:10D8F0000000000000000000000000000000000028
:10D900000000000000000000000000000000000017
:10D910000000000000000000000000005D00160094
:10D92000330017001A001700190019003100190000
:10D930001800190017001A0030001B0017001B0008
:10D9400030001B0017001B002F001B002E001C00C6
:10D950002F001B0016001B0014001B002F001B00D3
:10D9600016001C0016001B002F001B0017022200CF
:10D9700061001B002F001B0016001B0016001B007F
:10D980002F001C0016001C0016001C002E001C009E
:10D9900016001C002F001B0016001B002F001C008F
:10D9A0002F001C002E001C0015001C0015001D007F
:10D9B0002D001D0015001D0014001D002D001D0070
:10D9C0001502200000000000000000000000000020
:10D9D00063001700320018001A0018003100190007
:10D9E0001900190031001A0018001A0018001A0056
:10D9F00018001A0030001A0017001B002F001B002F
:10DA00002F001B002F001B0016001B0016001B0020
:10DA10002F001B0016001B0016001B002F001C000F
:10DA200014022700000000000000000000000000B9
:10DA300000000000000000000000000000000000E6
:10DA400000000000000000000000000000000000D6
:10DA500000000000000000000000000000000000C6
:10DA600000000000000000000000000000000000B6
:10DA700000000000000000000000000000000000A6
:10DA800000000000630017001A00170032001800A1
:10DA9000310019001900190031001A0018001A008D
:10DAA00018001A0017001A0030001B0017001B0096
:10DAB0002F001B002F001B002F001B0016001B0057
:10DAC00016001B002F001B0016001B0014001C007A
:10DAD0002E001C00140227000000000000000000BF
:10DAE0000000000000000000000000000000000036
:10DAF0000000000000000000000000000000000026
:10DB00000000000000000000000000000000000015
:10DB10000000000000000000000000000000000005
:10DB200000000000000000000000000000000000F5
:10DB30000000000000000000630017001B00170039
:10DB40001A001800310019001900190018001900F6
:10DB500031001A0030001A0018001A0030001A00B4
:10DB600017001B002F001B002F001B002F001B00A5
:10DB700016001B0016001B002F001B0016001B00C8
:10DB800016001B002E001C001402270000000000DD
:10DB90000000000000000000000000000000000085
:10DBA0000000000000000000000000000000000075
:10DBB0000000000000000000000000000000000065
:10DBC0000000000000000000000000000000000055
:10DBD0000000000000000000000000000000000045
:10DBE00000000000000000000000000063001700BB
:10DBF000320018001900180031001900180019002F
:10DC000018001A0030001A0030001A0017001A001D
:10DC100030001B0017001B0030001B002F001B00F2
:10DC20002F001B0016001B0016001B002F001B00FE
:10DC300016001C0014001C002E001C0014020D0015
:10DC400000000000000000000000000000000000D4
:10DC500000000000000000000000000000000000C4
:10DC600000000000000000000000000000000000B4
:10DC700000000000000000000000000000000000A4
:10DC80000000000000000000000000000000000094
:10DC90000000000000000000000000000000000084
:10DCA0006300170032001800310019001900190034
:10DCB0001800190018001A0030001A0030001A006D
:10DCC00017001A0030001B0017001B002F001B005C
:10DCD0002F001B002F001B0016001B0016001B004E
:10DCE0002F001B0016001B0014001C002E001C003F
:10DCF00014020D0000000000000000000000000001
:10DD00000000000000000000000000000000000013
:10DD10000000000000000000000000000000000003
:10DD200000000000000000000000000000000000F3
:10DD300000000000000000000000000000000000E3
:10DD400000000000000000000000000000000000D3
:10DD500000000000630017003200180019001900CD
:10DD600019001900190019001900190031001A00D2
:10DD700018001A0018001A0030001A0017001A00C4
:10DD800030001B002F001B002F001B0016001B0083
:10DD900016001B002F001B0016001B0016001B00A6
:10DDA0002F001C00140240000000000000000000D2
:10DDB0000000000000000000000000000000000063
:10DDC0000000000000000000000000000000000053
:10DDD0000000000000000000000000000000000043
:10DDE0000000000000000000000000000000000033
:10DDF0000000000000000000000000000000000023
:10DE00000000000000000000640017001A00170066
:10DE10001A0018001900180019001900190019003B
:10DE200031001A0018001A0018001A0030001A00F9
:10DE300017001A0030001B002F001B002F001B00D2
:10DE400016001B0016001B002F001B0016001B00F5
:10DE500016001B002F001B001602580000000000D7
:10DE600000000000000000000000000000000000B2
:10DE700000000000000000000000000000000000A2
:10DE80000000000000000000000000000000000092
:10DE90000000000000000000000000000000000082
:10DEA0000000000000000000000000000000000072
:10DEB000000000000000000000000073656E645F59
:10DEC0006E756D6265723A206E65775F76616C750E
:10DED00065200020536F6E7920445644204952201B
:10DEE0006465636B20285459504520313529203012
:10DEF0003430383131200D0A0020536F6E792044C0
:10DF00005644204368616E676572206465636B20C8
:10DF1000495220285459504520313829200D0A00F3
:10DF2000534F4E5920313820494E495444454620DC
:10DF30000D0A00534F4E59204952204D4F4445443D
:10DF4000454620617267756D656E74203D200053F3
:10DF50006F6E79204952204E554D42200D0A0053D4
:10DF60004F4E59204952204D4F5645444546206654
:10DF70006C61677320617267756D656E74203D20FA
:10DF800000464F525741524420534F4E5920495258
:10DF9000204D4F564544454620666C6167732061AD
:10DFA0007267756D656E74203D200073656E6469DF
:10DFB0006E6720534F4E5920495220504C41590D05
:10DFC0000A00050C050C050C050C050C050C050CD0
:10DFD000050C050C050C050C050C050C050C050CB9
:10DFE00005520552050C0552050C050C050C050CD7
:10DFF000050C050C050C050C050C04E704E704E70B
:10E0000004E704E704E704E704E704E704E704E7B8
:10E0100004E704E704E704E70B8A065506550B8A74
:10E0200004E704E704E704E704E704E704E704E798
:10E0300004E742434431204D4F4445444546206661
:10E040006C6167732C20617267756D656E7420005A
:10E0500042434431204D6F766544454620666C61ED
:10E0600067732C20617267756D656E742000424382
:10E070004431204544495444454620666C616773E9
:10E080002C20617267756D656E740D0A0023312056
:10E090006770695F6368616E676564203D2000207A
:10E0A000424344312042414E4B31206770695F63E7
:10E0B00068616E67656420646F5F67706920677070
:10E0C00069315F61637469766520206770695F7488
:10E0D000656D70200D0A0020424344312042414EBC
:10E0E0004B31206770695F736F757263652067706D
:10E0F000695F776F726B200D0A003031323334352F
:10E10000363738394142434445460D0A0020002C39
:10E11000003A002D000000FCF8F0E1C2000096007B
:10E120004B00258012C0096068A8E869617020442E
:10E130006576696365204944200069617020446503
:10E14000766963652049442023312000696170208D
:10E150004465766963652049442023322000475096
:10E160004953302020646F5F6770692C20677069A5
:10E170005F74656D702C20677069325F74656D70B7
:10E1800020677069325F616374697665203D2000A5
:10E190002053657420547970652C20576169742070
:10E1A0000D0A000D0A0057726974696E672C2049C8
:10E1B0004E4D4F54494F4E2C204D4F56494E4746D9
:10E1C00057442C207570646174655F6672616D657B
:10E1D0002C206E65775F6672616D65200D0A006E9A
:10E1E000762E726570745F76616C75652C206E7525
:10E1F0006D6265725F6F6666736574206D757465B8
:10E20000645F666C61670D0A004D6F64652C205475
:10E2100069746C652C20436861707465722C20648D
:10E220006D322C20646D330D0A002C6D6F76652ED7
:10E230000D0A002C73746F702E0D0A004243443097
:10E24000206D7574655F636D64206D757465645FC2
:10E25000666C6167204245464F5245206D75746576
:10E260002000206D6F6E695F636D645F6263642080
:10E270000D0A0020667373735F636D645F6263648D
:10E28000200D0A00206E6578745F636D645F6263C1
:10E2900064200D0A0020737973745F636D645F629C
:10E2A0006364200D0A00204243443020646E756D83
:10E2B0005F636D645F626364200D0A0020313D4935
:10E2C000676E6F7265204261642041636B20457206
:10E2D000726F72732066726F6D206465636B2E0DB2
:10E2E0000A00203D5030202438302000203D50319D
:10E2F000202439302000203D50322024413020009D
:10E30000203D5033202442300D0A00313520313475
:10E31000203133203132203131203130203039204A
:10E32000303820202030372030362030352030342F
:10E33000203033203032203031203030200D0A00A0
:10E34000506F72742026205346522076616C75659A
:10E35000733A200D0A0050302050312050322050A6
:10E36000332049452053434F4E2054434F4E2020E5
:10E370005432434F4E20544D4F442054324D4F445D
:10E3800020455432204554323220495020495048CB
:10E390002045430D0A0020200020202000202020BE
:10E3A000002020200020200020200000200020004D
:10E3B000434D4F442043434F4E20200D0A00202060
:10E3C000007077725F6D61782C207077725F636F79
:10E3D000756E74200D0A0062636430207265637389
:10E3E000200D0A00202072656373206E6F706172C9
:10E3F0006D73200D0A00426567696E204572617376
:10E4000065200D0A00457261736520436F6D706C65
:10E41000657465200D0A0050726F6772616D6D69D9
:10E420006E67200D0A004261642050726F6772614E
:10E430006D2061742052414D200053617665204368
:10E440006F6D706C657465200D0A00556E6B6E6F94
:10E45000776E206261756420726174650D0A0041F7
:10E460007661696C61626C653A20203338343030F3
:10E470002C31393230302C20393630302C203438A1
:10E4800030302C202032343030200D0A00203D2046
:10E490004355525F4652414D450D0A00203D2043F1
:10E4A000544C5F4652414D450D0A00203D20434FDC
:10E4B00044455F4652414D450D0A00203D205354CE
:10E4C000445F4652414D450D0A00203D204E4557C0
:10E4D0005F4652414D450D0A00203D20574F524B9B
:10E4E0005F4652414D450D0A00203D20534552499B
:10E4F000414C5F414343554D0D0A002063687070E5
:10E500005F636D645F626364200D0A006263643060
:10E51000206368646E5F636D645F626364200D0AEC
:10E52000006263643020636875705F636D645F626E
:10E530006364200D0A00626364302073656C655F5C
:10E54000636D645F626364200D0A0056432D434D82
:10E5500020537461745F636D64200D0A00706175EF
:10E560007365645F666C616720006D757465645FD8
:10E57000666C616720006D75746D5F6163746976A8
:10E580006520006D7574655F6C696D697420006D40
:10E590007574655F74696D65722000706F6C6C5F77
:10E5A00064656C61792000696E697469616C697A6F
:10E5B000656420000D0A007374696C5F636D6420EC
:10E5C000696E2062636430200D0A0054303330538A
:10E5D000657420543033302064656661756C7473E3
:10E5E000200D0A00543036305365742054303630D4
:10E5F0002064656661756C7473200D0A00543039AF
:10E600003053657420543039302064656661756C10
:10E610007473200D0A005431323053657420543124
:10E6200032302064656661756C7473200D0A005485
:10E630003138305365742054313830206465666158
:10E64000756C7473200D0A0053686F7720746170C5
:10E6500065207061636B2064656661756C747320FE
:10E660000D0A00203D20746F646F5F68656164204F
:10E67000746F646F5F7461696C207374617465207A
:10E68000726573756D655F616464720D0A00206F59
:10E690007574206F6620000D0A004254303120004E
:10E6A000524C30312000425430322000425430333A
:10E6B000200042543034200042543035200042546F
:10E6C00030362000425430372000494E4932200075
:10E6D0004254303820004254303920004254313006
:10E6E0002000425431312000425431322000425443
:10E6F000313320004254313420004254313520005F
:10E7000042543136200053545550004E554C4C0065
:10E710005354444E0053544C4600535452540045F5
:10E720004E54520050524556004E455854005245E2
:10E73000544E004E554D4231004E554D4232004E22
:10E74000554D4233004E554D4234004E554D4235E5
:10E75000004E554D4236004E554D4237004E554DF8
:10E760004238004E554C4C004E554C4C003430381D
:10E7700031392020004243442056432D3136622057
:10E78000436F6E74726F6C2053797374656D3A0DBC
:10E790000A436F7079726967687420313938362D91
:10E7A0003230303420424344204173736F632E2C47
:10E7B00020496E632E200056622D004375727265EB
:10E7C0006E74204465766963653A2000446566612D
:10E7D000756C74206465636B5F7479706520697310
:10E7E0003A20000D0A0000000000588F00000000D1
:10E7F0000000000000004155445849840100000019
:10E8000000000300000042415544653E0100000045
:10E8100000FFFF000000424F4F54499C00000000E1
:10E820000000000000004253455478C20000000080
:10E8300000000000000042543031704A0300000024
:10E8400000000000000042543032713C0300000020
:10E850000000000000004254303371AD030000009E
:10E8600000000000000042543034721E030000001B
:10E8700000000000000042543035728F0300000099
:10E880000000000000004254303673000300000016
:10E890000000000000004254303773710300000094
:10E8A00000000000000042543038745303000000A0
:10E8B0000000000000004254303974C4030000001E
:10E8C00000000000000042543130753503000000A4
:10E8D0000000000000004254313175A60300000022
:10E8E000000000000000425431327617030000009F
:10E8F000000000000000425431337688030000001D
:10E900000000000000004254313476F9030000009A
:10E9100000000000000042543135776A0300000017
:10E920000000000000004254313677DB0300000095
:10E9300000000000000042555453784C03000000D2
:10E940000000000000004348415057F701C000009C
:10E950004000000000004348444E66EB0100000008
:10E960000000030000004348505066C10100000051
:10E970000000FF00000043485550671501000000EB
:10E98000000003000000434C4552552100000000E8
:10E990000000000000004445424749E40100000037
:10E9A00000000A0000004445434B6FA20100000034
:10E9B0000000FF0000004445434E6F7A0100000054
:10E9C0000000FF0000004449535053D701000000ED
:10E9D0000000FF000000444E554D5730010000007C
:10E9E00000FFFF00000044554D504A320200000075
:10E9F00000FFFF0000004543484F4ABA01000000F5
:10EA000000000100000045434F464AE400000000BA
:10EA100000000000000045434F4E4AEA000000009D
:10EA2000000000000000454E545256500000000007
:10EA30000000000000004552523F4BFF0100000063
:10EA40000000FF000000455252414B7B01000000D6
:10EA50000000FF000000455252464BAC0100000090
:10EA60000000FF00000046414354499C00000000A4
:10EA7000000000000001464657444C5A01C0000007
:10EA8000400000400000464C445656FA01C00000C9
:10EA90004000000000004652414D4D4701C00000BB
:10EAA000400000000000465245514D0601000000A4
:10EAB0000000FF00000046524D535768010000005F
:10EAC00040000000000047444C594DA701000000E1
:10EAD0000000FF000000474C49544E9B010000001D
:10EAE0000000FF000000475255506FFD010000007C
:10EAF0000000FF0000004754313053F501000000D2
:10EB00000000FF00000048454C504ECE01000000C0
:10EB1000000000000000494150314885010000001C
:10EB200000FFFF000000494E493273E2030000007D
:10EB3000000000000000494E49544ECF0000000084
:10EB4000000000000000494E505450080100000031
:10EB50000000FF0000004C41424C5009030000003F
:10EB60000000000000004C415354502400000000FD
:10EB70000000000000004C4249546F780100000082
:10EB80000000020000004C454E4450E80000000028
:10EB90000000000000004C49544550900100000066
:10EBA0000000FF0000004C4F4F50510C01000001CD
:10EBB0004000000000004C4F5554508F01000000F1
:10EBC0000000FF0000004D454E5555FF00000000BD
:10EBD0000000000000004D49534351640000000054
:10EBE0000000000000004D4F4430524701C00000BB
:10EBF0004000000000004D4F4431525701C000005A
:10EC00004000000000004D4F4445526700000000E6
:10EC10000000000000004D4F4446539701000000E3
:10EC20000000FF0000004D4F4E49553C0000000021
:10EC30000000000000004D4F5645537700000000D3
:10EC40000000000000004D4F564653B70100000081
:10EC50000000FF0000004D55544554950100000090
:10EC60000000010000004D55544D541301000000F8
:10EC70004000000000004E45585455900000000030
:10EC80000000000000004E4F414B585A01C00000E8
:10EC90004000000000004E554C4C588F0000000012
:10ECA0000000000000004E554D4257F701C0000023
:10ECB0004000000000004E554D53583001C0000088
:10ECC0004000000000004F46535458AE01C0000001
:10ECD0004000000000004F4B4F4B5650000000001A
:10ECE0000000000000005041555358AF01C0000023
:10ECF00040000000000050434C52596302000000E5
:10ED00000000FF0000005045454B59D102000000B3
:10ED100000FFFF00000050494E5359F10000000071
:10ED2000000000000000504C41595C16010000003A
:10ED3000400000400000504D41585EF501000000C9
:10ED40000000FF000005504F4B455C790280000039
:10ED50007FFFFF000000504F4C4C5C8D0100000015
:10ED6000400000400000504F52545CC500000000BD
:10ED7000000001000000504F57525F4001000000AA
:10ED80000000014000005052414D5F64020000004D
:10ED90000000FF0000005052455655BA0000000028
:10EDA00000000000000050524D545F82030000003C
:10EDB00000000000000050524F4C5FA20100000014
:10EDC00040000000000050524F4D5FCC0200000098
:10EDD00000FFFF0000005053455460850200000012
:10EDE0000000FF0000005232333267690300000068
:10EDF0000000000000005243565460F30100000080
:10EE000000FFFF00000052444C5961270100000040
:10EE100000FFFF000000524543536159010000000C
:10EE20004000004000005245473061DA01C0000058
:10EE300040000000000052454731620601C000005A
:10EE400040000000000052454A45623200000000C8
:10EE500000000000000052455054624D01000000C7
:10EE60000000FF0000005245544E561A00000000FA
:10EE700000000000000052455744629B01C00000A2
:10EE8000400000C00000524C303170CB0300000045
:10EE9000000000000000524C534563470000000092
:10EEA0000000000000005253554D56350000000090
:10EEB0000000000000005341444463620000000071
:10EEC000000000000000534156456421000000008E
:10EED0000000000000005345454B4AF102C000000D
:10EEE00040000000000053454C45673F0000000013
:10EEF00000000000000053455155637800000000F9
:10EF0000000000000000534C4F5765DF0000000078
:10EF1000000000000000534D505465FA000000004E
:10EF20000000000000005352434869420100000005
:10EF300000000A00000053544132687A00000000CB
:10EF40000000000000005354415467870100000096
:10EF50000000FF0000005354444E56A9000000007A
:10EF600000000000000053544550690801000000F3
:10EF70004000000000005354494C698E010000001D
:10EF80004000000000005354494D69E201000000B8
:10EF90000000FF00000053544C4656C4000000001F
:10EFA00000000000000053544F506A0C01000000A4
:10EFB0004000000000005354525456DF000000008F
:10EFC00000000000000053545550568E0000000011
:10EFD000000000000000535749546A7E0100000001
:10EFE0000000FF0000005359535455D500000000A5
:10EFF00000000000000054414C4B6BBB01000000BE
:10F00000000002000001544553546BBC0300000093
:10F01000400000000001544852446BBD0100000054
:10F0200000000100000054494D456BE7020000005C
:10F0300000FFFF0000005449544C57150000000029
:10F04000000000000000544D454E57150000000020
:10F05000000000000000544F444F6C4401000000C9
:10F060000000FF00000054594D456E5F0000000095
:10F0700000001E000000545950456ED101000000F0
:10F0800000001E000000554E49546F790100000039
:10F090000000FF000000555330307ACA0300000022
:10F0A000000000000000555330317B600300000079
:10F0B0000000000000005553415665280000000084
:10F0C000000000000000564552537BF6000000008F
:10F0D000000000000000565354447D9201C000001F
:10F0E00000001E00001E574149547DD5000000005D
:10F0F00000000000000057454E447DDC0000000089
:10F100000000000000005A45524F7DE3000000005F
:10F11000000000000000FFFFFFFF588F000000000C
:10F12000000000000000556E6B6E6F776E206572F8
:10F13000726F722020202020202000556E6B6E6F91
:10F14000776E20636F6D6D616E642020202020003B
:10F15000417267756D656E7420526571756972656F
:10F160006420202000426164206865782061726715
:10F17000756D656E742020202000417267756D6585
:10F180006E742072616E6765206572726F720055D1
:10F190006E6B6E6F776E20446973632076616C7559
:10F1A0006520200053656E6420746F20446973638A
:10F1B000206572726F7220200044697363206C694D
:10F1C00064206F70656E2E20202020202000507259
:10F1D00065726F6C6C20746F6F20736D616C6C2046
:10F1E000202000417267756D656E74206E6F74200B
:10F1F000616C6C6F77656400556E657870656374DB
:10F200006564206D6F74696F6E2E2020004E414B37
:10F210002066726F6D20446973632E2020202020A9
:10F220002000556E6B6E6F776E20446973632065A6
:10F2300072726F722020004672616D65206E6F746D
:10F2400020666F756E642E20202020004672616D4E
:10F250006520646F6573206E6F74206578697374C0
:10F2600000504C522054797065206E6F7420617686
:10F2700061696C2E20005265747279206C696D6929
:10F28000742065786365656465640046756E6374B3
:10F29000696F6E2E204E6F7420417661696C2E006E
:10F2A000556E6578706563746564204D6F74696F21
:10F2B0006E202020004672616D6520507265762EAA
:10F2C000205265636F726465640042616420566910
:10F2D00064656F206F722053796E632E2020004D7D
:10F2E000697373656420437574204F75742041649D
:10F2F000727373004C6F63616C20456469742045C0
:10F3000072726F722E202020004E6F204564697447
:10F310002054797065205365742E20202000436F9F
:10F320006C6F72204672616D696E67204572726FF4
:10F33000722E00544243204E6F74204163746976EC
:10F34000652E2020202020005461706520697320E4
:10F35000456A65637465642E2020202000506F7715
:10F360006572206973206F66662E20202020202081
:10F3700020004465636B2054797065204E6F7420C3
:10F380005365742E20200042616420436C6F636BD0
:10F3900020426174746572792E20200042616420DD
:10F3A00041434B2076616C75652E20202020202063
:10F3B000004E6F204164647265737320436F64650F
:10F3C0002E202020200053657269616C2074696DC5
:10F3D000656F75742E2020202020004469736320FF
:10F3E0004175746F20506C6179206572726F720084
:10F3F0004469736320536561726368204572727259
:10F400006F722E200042616420534D5054452043BA
:10F410006F64652E2020202020004E6F20667261D0
:10F420006D65206D6F74696F6E2E20202020004264
:10F4300061642054696D6520436F6465202020203D
:10F4400020202000F126F13BF150F165F17AF18F97
:10F45000F1A4F1B9F1CEF1E3F1F8F20DF222F237B5
:10F46000F24CF261F276F28BF2A0F2B5F2CAF2DF60
:10F47000F2F4F309F31EF333F126F126F126F348F3
:10F48000F35DF372F126F126F126F126F126F1263D
:10F49000F126F126F126F126F387F126F126F12651
:10F4A000F126F126F126F126F126F126F126F126A4
:10F4B000F126F126F126F126F126F126F126F12694
:10F4C000F126F126F126F126F126F126F126F12684
:10F4D000F126F126F126F126F126F126F126F12674
:10F4E000F126F126F126F126F126F126F126F12664
:10F4F000F126F126F126F126F126F126F126F12654
:10F50000F126F126F126F126F126F126F126F12643
:10F51000F126F126F126F126F126F126F126F12633
:10F52000F126F126F126F126F126F126F126F12623
:10F53000F126F126F126F126F126F126F126F12613
:10F54000F126F126F126F126F126F126F126F12603
:10F55000F126F126F126F126F126F126F126F126F3
:10F56000F126F126F126F126F126F126F126F126E3
:10F57000F126F126F126F126F126F126F126F126D3
:10F58000F126F126F126F126F126F126F126F126C3
:10F59000F126F126F126F126F126F126F126F126B3
:10F5A000F126F126F126F126F126F126F126F126A3
:10F5B000F126F126F126F126F126F126F126F12693
:10F5C000F126F126F126F126F126F126F126F12683
:10F5D000F126F126F126F126F126F126F126F12673
:10F5E000F126F126F126F126F126F126F126F12663
:10F5F000F126F126F126F126F126F126F126F12653
:10F60000F126F126F126F126F126F126F126F12642
:10F61000F126F126F126F126F126F126F126F12632
:10F62000F126F126F126F126F126F126F126F12622
:10F63000F39CF3B1F3C6F3DBF3F0F405F41AF42F03
:10F64000F126F1266469676974203D202000646911
:10F650006769745F73756D203D202000537461727B
:10F6600074696E672075702E2E2E200D0A00696E4B
:10F67000697469616C697A6564203D20006E762E3C
:10F68000627574746F6E5F736967203D200020504F
:10F690006C73207374616E642062792E2E2E200D9F
:10F6A0000A002063616C6C206C697465200D0A008F
:10F6B00020626164206E762E627574746F6E5F7363
:10F6C00069673A20496E697420427574746F6E736D
:10F6D0002E2E2E200D0A00206D61785F6465636B0D
:10F6E00073203D2000206E762E6465636B5F747915
:10F6F0007065203D20006465636B5F7479706520E0
:10F700003D20002053657420547970652044656362
:10F710006B2054797065203D2000204465636B2088
:10F7200054797065203D20002044656661756C74D5
:10F73000204465636B2054797065203D2000494E5C
:10F74000493220697320757365722070676D2E20B1
:10F750000D0A004E4F5720696E697469616C697AB1
:10F760006564203D200042434430206770695F6338
:10F7700068616E67656420646F5F6770692C2067DD
:10F7800070695F696E2C206770695F74656D702C9D
:10F7900020677069315F616374697665203D200D73
:10F7A0000A00424344302042544E2031200D0A00CA
:10F7B000424344302042544E2032200D0A0042433E
:10F7C00044302042544E2033200D0A00424344303E
:10F7D0002042544E2034200D0A004243443020423F
:10F7E000544E2035200D0A00424344302042544EEE
:10F7F0002036200D0A00424344302042544E203728
:10F80000200D0A00424344302042544E2038200D3F
:10F810000A00424344302042544E2039200D0A0051
:10F82000424344302042544E203130200D0A0042E1
:10F830004344302042544E203131200D0A004243CF
:10F8400044302042544E203132200D0A00424344BD
:10F85000302042544E203133200D0A0042434430C0
:10F860002042544E203134200D0A004243443020BF
:10F8700042544E203135200D0A004243443020428C
:10F88000544E203136200D0A00524547305245472C
:10F89000314F46464F4E464F524556455254686585
:10F8A0007365206172652074686520617661696C9A
:10F8B00061626C6520636F6D6D616E64733A0D0AF1
:10F8C000002A2A2A2A0012BFCE800000C000004071
:10F8D000000020F580278D002782E0000000000056
:10F8E0000100000200000300001E000400000800E8
:10F8F000000708466163746F7279205265736574FE
:10F90000202830290D0A00855483855582E0F8A30C
:10F91000E0F9A3E0FA85568385578275F000E06828
:10F9200030E70375F003E0C39840157018A3E0C3F7
:10F9300099400D7010A3E0C39A400570087400222E
:10F94000740165F022740265F02285548385558226
:10F95000E0F8A3E0F9A3E0FA855683855782E8F042
:10F96000A3E9F0A3EAF022855483855582E0F8A349
:10F97000E0F9A3E0C39401FAE99400F9E894008562
:10F980005483855582F0A3E9F0A3EAF022855683DB
:10F99000855782E0A3F8E0A3F9E0FA855483855502
:10F9A000827C987D967E8012FA60E55B2430F0A31D
:10F9B0007C0F7D427E4012FA60E55B2430F0A37C30
:10F9C000017D867EA012FA60E55B2430F0A37C0006
:10F9D0007D277E1012FA60E55B2430F0A37C007D69
:10F9E000037EE812FA60E55B2430F0A37C007D0022
:10F9F0007E6412FA60E55B2430F0A37C007D007E1B
:10FA00000A12FA60E55B2430F0A3EA2430F0A37414
:10FA100000F022855483855582E0F8A3E0F9A3E045
:10FA20002401FAE93400F9E83400855483855582CD
:10FA3000F0A3E9F0A3EAF022855483855582E0F82B
:10FA4000A3E0F9A3E0F42401FAE9F43400F9E8F4BE
:10FA50003400855483855582F0A3E9F0A3EAF022AF
:10FA60008859895A8A5B780079007A007F19C3CA5D
:10FA70009ECAC99DC9C89CC8401ED3C55B33C55B1F
:10FA8000C55A33C55AC55933C559CA33CAC933C90A
:10FA9000C833C8DFD902FABCCA2ECAC93DC9C83C9E
:10FAA000C8C3C55B33C55BC55A33C55AC55933C5D1
:10FAB00059CA33CAC933C9C833C8DFB2C813C8C9A1
:10FAC00013C9CA13CA2210AF028003D38001C392A4
:10FAD00011900925E0B4010A900925E4F0856299A6
:10FAE000802C900DABE0FEA3E0FF0FBF00010E7C69
:10FAF000037DFFEE521CEF521D900DABECF0A3ED19
:10FB0000F08C1E8D1F9009A912FF02E562F0A21170
:10FB100092AF22856383856482E493601485638356
:10FB2000856482E493F56212FAC6786312FF42801C
:10FB3000E222308C1EB28290106CE0F58C90106D39
:10FB4000E0F58A900DC8E0B402077443F56212FA3A
:10FB5000C68056D282901073E0F8A3E0901071C86E
:10FB6000F0A3C8F0A205920490000CE090106FF092
:10FB700090106EE4F090107112FEDFE493FE7401B9
:10FB800093FF12FF3A90106CEEF0A3EFF090106C20
:10FB9000E0F58C90106DE0F58AD28C900DC8E0B441
:10FBA00002077453F56212FAC690106EE004F090EA
:10FBB000106EE0FE90107112FEDFEE12FEA6E493CE
:10FBC000FE740193FF12FF3A90106CEEF0A3EFF079
:10FBD000EF4E703890106FE0600690106FE014F0F8
:10FBE00020040690106FE0601F90106EE4F09010FB
:10FBF0007112FEDFE493FE740193FF12FF3A90103E
:10FC00006CEEF0A3EFF08004C28CC28222BC000F25
:10FC1000BE0008ED8FF084FFADF022E4FEFF22BEAF
:10FC2000000DEF60FE54F0606F20E70302FCC3EAB2
:10FC3000C0E0EBC0E078017A0075F001EE20E7103B
:10FC4000EF25E0FFEE33FE0AC5F023C5F030E7F004
:10FC5000EA5407F9096A7A007B00600108C3EC9E48
:10FC600040167004ED9F4010ED9FFDEC9EFCE5F00A
:10FC7000CA4ACA03F5F08005E5F003F5F0C3EE13B8
:10FC8000FEEF13FFD9D77908CACBCAD8D0EAFEEB6A
:10FC9000FFD0E0FBD0E0FA22EC8FF084FCED54F0D2
:10FCA00045F0C48FF084FEEDC454F045F0C48FF0ED
:10FCB00084FDEEC4FE54F02DFFEE540F3CFEADF07B
:10FCC0007C0022790078008FF0EC7E0820E70DC3DD
:10FCD000CD33CD33C933C9C833C8DEF08449F9E523
:10FCE000F08FF0BE00E6FD7C00E9FFE8FE22AC5C90
:10FCF000AD5DAE5EAF5F0560056102FD168D828C65
:10FD000083E493A3AD82AC838F828E83F8E0687026
:10FD100010A3AF82AE83D561E4D560E17EFF7FFFA3
:10FD200022C3EF955FFFEE955EFE22AC5CAD5DAE4B
:10FD30005EAF5F0560056102FD528D828C83E0A39A
:10FD4000AD82AC838F828E83F8E0687010A3AF829F
:10FD5000AE83D561E5D560E27EFF7FFF22C3EF95DC
:10FD60005FFFEE955EFE224669726D7761726520D7
:10FD700056657273696F6E204672692041756720FF
:10FD800032302031303A33383A3033203230303468
:10FD9000200D0A00AE5CAF5DAC5EAD5F0560056135
:10FDA00002FDB88F828E83E493A3AF82AE838D82EF
:10FDB0008C83F0A3AD82AC83D561E8D560E522AE3B
:10FDC0005CAF5DAC5EAD5F0560056102FDE28F82F8
:10FDD0008E83E0A3AF82AE838D828C83F0A3AD824D
:10FDE000AC83D561E9D560E622C0E0C0F0C083C035
:10FDF00082C0D075D010121F45D0D0D082D083D011
:10FE0000F0D0E032C0E0C0F0C083C082C0D075D076
:10FE10000812107CD0D0D082D083D0F0D0E032E471
:10FE200093F5F0740193800BE0F5F0A3E080048675
:10FE3000F008E6C0E0C0F02200FCF8F0E1C20000EB
:10FE400096004B00258012C0096068A8E832FE4D7C
:10FE5000EF8DF0A4F9A8F0EF8CF0A428F8EE8DF067
:10FE6000A428FEE9FF22600D782B02FE7000783096
:10FE7000D8FED5E0F822EEC0E07E0012FC0DEFFDCA
:10FE8000EEFCD0E0FE227E0012FED1EF2582F5824C
:10FE9000EE3583F583227E0012FE50EF2582F58237
:10FEA000EE3583F5832225E050020583258250023A
:10FEB0000583F58222A3E014F0B4FF0612FF0DE0E3
:10FEC00014F022048007C3CE13CECF13CFD5E0F6B3
:10FED00022F88FF0A4FFE5F0CE88F0A42EFE22E0F9
:10FEE000C0E0A3E0F582D0E0F58322EEC0E07E0022
:10FEF00012FC0DD0E0FE22EF2582F582EE3583F56F
:10FF00008322E5822FF582E5833EF583220582D5A3
:10FF1000820215831582222582F5825002058322F2
:10FF2000E493F608740193F62275816875D0000297
:10FF30009FE9C3EF9DFFEE9CFE22E4C39FFFE49E7A
:10FF4000FE220806B600021806220816B6FF02189E
:10FF50001622FFFFFFFFFFFFFFFFFFFFFFFFFFFF77
:10FF6000FFFFFFFFFFFFFFFFFFFFFFFFFFFFFFFFA1
:10FF7000FFFFFFFFFFFFFFFFFFFFFFFFFFFFFFFF91
:10FF8000FFFFFFFFFFFFFFFFFFFFFFFFFFFFFFFF81
:10FF9000FFFFFFFFFFFFFFFFFFFFFFFFFFFFFFFF71
:10FFA000FFFFFFFFFFFFFFFFFFFFFFFFFFFFFFFF61
:10FFB000FFFFFFFFFFFFFFFFFFFFFFFFFFFFFFFF51
:10FFC000FFFFFFFFFFFFFFFFFFFFFFFFFFFFFFFF41
:10FFD000FFFFFFFFFFFFFFFFFFFFFFFFFFFFFFFF31
:10FFE000FFFFFFFFFFFFFFFFFFFFFFFFFFFFFFFF21
:10FFF000FFFFFFFFFFFFFFFFFFFFFFFFFFFFFFFF11
:00000001FF
